:020000040800F2
:10000000083F012001040008250400082704000817
:10001000290400082B0400082D040008000000003B
:100020000000000000000000000000002F04000895
:100030003104000800000000330400083504000803
:100040001B0400081B0400081B0400081B04000814
:100050001B0400081B0400081B0400081B04000804
:100060001B0400081B0400081B0400081B040008F4
:100070001B0400081B0400081B0400081B040008E4
:100080001B0400081B0400081B0400081B040008D4
:100090001B0400081B0400081B0400080189000859
:1000A0001B0400081B0400081B0400081B040008B4
:1000B000A50200081B0400081B0400081B0400081C
:1000C0001B0400081B0400081B0400081B04000894
:1000D0001B0400081B0400081B0400081B04000884
:1000E0002B8900081B0400081B0400081B040008DF
:1000F0001B0400081B0400081B0400081B04000864
:100100001B0400081B040008C50200081B040008AB
:100110001B0400081B0400081B0400081B04000843
:100120001B0400081B0400081B0400081B04000833
:100130001B0400081B0400081B0400081B04000823
:100140001B0400081B0400081B0400081B04000813
:100150001B0400081B0400081B0400081B04000803
:100160001B0400081B0400081B0400081B040008F3
:100170001B0400081B0400081B0400081B040008E3
:100180001B0400081B040008DFF80CD009F02CFE4B
:100190000048004755030008083F012030B589B0EA
:1001A00000F027FA00F0CAF97A497B4800F038FAE3
:1001B00003A804F091FD4FF48270ADF80E004FF4E7
:1001C0000070ADF816003020744CADF8180003A98B
:1001D000204604F057FD0021204604F092FD012145
:1001E000204604F085FD28206D4CADF8180003A9C9
:1001F000204604F047FD0021204604F082FD012145
:10020000204604F075FD6748016867A009F080FE8C
:1002100000244CF25030ADF800400190ADF8084099
:10022000ADF802408DF80A406946800604F08AFC69
:100230000121880704F0C1FC6248634DADF800401D
:100240000190ADF80840ADF802408DF80A406946CB
:10025000284604F077FC01221146284604F0B6FC3B
:100260000121284604F0A9FC32208DF8200001204D
:100270008DF823008DF821408DF8224008A804F065
:10028000BFFC601F04F0EFFC4FF0E02045F20721B7
:100290004161016941F0030101614CA009F038FEA0
:1002A00009B030BD10B50121880704F097FC002883
:1002B00008BF10BD0121880704F09BFC49490120BB
:1002C000087510BD10B5404C0121204604F086FC95
:1002D000002808BF10BD0121204604F08AFC2088B8
:1002E00020F00100208040490C20088310BD3F48C9
:1002F00010B58168491C8160016800291CBF491E36
:1003000001604168491C4160642928BF01F028FE52
:100310002148008810F0200F08D0354800881B289D
:1003200004D13048817B41F08001817331480168FC
:10033000002908BF10BD491E016018BF10BD102064
:100340002D49887710BD29498A688B689B1A83429A
:10035000FBD37047FFF722FF00F09EFA00F019FA76
:1003600000F0C1FC254C0120207000F012FB00F0D1
:100370007EFF00F0B8FC0020207001F03BF800F098
:1003800007FE01F0FCFE00F003FE002008F062F81A
:10039000FBE7000040420F0000140140003800401D
:1003A000003001400C0000200D0A53797374656D14
:1003B000206672657175656E63793A202564487AA6
:1003C0000D0A000000453300000C00405344313555
:1003D000343120494E495420434F4D504C455445EB
:1003E0000D0A00002405012000000240000000204A
:1003F0000414014068040020780501202600002034
:100400000648804706480047FEE7FEE7FEE7FEE7AE
:10041000FEE7FEE7FEE7FEE7FEE7FEE73904000839
:10042000890100087047FEE7FEE7FEE7FEE7704738
:1004300070477047FFF75BBF374882B0016841F4EF
:10044000700101603548016841F0010101603449E3
:1004500000230B60026822F4102222F080720260F6
:1004600000F1040C2F4ACCF80020026822F480220C
:1004700002600A1D136001930093026842F4803207
:100480000260026802F400320092019A521C01924A
:10049000009A1AB9019AB2F5A04FF2D1026812F48B
:1004A000003F08BF009331D0012200921E4A13681A
:1004B00043F0805313601D4A136843F440431360B4
:1004C0000A680A600A6842F400420A600A6842F454
:1004D000A0520A60164ACCF80020026842F08072EE
:1004E0000260026812F0007FFBD0124A40F20570F1
:1004F0001060086820F003000860086840F00200FF
:100500000860086800F00C000828FAD10A494FF08A
:100510000060086002B0704788ED00E000380240DB
:10052000083802401030002440380240007000407B
:1005300019544007003C024008ED00E070B586B059
:100540000025464C03208DF8050020682E46D0B1CA
:1005500005EB450104EB81008288009282798DF8D9
:100560000420C2798DF80620007A8DF8070054F82F
:100570002100694604F092F96D1C05EB450054F822
:1005800020000028E4D1374835490162364A11601D
:10059000364A4FF0084111600F21416128208DF843
:1005A000100001208DF813008DF811608DF8126095
:1005B00004A804F025FB17208DF8100004A804F00F
:1005C0001FFB2B494FF4405008602A4A43F2333155
:1005D0001160111D086028494FF484500860091DFE
:1005E0004FF41F400860254949F68070086006B046
:1005F00070BD10B5002004F0A3F9002004F0A7F9A5
:10060000012144F2090004F0FEF9012145F2210024
:1006100004F002FA0121BDE810401F2004F0EAB9FD
:1006200030B50C4685B00546002104F069FA00217A
:10063000ADF80810ADF804100C20ADF80610ADF8B8
:100640000C10ADF80A0000946946284604F0FEF943
:100650000121284604F054FA05B030BDE0A300089B
:1006600000005055000002402404024020080240CF
:100670000C38014010380140083C0140003C01406A
:1006800070B50C4640F0800500224FF48061FE4EAC
:10069000304604F04FF9B114304604F049F92946C8
:1006A000FA4D284604F036FBA914304604F03EF912
:1006B00044F0400400222915304604F03BF9A91407
:1006C000304604F035F92146284604F023FBA914EE
:1006D0003046BDE8704004F029B92DE9F05F0646C8
:1006E000107815468A4600281ABFE74FDFF89CB3FA
:1006F000BDE8F09FF0B215F8012B761C203A02F00D
:10070000FF080AF0FF01B8F1600F28BF4FF01F0883
:1007100000EB40004006000EFFF7B2FFDC4908EB9B
:100720008800002400EB0108012218F804909102CF
:10073000384604F0FFF84FF48051384604F0F8F8DA
:100740004946584604F0E6FA4FF48051384604F022
:10075000EDF8641C052CE7D30122002491023846F1
:1007600004F0E8F84FF48051384604F0E1F82146EF
:10077000584604F0CFFA4FF48051384604F0D6F8CA
:100780000E2E28BFBDE8F09F28780028B2D1BDE822
:10079000F09F2DE9F04100210846FFF771FFBA4EA6
:1007A000BA4F0024012200259102304604F0C2F81D
:1007B0004FF48051304604F0BBF82946384604F027
:1007C000A9FA4FF48051304604F0B0F8641CB4F537
:1007D000FC7FE7D3BDE8F0812DE9F0410146002020
:1007E000FFF74EFFA84EA94F0024012200259102D9
:1007F000304604F09FF84FF48051304604F098F8EA
:100800002946384604F086FA4FF48051304604F009
:100810008DF8641C542CE8D3BDE8F08170B59A4E75
:100820000446212500224FF48061304604F082F80E
:10083000B114304604F07CF82946944D284604F063
:1008400069FAA914304604F071F844F080040022DB
:100850002915304604F06EF8A914304604F068F803
:100860002146284604F056FAA914304604F05EF8F2
:10087000202400226101304604F05CF8E10130469A
:1008800004F056F82146284604F044FAE1013046C7
:10089000BDE8704004F04AB870B57B4D4FF400617C
:1008A000284604F045F80A20FFF74DFDE9142846D4
:1008B00004F03CF8212400222915284604F03AF8D7
:1008C000A914284604F034F8704E2146304604F04E
:1008D00021FAA914284604F029F8B4240022291585
:1008E000284604F027F8A914284604F021F82146E8
:1008F000304604F00FFAA914284604F017F804242F
:1009000000222102284604F015F8A102284604F02E
:100910000FF82146304604F0FDF9A102284604F004
:1009200005F8142400222915284604F003F8A91418
:10093000284603F0FDFF2146304604F0EBF9A914E8
:10094000284603F0F3FF202400226101284603F02B
:10095000F1FFE101284603F0EBFF2146304604F0A9
:10096000D9F9E101284603F0E1FF0C240022291502
:10097000284603F0DFFFA914284603F0D9FF2146DB
:10098000304604F0C7F9A9142846BDE8704003F0CA
:10099000CDBF2DE9F0473F483B4DDFF8F0A0007890
:1009A00084B000280EBF00240026DFF8EC9052D05F
:1009B000F4B29A2700224FF48061284603F0BAFF70
:1009C0004FF48051284603F0B3FF3946504604F0F7
:1009D000A1F94FF48051284603F0A8FF44F04004E9
:1009E00000224FF48061284603F0A4FF4FF48051A9
:1009F000284603F09DFF2146504604F08BF94FF442
:100A00008051284603F092FF002406EB4617381960
:100A1000012219F800809102284603F08BFF4FF461
:100A20008051284603F084FF4146504604F072F995
:100A30004FF48051284603F079FF641C212CE6D343
:100A4000761C052EB4D315A205210020FFF745FE24
:100A500004B0BDE8F087E1B20020FFF711FE0026E8
:100A6000012200279102284603F064FF4FF48051D1
:100A7000284603F05DFF3946504604F04BF94FF429
:100A80008051284612E00000000402400038004077
:100A900054A500082600002034A70008434F4D4D00
:100AA0004F444F52452031353431000003F03EFFB2
:100AB000761C542ED4D3641C052CCCD35448007817
:100AC000B8B1002153A20846FFF707FE554D002498
:100AD00055A155F82420684609F02AFA6A46611C97
:100AE0000020FFF7FAFD641C032CF1D304B0BDE82D
:100AF000F08700214FA20846FFF7EFFDE6E7203917
:100B0000C9B2602928BF1F2101EB81034D494E4A1C
:100B100011F803C002F800C0194410444B78437028
:100B20008A788270CA78C270097901710021417196
:100B300070472DE9F04188460746002409F004F982
:100B400006464FF49071404809F0E7F818F0100F8E
:100B500004D03C210020FFF7D2FF06240025002E00
:100B600007D9795D2046FFF7CAFFA41D6D1CAE4270
:100B7000F7D818F0100F04D03E212046FFF7BFFF32
:100B8000A41D20212046FFF7BAFFA01D2021FFF75A
:100B9000B6FF0C3420212046FFF7B1FFA01D80B224
:100BA000BDE8F0812DE9F04700EB40004006984693
:100BB0001546000EFFF764FDDFF88C90234FDFF839
:100BC00090A00024288809EB04010122465C9102D0
:100BD000384603F0AFFE4FF48051384603F0A8FECC
:100BE0003146504604F096F84FF48051384603F0F1
:100BF0009DFE641C482CE5D32888A8F14801401CC0
:100C000080B228808842A4BF00202880BDE8F087F9
:100C100024000020545249414C2056455220312E88
:100C200032000000A4040120202020253038582064
:100C30002020000053455249414C20232056312E9C
:100C40003200000054A50008900800200004024073
:100C50000038004010B510282BD2DFE800F0080A59
:100C60000C0E10121416181A1C1E20222426DCA0AA
:100C70001CE0DCA01AE0DEA018E0DFA016E0E1A096
:100C800014E0E2A012E0E3A010E0E6A00EE0E7A08E
:100C90000CE0E8A00AE0EBA008E0EEA006E0F1A07E
:100CA00004E0F3A002E0F6A000E0F9A009F030F9BA
:100CB00003E00146F9A009F02BF9BDE81040FCA0C3
:100CC00009F026B910B5FB4C2021204603F025FF82
:100CD00020B12046BDE8104003F01BBFF6490022BA
:100CE00048794A7110BDF54830B4F54BF5490068B4
:100CF0001860F54A0968596012689A60F34BEE4C27
:100D000043435B1C01EB1341F04B08444B435B1C1A
:100D100002EB1342EE491044484000216061EB4A67
:100D2000491C5043401C1029F9D3EA4AEA4B0021E0
:100D30006061DFF898C3555C00FB0CF0401C85EA4D
:100D4000106C03F801C0491C1029F2D3606130BC5B
:100D5000704700B58BB0E1A002F035FF0B22E1A196
:100D6000684602F0E7FA00281CBF0BB000BD09ABD3
:100D70004FF48072DF49684602F051FC09AB4FF432
:100D80000072DD49684602F04AFC09AB0422DB49E7
:100D9000684602F044FC09AB0122D949684602F0DA
:100DA0003EFC09AB0222D749684602F038FC09AB89
:100DB00041F29A02D449684602F031FC09AB0122A3
:100DC000D249684602F02BFC684602F064FD0BB085
:100DD00000BD70B5CE4D0446D5F8580238B14FF07D
:100DE000FF3008F002FE05F5167002F054FD2146B2
:100DF00005F5427008F0BDFFFFF7CBFCFFF7C9FD1A
:100E00000520FFF7E9FC204608F0EAFE30B1224653
:100E1000BDE8704005210020FFF75FBCBDE87040D1
:100E20000521BC4A0020FFF758BC2DE9F0410E46D1
:100E3000074608F089FF0446042828BF032507D386
:100E4000641E385D08F04AFF715DC0B2814202D075
:100E50000020BDE8F0816D1EF2D20120BDE8F081D6
:100E60002DE9F84FACA205210020FFF736FCA84E73
:100E700000205EA1C6F8A40206F50D7002F037FE50
:100E80000090FFF7E7FE06F57B40C6F894022820A5
:100E9000C6F8980206F51F7106F50D7002F055FEB2
:100EA000002804BF06F23E3844F23F7966D100BF05
:100EB000D6F84402002861D0D6F8A41296F884022D
:100EC00006F2852A01F8080096F88402C0F300179C
:100ED0000FF2542B504608F037FF0446042828BF71
:100EE00003250CD3641E1AF8040008F0F7FE1BF863
:100EF0000510C0B2814202D16D1EF3D2012706F265
:100F0000852A0FF22C2B504608F01EFF04460428B9
:100F100028BF03250CD3641E1AF8040008F0DEFE77
:100F20001BF80510C0B2814202D16D1EF3D200E061
:100F3000BFB1D6F8A402D6F8941200EB800006EBFD
:100F4000C000484408F015FFD6F8A41206EB0110C3
:100F5000491CC6F8A41200F23F7006F2852108F081
:100F600008FFD6F8A402B0F5806F07D206F51F710E
:100F700006F50D7002F0E9FD002899D00520FFF775
:100F80002BFC009800280CBF01200020BDE8F88F42
:100F90002DE9F0414A4898B081680091D0E90023DA
:100FA00065A10CA808F0C4FF434E01200246B070B2
:100FB00000250CA901A802F0BDF90027002804BFF4
:100FC0000024DFF814810AD114F0010F08BF0025B6
:100FD0000BAB01220AA901A802F05FFAB8E0D0E049
:100FE0004F4B00004469736B204572720000000093
:100FF000496E7420457272004E6F742052656164B0
:10100000790000004E6F2046696C65004E6F2050DD
:1010100061746800496E76616C6964204E616D652B
:101020000000000044656E696564000045786973DE
:1010300074000000496E76616C6964204F626A65D5
:101040006374000057726974652050726F74656331
:1010500074656400496E76616C69642044726976D7
:10106000650000004E6F7420456E61626C6564001F
:101070004E6F2046696C6573797374656D0000006E
:101080004D4B46532041626F72746564000000004E
:1010900054696D65204F7574000000004572726FD1
:1010A0007220636F64653A202530325800000000DA
:1010B0000D0A00000014014024000020107AFF1FD8
:1010C000A4040120147AFF1F187AFF1F0584080862
:1010D000915BF73CDCA70008920401202F494E49A0
:1010E000000000002F494E492F5344313534312E32
:1010F000494E4900F6F20020F0F000204C0C002090
:1011000020000020F0F20020F8F30020250000204D
:10111000B0090020ECA700084C4F4144494E472E2F
:101120002E2E2020202000002E4436340000000007
:101130002E524F4D000000002F494E492F253038C8
:101140005825303858253038582E6C696300000017
:101150009DF8280008F0C2FDC0B28DF82800412893
:1011600034BF303837388DF82800C0B240EA051057
:10117000C5B214F0010F06D008EB54000078A84265
:1011800001D0B77003E0641C202CFFF41DAF0122D6
:10119000AFF2B00101A802F0CDF800281CBF18B0D2
:1011A000BDE8F0810BABFC494FF480720E4601A8FC
:1011B00002F073F90BAB4FF40072F84901A802F08A
:1011C0006CF9F74C0BAB042204F5277101A802F06F
:1011D00064F90BAB0122F34901A802F05EF9F24970
:1011E0000BAB02220D4601A802F057F90BAB41F2FE
:1011F0009A02EE4901A802F050F90BAB0122EC492A
:1012000001A802F04AF901A802F045FBE548007880
:10121000A0F19801482998BFFFF700FBE549D4F8F1
:101220009C02A1FB0010800800EB40004000C4F8C5
:10123000A002304602F07FFBFFF7ABFAFFF7A9FBF5
:10124000FFF70EFED4F89C0204EB001000F23F7092
:10125000FFF7BFFD2988B4F89C0204EB41014EF270
:1012600040728852D448877718B0BDE8F08110B535
:101270004FF48042D149D24808F036FDC8490020D9
:1012800081F8180310BD70B5C54C054601468AB0FB
:1012900004F5467008F06DFD01222946684602F00B
:1012A00049F8C84D0026C0B14FF48042C34905F546
:1012B000404008F019FD84F8186300BFFFF769FA91
:1012C00004F5467202210020FFF707FABEA20421AE
:1012D0000220FFF702FA0AB070BD09AB4FF480425A
:1012E00005F54041684602F0D8F80998B0F5804FFE
:1012F00008D04FF48042B14905F5404008F0F4FCB5
:1013000084F81863684602F0C6FAD7E72DE9F0477B
:1013100081464FF0000AAFA108F01DFD002808BF6C
:10132000BDE8F087ACA1484608F015FD9C4C4EF690
:1013300046116718891F00266518002828884EF274
:10134000407821D0F02817D204EB4000B4F89C126A
:1013500020F80810A1A1384608F0EAFC49463846B2
:1013600008F0E6FC2888401C28800220C4E9A70673
:10137000484602F0E0FA82462A88394698A008F0EA
:10138000C7FD5046BDE8F0870028F5D0401E2880F4
:10139000384608F0D9FC002818BF4EF646111BD07D
:1013A000401E2218525C2F2A21D00028F8D148462E
:1013B00002F0C1FA824628887E4904EB400030F8EA
:1013C0000800C4F89C02A1FB0010800800EB40005C
:1013D0004000C4F8A002CFE73E70C4F8A062C4F891
:1013E0009C622E807DA002F0A6FA8246C4E72044CB
:1013F0004654DCE770B57C4D287800280CBF0024EB
:1014000070BD002002F0AEFEF8B178A008F080FDBB
:10141000641C082CF5D36249002081F83E07C1F80E
:10142000A402C1F89C02C1F8A0022878002818BFC5
:1014300070BDFFF7AEFA0520FFF7CEF9BDE87040AA
:10144000052170A20020FFF748B9012028705449F7
:10145000002001F05FFFDEE72DE9F04F89B00020AA
:10146000DFF8B8910890A9F20220059000F500700D
:1014700000F584760790801DDFF898A1DFF898B119
:10148000594CA0F102080490FFF783F9002164A2EF
:101490000846FFF722F90025E07885420CBF64A2D8
:1014A000AFF28032691C0020FFF717F940F2A91053
:1014B000684306EB400707F5887008F045FC0028F4
:1014C00014BF07F5887207F58072691C0220FFF7C8
:1014D00004F96D1C052DDFD30027A8F80070677193
:1014E000E0783D4640F2A91110FB01F006EB400008
:1014F00000F5887008F028FC68B1E07840F2A91186
:1015000010FB01F106EB410000F588700021FFF7A8
:1015100010FBA9F800002021504603F0FEFA002835
:1015200013BF50466079677103F0F3FA10F0FF00C3
:101530000CD023282FD07FDC0D287ED01B287DD017
:1015400021287CD0222826D000F046B9B8F8000027
:101550006D1C002814BF584636488542DBD3E0781E
:10156000002540F2A91110FB01F006EB400000F548
:10157000887008F0E9FB0028CDD0E078B9F8003099
:10158000401CC1B242460220FFF70CFBB8F8000035
:101590000028C0D154E077E0F6F20020F0F00020FF
:1015A000B009002020000020F0F20020F8F3002015
:1015B00025000020ABAAAAAA7805012044B00008A3
:1015C00000C0001000000010524F4D204C4F41440D
:1015D000454400002E0000002E2E00002F000000C9
:1015E00025732025640D0A0024000020496E6974CB
:1015F00069616C697A6520534420436172640D0A05
:101600000000000053442043415244204552524FB1
:101610005200000000140140E0930400F2F20020A8
:101620004641564F52495445204449534B530000BC
:101630002A200000404B4C000EE028E05CE021E056
:10164000E078B9F80030401CC1B242460220FFF7F2
:10165000A9FAA8F800705EE7242813D025287CD0CA
:10166000262802D0282807D0B6E0E078002818BF46
:10167000401E73D0E070AFE0E078042838BF401C13
:10168000F8D3ABE0E770B7E00420E070A6E0E078C4
:1016900040F2A91110FB01F006EB4001049808F09C
:1016A00068FB049802F047F9FFF7DAFBFA4981F882
:1016B0003E0708B30D46C5F89C72D5F8A402002871
:1016C0001AD9E07840F2A91110FB01F006EB4000B6
:1016D00000F58071D5F89C0205EB001000F23F7018
:1016E00008F039FB58B1D5F89C02401CC5F89C02A3
:1016F000D5F8A4128842E4D3012008906CE0E07889
:1017000040F2A91110FB01F006EB400000F5A871B2
:1017100002904FF40072059808F0E6FA0298B0F8CB
:10172000501307980180D5F89C0205EB001000F2D9
:101730003F700190D5F8580238B14FF0FF3008F0F3
:1017400054F905F5167002F0A6F805F542700199F6
:1017500008F00FFBFFF71DF801E022E04CE0FFF777
:1017600018F90520FFF738F8019808F039FA28B180
:1017700005210020019AFEF7B0FF04E0C74A0521C9
:101780000020FEF7AAFF0799B5F89C02098805EB2F
:1017900041024EF240715052FFF7DBFAC0488777A2
:1017A000AAE7E578042D0DD240F2A910684306EBB4
:1017B000400000F2523140F2523208F095FA6D1CAE
:1017C000042DF1D340F2523106F6485008F0A5FA44
:1017D00096F8000100288FD0E07868B1C0B240F2DE
:1017E000A91110FB01F106EB410191F8001100294C
:1017F00004BF401EE070EFD0089800283FF444AECC
:10180000FFF7A7FAA74CFEF7C4FFFFF7C2F80520C1
:10181000FEF7E2FF204608F0E3F938B109B02246AE
:10182000BDE8F04F05210020FEF757BF09B00521A4
:10183000BDE8F04F994A0020FEF74FBF2DE9F14F68
:10184000994F0026944C38789AB04FF00108002840
:1018500008BF00252ED1002002F084FC90B1AFF229
:10186000742008F055FB6D1C082DF4D38A4880F8CD
:101870003E67C4F8A462C4F89C62C4F8A0623878D9
:10188000C0B906E087F800808349002001F042FDDE
:10189000ECE7FFF77EF80520FEF79EFFAFF29C22F3
:1018A00005210020FEF719FF3878002804BF1BB07F
:1018B000BDE8F08FDFF8F4B14EF6421004EB000AF9
:1018C00004F23E3016904EF64010204417904EF62B
:1018D0004610204403904EF6441027186E4890F8A6
:1018E0003E0720B9FFF7BCFA6B4981F83E07D4F8F0
:1018F0009C12D4F8A402814224BF401EC4F89C026A
:101900006B48D4F89C120026A0FB0110800800EB65
:1019100040004500A81DC4F8A052A84288BF44F268
:101920003F7936D9F0B2FEF757FFD4F8A402A842A7
:1019300028D905EB850004EBC0004844804608F038
:1019400003FA002812BF424604EB051000F23F7272
:10195000601990F83E0310F0100F14BF5549564916
:1019600006A808F0E5FAD4F89C02A8420CBF534A36
:10197000534A31460020FEF7B0FE06AA3146022047
:10198000FEF7ABFED4F8A002761C6D1C801DA842A9
:10199000C8D80020DFF810810590054688F80500BA
:1019A0003880D4F89C0244F23F7900EB800004EBCD
:1019B000C0002E46484408F0C7F960B1D4F89C0234
:1019C0001699415C00EB800004EBC0004844FFF72F
:1019D000B0F8AAF800002021584603F09EF800282D
:1019E00013BF584698F8050088F8055003F091F8A1
:1019F00010F0FF000DD0242868D06ADC212867D0C1
:101A000038DC08287DD00D287CD01B287FF466AFF9
:101A100082E03888761C002814BF2A482A4886426B
:101A2000D9D3D4F89C02002600EB800004EBC00060
:101A3000484408F089F90028CDD094F89C0294F825
:101A4000A012BAF80030401AC1B23A460220FFF79D
:101A5000A9F838880028BED194F89C0294F8A01206
:101A6000BAF80030401AC1B23A460220FFF79AF89D
:101A70003D80B0E7222875D023287FF42FAFD4F81B
:101A8000A4020B49401EA1FB0021890801EB410182
:101A90004900C4E9A70121E7B0090020ECA700082C
:101AA00078050120B80C002024000020001401401B
:101AB000ABAAAAAAFCA7000804A8000808A8000866
:101AC0000CA80008E0930400404B4C006FE000E0DD
:101AD00049E0272804BF012005907BD017DC25288A
:101AE0006AD026287FF4FAAED4F89C0200281CBFE6
:101AF000401EC4F89C02D4E9A710884288BF801F0A
:101B000001E047E066E088BFC4F8A002E6E62828C6
:101B100015D078287FF4E2AE1A9800281FBF002065
:101B200084F818031BB0BDE8F08FFE4890F8000160
:101B3000002800F0DB811BB0BDE8F04F8CE4D4F846
:101B40009C02D4F8A412401C884238BFC4F89C02FE
:101B5000D4F8A002D4F89C12801D884298BFC4F823
:101B6000A002BBE60AE0D4F8A00200283FF4B6AE1B
:101B7000801FC4F8A002C4F89C02AFE6D4F8A0020B
:101B8000D4F8A412801D88423CBFC4F8A002C4F857
:101B90009C02A3E6AFF2BC50FFF7B8FBFFF75AF880
:101BA0000398057017980580DF4880F83E57C4F801
:101BB0009C52C4F8A05291E61A9800287FF48EAE89
:101BC000AFF2EC50FFF7A2FBFFF744F8D64880F8DD
:101BD0003E5783E6D4F89C021699415C11F0100F31
:101BE0000FD01A9900297FF479AE04EB001000F2AF
:101BF0003F70FFF78BFBFFF72DF8CB4880F83E577F
:101C00006CE604EB001000F23F78AFF6E4294046A2
:101C100008F09AF80546042828BF032679D36D1EDC
:101C200018F8050008F05AF819F80610C0B28142F9
:101C30006FD1761EF3D21A9800287FF44FAEBB48BE
:101C4000DFF8EC828178E9B30598D0B1FEF7A1FD09
:101C5000B8A202210020FEF740FDAFF23C62032152
:101C60000020FEF73AFDB74940F2F23008604FF02D
:101C7000E020016941F0020101614FF47A70FEF742
:101C800062FBD4F89C0204EB001000F23F75D4F81C
:101C9000580238B14FF0FF3007F0A7FE04F5167078
:101CA00001F0F9FD294604F5427008F062F8FEF7EC
:101CB00070FDFEF76EFE0520FEF78EFD284607F04C
:101CC0008FFF00E006E028B32A4605210020FEF73A
:101CD00004FD24E0417800291CBF491E4170B3D1A6
:101CE0004FF0FF3007F081FE04F5167001F0D3FDD0
:101CF00000254FF400519448C4F8585208F00DF8EC
:101D0000FEF747FDFEF745FE88F81E501BB0BDE804
:101D1000F08F7EE08D4A05210020FEF7DEFC17994A
:101D2000B4F89C024EF24072098804EB41018852DB
:101D3000059800281CBF00267A4F62D0D4F89C0278
:101D400004EB001000F23F7140F2A910704307EB62
:101D5000400505F5807007F0FEFFD8B928460399C5
:101D600007F0F9FFB0B93546042E0DD240F2A910A4
:101D7000684307EB400000F2523140F2523207F064
:101D8000B3FF6D1C042DF1D340F2523107F64850D9
:101D900007F0C3FF761C052ED0D3042540F2A9100E
:101DA000684307EB4000A0F2523140F2523207F094
:101DB0009BFF6D1EF2D15B48039907F0DAFFD4F860
:101DC0009C0204EB001000F23F7107F5807007F0F1
:101DD000D0FFD4F89C0200EB800004EBC00144F279
:101DE0003F70014407F5887007F0C3FF4FF400729D
:101DF000574907F5A87007F077FF17980088A7F8EC
:101E00005003FEF7A6FF002088F81E001BB0BDE8B7
:101E1000F08FD4F89C0204EB001000F23F78AFF68C
:101E2000F049404607F090FF0546042828BF0326E6
:101E3000FFF454AD6D1E18F8050007F04FFF19F8B8
:101E40000610C0B281427FF449AD761EF2D21A98D4
:101E500000283FF443ADD4F89C0204EB001000F2DC
:101E60003F75294604F5467007F083FF0122294695
:101E7000684601F05FFA374DF0B14FF480423649C1
:101E800005F5404007F030FF002084F8180300BF3C
:101E9000FEF77FFC04F5467202210020FEF71DFCD0
:101EA000AFF6DC0204210220FEF717FC1BB0002075
:101EB000BDE8F04F06F05DBA09AB4FF4804205F57E
:101EC0004041684601F0E9FA0998B0F5804F09D021
:101ED0004FF48042204905F5404007F005FF0020FF
:101EE00084F81803684601F0D6FCD1E704F5427483
:101EF000FEF74FFCFEF74DFD0520FEF76DFC20467A
:101F000007F06EFE38B11BB02246BDE8F04F052148
:101F10000020FEF7E2BB1BB00521BDE8F04F0B4AE5
:101F200000201BE0F8F30020B0090020240000206E
:101F300078050120202020414444454420544F206E
:101F40002020000000000020EC050120ECA7000884
:101F5000F0F000200000001044B00008FEF7BDBB08
:101F60002DE9F047B6480068B649C0F30720096874
:101F700041B98F21814305D14FF0E0210A6922F058
:101F800002020A61B04C214622798968824202BF6E
:101F9000481CA060BDE8F08720EA02088243207157
:101FA0004FF000061CBFA660BDE8F08718F0800F58
:101FB000DFF89892A64FA74D21D04846B1F5FA7F99
:101FC000807B07D2002807BF012089F80E001B2064
:101FD000607114E098B94FF0FF3007F006FD05F589
:101FE000167001F058FC4FF400519B48C5F8586238
:101FF00007F093FEFEF7CDFBFEF7CBFCBE77DFF8D4
:102000005CA218F0010F0DD099F80E0040B3A06843
:10201000B0F57A7F28BF242003D2FA282CBF2120D4
:102020002620607118F0020F0DD099F80E0010B341
:10203000A068B0F57A7F28BF232003D2FA282CBFEE
:1020400022202820607118F0040F51D099F80E005A
:10205000E0B1A068FA282CBF27200D20607147E06E
:102060009AF80000E028DDD2401CC0B28AF80000D7
:10207000FEF7D4FBD6E79AF800009828E3D9401E73
:10208000C0B28AF80000FEF7C9FBDCE7714890F89F
:102090003E0728B9FEF7E4FE6E4981F83E0738B3E3
:1020A000D5F89C02E060D5F8A0122161D5F8A422F1
:1020B000401C824288BFE060881DE168884298BF6A
:1020C000206105EB011000F23F70AFF6A471FEF73E
:1020D000ACFE68B1E06805EB001000F23F70FEF75F
:1020E00078FEBE77E068C5F89C022069C5F8A002BA
:1020F00018F0080F08BFBDE8F08799F80E0040B14E
:10210000A068B0F57A7F2CBF082025206071BDE85B
:10211000F087504890F83E0740B9FEF7A1FE4D49C0
:10212000002881F83E0708BFBDE8F087D5F89C027B
:10213000E060D5F8A012216100281CBF401EE060BD
:10214000814284BF891F216105EB001000F23F70BE
:1021500043A1FEF76AFE002808BFBDE8F087E068EB
:1021600005EB001000F23F70FEF733FEBE77E0682B
:10217000C5F89C022069C5F8A002BDE8F087F0B55B
:102180002F488BB00068334CC0F3072010F0010FCC
:1021900026D135A001F0CFFB2046002500F23E7687
:1021A00080F83E570220294FC4F89C020120B873E2
:1021B0002DA0FFF743FBBD7335702DA001F003FD8B
:1021C0000B222DA1684601F0B5F848B90AAB1022E0
:1021D00004F54671684601F022FA684601F05BFB9F
:1021E000012225A1684601F0A5F800281CBF0BB00C
:1021F000F0BD09AB102204F54671684601F04DF9B7
:10220000684601F048FB94F81803002804BF0BB09F
:10221000F0BD15A001F08FFB04F54670FFF733F811
:102220004FF0E020016941F002010161054941F2EE
:10223000040008604FF47A60FEF785F80BB0F0BD3B
:10224000100C024000000020240000202405012082
:1022500078050120B0090020EC05012020000020B5
:102260002E443634000000002F524F4D0000000075
:102270002F494E49000000002F494E492F53443149
:102280003534312E524F4D00521E531C002BD8BFF7
:102290007047491E401E12F0010F03D111F8012FA3
:1022A00000F8012F5A1008BF70474B78437011F89F
:1022B000023F00F8023F521EF7D170472DE9F0416E
:1022C000056B0F460446BD422FD02079F0B16078EF
:1022D00001232A4604F1340102F05CF810BB00200F
:1022E0002071E169606A0844A84284BFE678012E43
:1022F0000CD9E0690123054460782A4604F13401D1
:1023000002F048F8701EC6B2012EF2D86FB16078A4
:1023100001233A4604F1340101F0C8FF002808BF48
:10232000276302D00120BDE8F0810020BDE8F081E4
:1023300070B504460021FFF7C1FF050050D1207899
:10234000032845D16079002842D000264FF400725E
:10235000314604F13400266301F022FD552084F853
:102360003202AA2084F83302522084F8340084F820
:102370003500612084F83600412184F8371072223C
:1023800084F8182284F8192284F81A1284F81B029F
:10239000206984F81C02010A84F81D12010C84F8DB
:1023A0001E12000E84F81F02E06884F82002010A61
:1023B00084F82112010C84F82212000E84F8230202
:1023C0006078012304F13401626901F0E3FF667172
:1023D00000226078114602F079F8002818BF012524
:1023E000284670BD2DE9F0410C460546022924BF60
:1023F000286AA0429CBF0120BDE8F08128786E6A5F
:10240000012804D0022825D0032831D036E004EB7F
:10241000540706EB57212846FFF750FF70BBC7F360
:10242000080028447F1C90F8348006EB572128468A
:10243000FFF744FF10BBC7F30800284414F0010F56
:1024400090F8340048EA002014BF0009C0F30B00E4
:10245000BDE8F08106EB14212846FFF72FFF68B98D
:102460004FF4FF7000EA44002844808EBDE8F081FC
:1024700006EBD4112846FFF721FF18B14FF0FF30CB
:10248000BDE8F0814FF4FE7000EA8400284490F823
:102490003410D0F8350041EA002020F07040BDE84B
:1024A000F0812DE9F04716460C460546022924BF67
:1024B000286AA0429CBF0220BDE8F08728786F6A96
:1024C00006F0FF084FF0010A01280BD0C6F30729D8
:1024D000022839D0032818BF022046D085F804A06E
:1024E000BDE8F08704EB540907EB59212846FFF7B4
:1024F000E5FE0028F2D1C9F308002844343014F076
:10250000010F1ABF017868F31F113146017009F1FC
:10251000010885F804A007EB58212846FFF7CEFEF6
:102520000028DBD1C8F308012944343114F0010F2D
:1025300018BFC6F3071205D10A78C6F3032302F0C9
:10254000F0021A430A70C9E707EB14212846FFF787
:10255000B5FE0028C2D14FF4FF7101EA44012944BD
:1025600081F8348081F83590B8E707EBD41128461C
:10257000FFF7A4FE0028B1D14FF4FE7101EA8401F7
:102580002944320C81F8348081F8359081F8362066
:10259000320E81F83720A1E72DE9F041D0F82080F4
:1025A0000F0006460CD0FFF71DFF02283CBF01209C
:1025B000BDE8F08140452CBF3C46BDE8F08105E018
:1025C000F468002C18BF444528BF012425466D1C23
:1025D000A8459CBF0225022C0BD329463046FFF7A5
:1025E00001FF48B1411C14BF0128BDE8F081A5429C
:1025F000EDD10020BDE8F0816FF0704229463046F1
:10260000FFF74FFF30B94FB12A4639463046FFF742
:1026100048FF18B14FF0FF30BDE8F081F560306938
:10262000411C03D0401E3061012070712846BDE876
:10263000F08170B50D46C18081680446012919D02A
:102640002068026A8A4215D921B90278032A13D177
:10265000816A89B180780601B54225D32068FFF7E9
:10266000C1FE0146401C19D0022903D32068006A2C
:10267000884215D8022070BDE1600189A942F9D9CC
:10268000806A00EB1510206105F00F0134222068EC
:1026900002EB411108446061002070BD012070BD53
:1026A000A81B85B2AE42D9D9E1602068891E026AB2
:1026B000921E8A4291BF0020C26A807801FB0020EE
:1026C00000EB15102061DFE72DE9F0410446C088DA
:1026D0000F46401C0604360C1CBF2069002831D070
:1026E00016F00F0F76D1401C2061E16831B12268ED
:1026F0009078401E10EA161F05D06BE02068008914
:10270000B0421FD966E01046FFF76CFE054601286F
:102710001BD9681C40D02068016AA9424DD88FB1EE
:10272000E168FFF739FF050004BF0720BDE8F0812D
:10273000012D0AD0681C2FD000212068FFF7BEFDB4
:1027400030B129E00420BDE8F0810220BDE8F0812D
:1027500020684FF400723430002101F021FB206822
:10276000A91E026A921E8A4298BF002103D982786C
:10277000C36A01FB023101632068002780780028CA
:1027800088BF4FF0010814D92068002180F8048028
:102790002068FFF793FD10B10120BDE8F0812068AB
:1027A000016B491C0163781CC7B220688078B8426D
:1027B000EAD82068016BC91B0163E5602068A91E87
:1027C000026A921E8A4291BF0020C26A807801FB91
:1027D00000202061E68006F00F013422206802EB21
:1027E0004111084460610020BDE8F0812DE9F04FFF
:1027F00091B0044680690590E06904900C2206A817
:102800000599FFF741FD9DF8230010F0200F1EBF32
:10281000062011B0BDE8F08F10F0010FFD4E4FF60D
:10282000FF7500F0318105990020C872E061012038
:102830000990DDF8148006A90B224046DDF81090BF
:10284000099FFFF721FD052F0AD97808B9F8001074
:1028500000EBC730084487B239F8020F0028F4D1E2
:10286000ED4907200DF12803A1FB07C2D20852420F
:1028700002EB820207EB420230321A544CF6CD4290
:10288000401E7A43D70CEFD17E221A540021814298
:1028900006DA18F801C0BCF1200F18BF491CF6D1A8
:1028A0000828B4BF401C202208F80120491CC1F1AF
:1028B0000802002A23DD4144491E12F0010F08D00E
:1028C0000828AEBF4FF0200C13F800C0401C01F8E0
:1028D00001CF521013D00828BABF13F800C0401C13
:1028E0004FF0200C81F801C00828BABF13F800C0CF
:1028F000401C4FF0200C01F802CF521EEBD10021FA
:102900002046FFF796FE002873D1FF200B90019020
:1029100021692068FFF7D2FC5FEA000969D1676985
:10292000387858B1F97AE52801F03F0104D011F068
:10293000080F07D00F290AD0FF2058E00999642911
:102940007ED1D0E00F2902D00199C9B370E0D4F84C
:102950001CB0BBF1000F4BD010F0400F06D0797BBC
:1029600000F0BF000B910190E28822840199884217
:102970003BD1797B0B98814237D138784FF0000AF0
:1029800000F0BF00401E00EB800101EBC0094FF0DA
:10299000010800BF16F80A00B8F1000F384400889B
:1029A0000FD001F065FF8046B9F1240F1DDA3BF826
:1029B000190009F1010901F05BFF404515D102E062
:1029C00018E0A84211D10AF1010ABAF10D0FE1DBBA
:1029D000387810F0400F1DBFB8F1000F3BF8190018
:1029E0000028019808BF401E00D0FF20C0B201900F
:1029F00035E03BE00022791E5FF005034FEA520804
:102A000008EBC2121044C2B211F802CF4FEA5208CA
:102A100008EBC21248786244D2B25B1EEED1500875
:102A200000EBC211B87A08440B99C0B288424ED06C
:102A3000FF2001902584A069C17A11F0010F00E008
:102A40001CE008BF0A210AD101E0491E06D317F88D
:102A5000012B10F8013BD21A01D1F6E7B2B30021E5
:102A60002046FFF731FE00283FF452AF0999642950
:102A700039D004281CBF11B0BDE8F08F9DF8231099
:102A80000598C1720498E0619DF8230010F0020FD0
:102A900014BF002001270CD0049931F81010002930
:102AA0001CBF401C80B2F7D1193044F6C5614843C1
:102AB000870C00212046FFF7BCFD002807BF4FF020
:102AC000000AD14611B0BDE8F08F10E0FFE7099988
:102AD0004846491C89B209916429FFF4AAAE1CBF7B
:102AE00011B0BDE8F08F072011B0BDE8F08F21696B
:102AF0002068FFF7E3FB5FEA00087CD1606900789B
:102B0000E5281CBF00284FF0000907D0012120460E
:102B1000FFF7DAFD5FEA0008E9D0B2E0B9F1000F93
:102B200008BFB4F806A009F101001FFA80F9B94501
:102B3000ECD1012F72D951462046FFF77AFD5FEAAA
:102B4000000858D1D4F818800022A8F1010098F8A4
:102B5000001005234FEA520909EBC2121144CAB210
:102B600010F802CF4FEA520909EBC21241786244D1
:102B7000D2B25B1EEED1500898F80A1000EBC210DA
:102B80000844C0B20A90781E1FFA80FB21692068B1
:102B9000FFF794FB5FEA000873D16069D4F81C80EA
:102BA0000A9941730F21C1720021017381760BF0E4
:102BB000FF07C176791E01EB810202EBC102531CB3
:102BC00038F8121041700A0A8270002908BF4FF6C7
:102BD000FF710122944600F10109A9421CBF38F897
:102BE00013105B1C16F802A000F80A104FEA112A15
:102BF00016F802E000E044E00EF809A0002908BF42
:102C00004FF6FF71521C0CF1010CBCF10D0FE4DB0F
:102C1000A94204E00FA80008CDCCCCCC17E01ABF25
:102C200038F81310002947F0400707702168012089
:102C3000087100212046FFF747FD5FEA000820D118
:102C4000ABF101001FFA80FBBBF1000F9ED121699F
:102C50002068FFF733FB5FEA000812D16569202284
:102C60000021284601F09CF80B222846A169FFF7B5
:102C70000BFBA069C07A00F01800287321680120BE
:102C8000087111B04046BDE8F08F2DE9F34F83B0D5
:102C900080460498002400782F2811BF5C280498EF
:102CA000401C04900FBFC8F80840D8F800008069A5
:102CB000C8F8080004980078202808D2002140466F
:102CC000FFF7B7FCC8F8144005B0BDE8F08F00244A
:102CD000049ED8F81C702546705D6D1C20281CD3FE
:102CE0002F2818BF5C281CD0242C0EDA012101F0FB
:102CF000A3FD030009D0802B38BFFEA109D20A78BA
:102D00003AB1824218BF491CF9D105B00620BDE88E
:102D1000F08F27F81400641CDEE770190426049075
:102D200002E0701900260490012C3AD0022C4FD0FA
:102D3000002CEAD007EB440030F8020C202818BF22
:102D40002E284CD0002CE0D0002027F814000B22B5
:102D50002021D8F8180001F023F8002537F81500D5
:102D6000202814BF2E286D1CF8D0002D18BF46F067
:102D700003063CB107EB440030F8020C2E2818BFC4
:102D8000641EF6D14FF0000AD1464FF0080B00BF89
:102D900037F815006D1CE0B3202825D02E2821D04F
:102DA00025E038882E28C5D1002027F814000B21F3
:102DB000A042B4BF2E222022D8F818301A54401C4A
:102DC000491EF5D1D8F8181046F02000C8727AE0F4
:102DD00078882E2804BF38882E28ABD1E4E7641EFB
:102DE000A8D192E7A54202D046F00306D0E7DA4523
:102DF00001DAA5422CD1BBF10B0F10D0A54218BFB0
:102E000046F003060DDC25464FF0080A4FF00B0B89
:102E100000E006E04FEA89604FEA1069B8E746F043
:102E20000306D8F818000178E52904BF05210170D0
:102E3000BBF1080F04BF4FEA89604FEA10690C200C
:102E400030EA090036D0032030EA090032D033E0FE
:102E500080280ED3002101F0EFFC002808BF46F0C7
:102E600002060DD0A64946F00206084410F8800C70
:102E700030B1A4A10A783AB1824218BF491CF9D1F5
:102E80005F2046F003060EE0A0F14101192998BF2A
:102E900049F0020907D9A0F16101192903D82038A6
:102EA00049F0010980B2D8F8181001F80A000AF1B7
:102EB000010A6DE746F0020616F0020F0AD000BFC5
:102EC000D8F81800C67200214046FFF7B2FB002870
:102ED0006DD10CE009F00300012808BF46F0100690
:102EE00009F00C00042808BF46F00806E8E7FF20B8
:102EF000DFF818B201904FF6FF7A0090D8F8101062
:102F0000D8F80000FFF7DAF903007DD1D8F81440B3
:102F100094F800C0BCF1000F0CD0E07ABCF1E50FD2
:102F200000F03F0004D010F0080F05D00F2808D0A3
:102F3000FF2050E004238DE00F2802D00098A8B3B2
:102F400069E0D8F81C90B9F1000F7CD01CF0400F5C
:102F500008D0607B0CF0BF0CCDE900C0B8F80610BB
:102F6000A8F820100098844533D1617B01988142F4
:102F70002FD12078002700F0BF00411E01EB810017
:102F800000EBC1065FF001051BF807002044008834
:102F900075B101F06DFC0546242E1ADA39F81600D9
:102FA000761C01F065FCA84213D103E015E052E065
:102FB00050450ED17F1C0D2FE6DB207810F0400F1E
:102FC0001DBF002D39F816000028009808BF401ECC
:102FD00000D0FF20C0B2009035E00020611E052225
:102FE000460806EBC0106044C0B211F8025F460804
:102FF00006EBC01091F801C02844C0B2521EEFD1B8
:10300000410801EBC01100E024E0A07A08440199D6
:10301000C0B288421ED0FF200090A8F820A0D8F8A7
:103020001800C17A11F0010F08BF0A210BD101E08D
:10303000491E07D314F801CB10F8012BBCEB020298
:1030400001D1F5E732B100214046FFF73DFB030017
:103050003FF454AF1846D8F81810C97A01F00401AB
:1030600048B104280EBF002905B0BDE8F08F052047
:1030700005B0BDE8F08F00291CBF05B0BDE8F08F9A
:10308000D8F81400C17A11F0100FF0D0818A408B6B
:1030900061F31F40C8F8080019E62DE9F047D0F8A1
:1030A00000C01646DFF868809CF80020A2F13003CB
:1030B000092B9CBF9CF801203A2A12BF98F80030D7
:1030C0000CF102020260002B1CBF0B20BDE8F08750
:1030D000104804680C60002C04BF0C20BDE8F08789
:1030E000207828B1607801F0DBF810F0010F26D0CD
:1030F000002511E0222A3A3C3E3F7C7F0000000080
:103100001CA800082B2C3B5B3D5D00000FA80008AD
:103110003C0000204000002025702846657001F02A
:1031200021F810F0010F1CBF0320BDE8F087002E2E
:1031300018BF10F0040F0AD00A20BDE8F087002E57
:1031400014BF10F0040F0020F6D1BDE8F087002670
:1031500032466078012304F1340101F0A7F860BB26
:10316000B4F832024AF65529484546D194F86A1017
:10317000B4F86B00FE4F41EA002020F07F40B842D7
:1031800036D094F88610B4F8870041EA002020F089
:103190007F40B8422CD094F8F61104F5F97061B371
:1031A000017AD0F80900012341EA0022164660782E
:1031B00004F1340101F07AF810B10120BDE8F08784
:1031C000B4F83202484518D194F86A10B4F86B008C
:1031D00041EA002020F07F40B84209D094F88610E0
:1031E000B4F8870041EA002020F07F40B84204D1C3
:1031F000B4F83F00B0F5007F02D00D20BDE8F087A5
:10320000B4F84A0028B994F85800D4F8591040EAA4
:103210000120E06194F84410E170B4F84270484332
:10322000BB19636294F841C084F802C0B4F8452029
:103230002281B4F8471029B994F85410D4F855A055
:1032400041EA0A21C91B091AA1EB1211B1FBFCF1D9
:10325000891C012740F6F77C2162614528BF0227BF
:103260004FF6F77C614528BF03270FD2032F18BF05
:1032700019180BD000EB12101844A162E0624FF055
:10328000FF3020612571032F38D106E094F86010DB
:10329000D4F861C041EA0C21ECE76571B4F8640030
:1032A000012382196261607804F1340100F0FEFFAD
:1032B000002804BFB4F8320248451FD194F8340006
:1032C000D4F8351040EA0120AA49884216D194F872
:1032D0001802D4F8191240EA0120A74988420DD1FA
:1032E00094F82002D4F8211240EA0120E06094F81A
:1032F0001C02D4F81D1240EA0120206127702563CA
:10330000A561B8F80200401CA8F80200E080002087
:10331000BDE8F08700281CBF0B207047974A0023A8
:103320001068002818BF0370002918BF0B70002018
:10333000116070472DE9F7478DB00027064602F06F
:103340001F0507608E4C05F01E0269460EA8FFF7A8
:10335000A4FE00281CBF10B0BDE8F08709A8CDE985
:10336000060468460E99FFF790FC15F01C0F61D01B
:103370004FF0010998B104281CBF10B0BDE8F087D8
:103380006846FFF733FA00281CBF10B0BDE8F0878D
:1033900045F00805059C15F0080F3FD15FE015F0DA
:1033A000040F1EBF082010B0BDE8F087059C1CB1BB
:1033B000E07A10F0110F03D010B00720BDE8F087BD
:1033C00015F0080F4BD0A08AB4F81A8027756775DE
:1033D000A776E77627776777A77760F31F48E777C1
:1033E0000098B8F1000F80F804900098D0F830A051
:1033F0000BD0414600F0E9FC00281CBF10B0BDE82E
:10340000F087A8F101000099C86051460098FEF7C6
:1034100055FF00281CBF10B0BDE8F087E772A77306
:10342000E773212020746774009845F0200580F828
:10343000049014E000281CBF10B0BDE8F087059C84
:103440001CB1E07A10F0100F03D010B00420BDE8DA
:10345000F08715F0020F18BF10F0010FACD10098E3
:10346000006BF06105983062B571A18A608B61F3E1
:103470001F403061207FD4F81D1040EA0120C6E9CA
:103480000270FF20F071B761009830600098C0882A
:10349000B08010B00020BDE8F0872DE9F0474FF074
:1034A00000090446C3F8009015460F460068A2883C
:1034B0000921984600281CBF0378002B02D0C3883E
:1034C000934202D00846BDE8F087407800F0E8FE5D
:1034D00010F0010F1CBF0320BDE8F087A07910F0A9
:1034E000800F1CBF0220BDE8F08710F0010F04BF61
:1034F0000720BDE8F087D4E90210401A854288BF52
:103500000546002D71D0A168C805C00D59D12068AD
:10351000E379827893420DD3002916BF616920694F
:10352000FEF760FF01282DD9411C1CBF606184F8A3
:10353000079053D020686169026A891E921E9142E9
:1035400020D28378D0F82CC001FB03C2D2B1E1793C
:103550006E0A01EB020A30D08A199A4288BF5E1ABD
:10356000F3B240785246394600F0A0FEB0BB10E0FE
:103570004641540052526141727241614000002044
:10358000D8040120A07940F08000A0710220BDE89D
:10359000F0872168087958B1086BA0EB0A00B042A7
:1035A00006D2343107EB40204FF40072FEF76CFE78
:1035B000E0793044E071760222E0481CC4F818A09B
:1035C000E0712089C0F30800C0F50076AE4288BFE4
:1035D0002E46A1692068FEF771FE38B1A07940F04F
:1035E0008000A0710120BDE8F08715E021892068E6
:1035F000C1F308013431014432463846FEF744FE37
:10360000A06837443044A060D8F80000AD1B3044B7
:10361000C8F800007FF477AF0020BDE8F0872DE9FF
:10362000F05F4FF00009C3F8009015460F460446BE
:10363000828801680920984600291ABF0B78002B60
:10364000BDE8F09FCB88934218BFBDE8F09F487853
:1036500000F026FE10F0010F1CBF0320BDE8F09F14
:10366000A07910F0800F1CBF0220BDE8F09F10F081
:10367000020F04BF0720BDE8F09FE06841198142B6
:103680007ED3002D18BF4FF0010A79D0A068C10584
:10369000C90D73D12268E179937899420ED3C0B1F4
:1036A00010466169FEF778FF002869D0012837D0FD
:1036B000411C1CBF606184F807906FD02068A1692D
:1036C000026B8A420ED10021FEF7F8FD002865D179
:1036D00008E020690028E9D100211046FEF75CFFD0
:1036E0002061E1E720686169026A891E921E8A42B0
:1036F00016D98378D0F82CC001FB03C181B1E279DF
:103700006E0A02EB010B27D09119994288BF9E1ACD
:10371000F3B240785A46394600F03CFE88BB06E0DA
:10372000A07940F08000A0710220BDE8F09F2068E1
:10373000016BA1EB0B01B14209D207EB41213430FF
:103740004FF40072FEF7A0FD206880F80490E07945
:103750003044E071760235E0D4E90212914208D398
:103760000021FEF7ABFD002804BF2068C0F830B090
:1037700014D1C4F818B0E079401CE071208901E050
:103780002CE00BE0C0F30800C0F50076AE4288BF25
:103790002E46A1692068FEF791FD30B1A07940F076
:1037A0008000A0710120BDE8F09F21892068C1F34D
:1037B00008013431084432463946FEF765FD206879
:1037C00080F804A0A06837443044A060D8F8000016
:1037D000AD1B3044C8F800007FF458AFD4E90201B3
:1037E000884298BF0846E060A07940F02000A071B0
:1037F0000020BDE8F09F70B504468288016809206A
:1038000000291ABF0B78002B70BDCB88934218BFDC
:1038100070BD487800F044FD10F0010F1CBF03207C
:1038200070BD0025A179284611F0200F08BF70BD9A
:10383000E1692068FEF742FD002818BF70BD206ACC
:10384000C17A41F02001C172217B0177A189090A67
:103850004177E168090C8177E168090EC177217C25
:103860008176218A090AC1762169090C01752169CD
:10387000090E41758575C575212101764576A079BA
:1038800020F02000A0712168012008712068BDE8A7
:103890007040FEF74DBD70B504468288016809206E
:1038A000002500291CBF0B78002B3FD0CB8893420A
:1038B0003CD1487800F0F4FC10F0010F1CBF03204D
:1038C00070BD2846A17911F0200F32D0E16920683F
:1038D000FEF7F4FC002829D1206AC17A41F02001CA
:1038E000C172217B0177A189090A4177E168090C3E
:1038F0008177E168090EC177217C8176218A090AE6
:10390000C1762169090C01752169090E417585751A
:10391000C575212101764576A07920F02001A1719D
:103920002068012101712068FEF702FD002818BF00
:1039300070BD256070BD11B58DB0FE4C002269468A
:103940000DA8FFF7AAFB00281CBF0EB010BD09A8E8
:10395000CDE9060468460D99FFF797F930B10428C0
:103960001CBF0EB010BD05200EB010BD059959B199
:10397000CA7A12F0100FF6D08A8A498B62F31F417F
:10398000009A91610EB010BD009A002191610EB0B5
:1039900010BD2DE9F0410D460446828801680920DA
:1039A00000291ABF0B78002BBDE8F081CB88934229
:1039B00018BFBDE8F081487800F072FC10F0010FEC
:1039C0001CBF0320BDE8F0810027A17911F0800F12
:1039D0001CBF0220BDE8F081E268AA4203D211F0C8
:1039E000020F08BF15464FF00008A168FF20A7602E
:1039F000E071002D5AD020688278560271B16A1E9B
:103A0000491EB2FBF6F2B1FBF6F39A4206D3701EE2
:103A100021EA0000A0602D1A616902E0216971B1FC
:103A20006161002942D0B54228D9A07910F0020F77
:103A3000206811D0FEF7B0FD01000BD00FE000218F
:103A4000FEF7AAFD014601284AD0481C18BF216193
:103A50003FD0E5E7354611E0FEF7C4FC0146481CBF
:103A600037D001293CD92068006A884238D9616181
:103A7000A068AD1B3044A060B542D6D8A068C5F39D
:103A800047222844A060E805E271C00D0ED02068EE
:103A9000891E036A9B1E8B4222D9C36A807801FB70
:103AA0000030E8B102EB0008501CE071A068C105CD
:103AB000C90D1EBFA1694145C4F81880E16888425C
:103AC00004D9E060A07940F02000A0713846BDE83C
:103AD000F081A07940F08000A0710120BDE8F08164
:103AE000A07940F08000A0710220BDE8F08133B5DC
:103AF00083B0044601468F4D002204A8FFF7CDFA9B
:103B000000281CBF05B030BD6846C4E90605204644
:103B10000499FFF7BAF888B9606940B1C17A11F029
:103B2000100F0FD0818A408B61F31F40A060206886
:103B30000021C088A0802046FEF77BFD04281CBF22
:103B400005B030BD052005B030BDF0B50E460446C9
:103B500081880268774F092083B0002A19BF137843
:103B6000002B03B0F0BDD3888B421CBF03B0F0BD67
:103B7000507800F095FB10F0010F1EBF032003B03A
:103B8000F0BD00256846C4E90607B6B1204600F03E
:103B90004DF904280FBF2561002803B0F0BD314660
:103BA000204600F0E4F900212046FEF78DFD0428B0
:103BB00004BF0020256103B0F0BD00212046FEF7C0
:103BC00038FD03B0F0BD2DE9F14F8EB0594C012204
:103BD00069460EA8FFF761FA00281CBF0FB0BDE8C8
:103BE000F08F0BA8CDE9060468460E99FFF74DF853
:103BF000002802BF08200FB0BDE8F08F04281CBFCA
:103C00000FB0BDE8F08F0698C07A10F0200F1EBFED
:103C100006200FB0BDE8F08F00210098FEF7BCFC35
:103C200005004FF0010902BF07200FB0BDE8F08F7B
:103C3000012D02BF02200FB0BDE8F08F681C02BF4B
:103C400001200FB0BDE8F08F00210098FEF736FB91
:103C500000281CBF0FB0BDE8F08FA91E0098026AB3
:103C6000921E8A4298BF002603D9C26A807801FB5F
:103C70000026009C4FF4007234340021204600F0EE
:103C80008FF80B222021204600F08AF84FF02E08F2
:103C900084F800801020E0720020A075E0752121DA
:103CA00021766076E8B20A90A076C5F307200990E5
:103CB000E076C5F3074B84F814B04FEA156A4FF469
:103CC000041784F815A02022214604F12000FEF7F5
:103CD000DBFA84F82180009902980978032904D13D
:103CE0000099896A814208BF002084F83A00010ADD
:103CF00084F83B10010C84F83410000E84F8350071
:103D000000984FF000088078002822D90098002100
:103D100006630098761C80F804900098FEF7CEFAAF
:103D200000281CBF0FB0BDE8F08F0020621E4FF4CA
:103D3000807101E0D8040120507002F8020F491E82
:103D4000F7D108F1010000F0FF08009880784045A5
:103D5000DCD86846FEF74AFD040004D029460098E6
:103D600000F033F818E005981021C1728775390A00
:103D7000C175390C0176390E41760A998176099917
:103D8000C17680F814B080F815A0009880F80490EF
:103D90000098FEF7CDFA04460FB02046BDE8F08F3C
:103DA000521E531C002BD8BF7047401E12F0010F4B
:103DB000CAB208BF00F8012F591008BF70474270FF
:103DC00000F8022F491EFAD170472DE9F0410E4646
:103DD0000746022924BF386AB04284BF00254FF04D
:103DE000010811D931463846FEF7FCFA04001AD012
:103DF000012C09D0601C09D0002231463846FEF75C
:103E000050FB050004D00EE002250CE001250AE07D
:103E10003869411C03D0401C386187F80580386A36
:103E20002646B042DED82846BDE8F0812DE9F05F95
:103E30000446FF2600690422B0464FF0000900281E
:103E40001CBF8E4D4FF6FF7766D021692068FEF7C4
:103E500035FA020060D16169087858B1CB7AE5285B
:103E600003F03F0304D013F0080F05D00F2B08D048
:103E7000FF264BE004224FE00F2B02D0002E50D043
:103E80006EE010F0400F06D091F80D8000F0BF00FA
:103E9000E28806462284B04204BF487B404533D1C5
:103EA0000878D4F81CA000F03F00401E00EB800210
:103EB00002EBC000B1F80120242825DA2AF81020EE
:103EC000401C01234FEA030C15F803B08B44BBF8E8
:103ED00000B032B1242817DA2AF810B05A46401C34
:103EE00001E0BB4510D15B1C0CF1010CBCF10D0FC6
:103EF000EADB097811F0400F04D02428B8BF2AF873
:103F0000109001DA701E00E0FF20C6B200212046AA
:103F1000FEF7DAFB020025D0C4F810901046BDE889
:103F2000F09F00200D784B1E4FF0050C4FEA500912
:103F300009EBC010284413F8026FC0B24FEA5009D1
:103F400009EBC0105D783044C0B2BCF1010CEDD17A
:103F5000430803EBC013887A1844C0B24045DDD053
:103F60002784DBE7206900287FF46FAFD6E72DE9CF
:103F7000F0410C4601F109020169002954D043695E
:103F8000002593F80CC0595D202910D0052908BFE1
:103F9000E5211CF0080F05D0A1F14106192E9CBFA8
:103FA0002031C9B202F8011B6D1C082DEBDB197A18
:103FB00020292DD02E2102F8011B197A202927D083
:103FC0001CF0100F05D0A1F14105192D9CBF203127
:103FD000C9B202F8011B597A202919D01CF0100F20
:103FE00005D0A1F14105192D9CBF2031C9B202F8BD
:103FF000011B997A20290BD01CF0100F06D0A1F1DB
:10400000410CBCF1190F9CBF2031C9B202F8011B51
:10401000D97A2172197FD3F81DC041EA0C212160A1
:10402000198BA180D98AE1804FF0000882F80080C6
:10403000A769002F08BFBDE8F08100250169C1B163
:10404000018CA1F57F42FF3A13D0C66936F8020B06
:1040500078B1002100F0F0FB18B1E169491EA942D6
:1040600001DC002505E0785536F8020B6D1C0028B0
:10407000EFD107F80580BDE8F08100000FA8000827
:104080002DE9F0410E46044610F0800F09D004F0EF
:104090007F0400217720FFF7F3FF012888BFBDE8E8
:1040A000F0811021DFF80084404600F03FFCFF4F14
:1040B000FF21384600F02EFE1021404600F038FC6B
:1040C000FB4DFF21384600F025FEFF21384600F069
:1040D00021FEC0B26D1EFF280CD0002DF5D110219D
:1040E000404600F023FCFF21384600F013FEFF207D
:1040F000BDE8F0812146384600F00CFE310E38460E
:1041000000F008FEC6F30741384600F003FEC6F390
:104110000721384600F0FEFDF1B2384600F0FAFD06
:104120000121402C08BF952102D0482C08BF8721CF
:10413000384600F0EFFD4C2C03D1FF21384600F04B
:10414000E9FD0A24FF21384600F0E4FDC0B210F07A
:10415000800F08BFBDE8F081611E11F0FF04F1D1AE
:10416000BDE8F08100281CBF012070472DE9F8430D
:10417000DFF8409399F8000010F0020F7ED1F02094
:10418000CA4E6424C9F80400FF21304600F0C2FD85
:10419000601E10F0FF04F7D1002529464020FFF7EC
:1041A0006FFF012862D1642089F801004FF42F7756
:1041B0004FF4D5714820FFF763FF012808BFE84698
:1041C0000CD00021E920FFF75BFF012899BF0225F1
:1041D000E9270125412740F2BB2437E0FF21304683
:1041E00000F098FD08F80400601CC4B2042CF5D35C
:1041F0009DF80200012802BF9DF80300AA287F1E37
:1042000034D101E07F1E07D34FF08041E920FFF752
:1042100037FF0028F6D14FB300217A20FFF730FF97
:10422000002808BF002421D1FF21304600F072FD94
:1042300008F80400601CC4B2042CF5D39DF80000FB
:1042400010F0400F14BF0C2504250FE00021384664
:10425000FFF716FF10B1641EF8D200E02CB14FF446
:1042600000715020FFF70CFF00B1002589F80250C3
:1042700010218D4800F05AFBFF2100E00CE0304691
:1042800000F048FD45B199F8000020F0010089F8E0
:1042900000000420C9F8040099F80000BDE8F88384
:1042A000002812BF012083480078704700B90BB97D
:1042B000042070472DE9F05FDFF8F8A11F4689461A
:1042C0009AF8000010F0010F1CBF0320BDE8F09F1A
:1042D0009AF8020010F0080F08BF5202DFF8CC81F4
:1042E000012F114608D05220FFF7CAFE002808BF50
:1042F0004FF0140B0ED03FE05120FFF7C1FE002815
:104300003AD14FF40071484600F019FA002818BF5E
:10431000002731E04C464FF400768AF801B0664D34
:10432000FF21404600F0F6FCC0B26D1EFF2802D00F
:10433000FE2803D01CE0002DF2D119E00025FF215A
:10434000404600F0E7FC6D1C04F8010B042DF6DB81
:10435000361FF3D1FF21404600F0DCFCFF21404630
:1043600000F0D8FC781E09F5007910F0FF07D1D1D4
:1043700000214C20FFF784FE10214B4800F0D6FAB4
:10438000FF21404600F0C6FC002F14BF0120002092
:10439000BDE8F09F00B90BB9042070472DE9F04744
:1043A000444889461F460178144611F0010F1CBF8E
:1043B0000320BDE8F087017811F0040F1CBF022034
:1043C000BDE8F087807810F0080F08BF5402DFF8CE
:1043D000DC80012F10D010F0060F03D01946D72033
:1043E000FFF74EFE21465920FFF74AFE002808BF7E
:1043F000DFF8BCA00ED050E021465820FFF740FE69
:1044000000284AD1FE21484600F0C9F9002818BF0B
:10441000002742E04C46FC265546FF21404600F06E
:1044200079FCFF21404600F075FCC0B26D1EFF28EC
:1044300002D0002DF5D129E03146404600F06AFC5B
:104440005FF0000614F8011B404600F063FC14F80E
:10445000011B404600F05EFC701E10F0FF06F1D11B
:10446000FF21404600F056FCFF21404600F052FC80
:10447000FF21404600F04EFC00F01F00052805D14A
:10448000781E09F5007910F0FF07C3D1FD21002047
:1044900000F085F9002808BF01271021024800F02C
:1044A00045FAFF21404609E000000240003001408B
:1044B0003057050044000020E022020000F02AFCF2
:1044C000002F14BF01200020BDE8F08700281CBF8A
:1044D00004207047F0B5012485B01546264604290E
:1044E00014D0D048007810F0010F1EBF032005B093
:1044F000F0BD0F2980F01781DFE801F016377377E0
:10450000F0F0F0F0F0F0D1D6E2F1EE0028780028DB
:1045100014BF0128002400F00F81022812BF0424D8
:104520005670002400F008B9BF4F1021384600F043
:10453000FFF9BF4EBD4DFF21304600F0EBFBFF21E0
:10454000304600F0E7FBC0B26D1EFF2802D0002D00
:10455000F5D100E000241021384600F0E7F9FF21F2
:10456000304600F0D7FB00F0DFB800214920FFF70C
:1045700087FD002840F0D8801021684600F0DFF861
:1045800000285BD09DF80000B6EB901F09D19DF884
:1045900008109DF8090006EB012108440004800979
:1045A0007BE09DF805009DF80A1000F00F0000EB7D
:1045B000D1109DF809109DF8072001F0030100EBD0
:1045C00041009DF80810890901EB82019DF8062041
:1045D00002F0030201EB8221491CC01F01FA00F026
:1045E0005BE04FF40070108027E08E4E4FF000012A
:1045F000B07810F0040F22D0CD20FFF741FD002845
:104600001CD18B4EFF21304600F084FB1021684600
:1046100000F095F8002818BF30240FD0FF21304655
:1046200000F078FB611E11F0FF04F7D19DF80A003D
:104630000009102101FA00F02860002474E04920EC
:10464000FFF71EFD00286FD11021684600F077F8B3
:10465000002869D0B07810F0020F10D09DF80A0041
:104660009DF80B108006400E00EBD1109DF80D1048
:104670004FF0FF32401C02EB911188400DE09DF895
:104680000B008107C90E01EB50109DF80A10401C69
:10469000C1F38401491C10FB01F02860CDE761489B
:1046A0000024807810703FE000214920FFF7E8FCEB
:1046B00040BB1021284600F042F80028BDD133E06D
:1046C00000214A20FFF7DCFCE0B91021284600F069
:1046D00036F80028B1D127E015E000E023E0002102
:1046E0007A20FFF7CDFC002804BF0424504E1BD1D4
:1046F000FF21304600F00EFB05F8010B601E10F0A4
:10470000FF04F5D110E00021CD20FFF7B9FC58B926
:10471000FF21474800F0FEFA4021284600F00FF83C
:1047200000288AD100E0042410213F4800F0FEF860
:10473000FF213F4800F0EEFA05B02046F0BD2DE91C
:10474000F0410E463749054614204870394C384F21
:10475000FF21384600F0DEFAC0B2641EFF2804D004
:10476000FE2805D00020BDE8F081002CF0D1F9E74B
:104770000024FF21384600F0CDFA641C05F8010B37
:10478000042CF6DB361FF3D1FF21384600F0C2FAC5
:10479000FF21384600F0BEFA0120BDE8F0812DE986
:1047A000F041234F0E460446204DFF21384600F0CD
:1047B000B1FAFF21384600F0ADFAC0B26D1EFF28F5
:1047C00002D0002DF5D127E03146384600F0A2FA9C
:1047D000FD2E1CBF00253E4621D000BF14F8011B52
:1047E000304600F097FA14F8011B304600F092FAB8
:1047F000681E10F0FF05F1D1FF21304600F08AFA63
:10480000FF21304600F086FAFF21304600F082FAA0
:1048100000F01F00052802D00020BDE8F081012033
:10482000BDE8F08144000020000002403057050040
:1048300000300140E0220200802838BF7047144A4F
:1048400051B1B0F5807F24BF0020704702EB4000DB
:10485000A0F580700088704732F81130834203D091
:10486000491C89B28029F7D301F18000C0B270479A
:10487000084A002132F81130002B08BF70478342EC
:1048800018BF491CF6D1044830F8110070470000E9
:104890009CA800089CA900087CAB00082DE9F00149
:1048A000002201255FF00306D1F800C005FA02F3EB
:1048B0000CEA030C9C4533D107684FEA420C06FA18
:1048C0000CF4A74307600F79D0F8008007FA0CF7C3
:1048D00047EA080707600F79012F18BF022F14D18C
:1048E0008768A74387604F79D0F8088007FA0CF7EC
:1048F00047EA08078760476827EA0303436043687D
:104900008F799740BFB23B434360C368A343C36002
:10491000CB7903FA0CF3D0F80CC043EA0C03C36064
:10492000521C102AC0D3BDE8F001704701837047C4
:1049300041837047002A14BF018341837047000000
:104940003A490A6822F4E052104308607047374938
:104950000A6822F4604242EAC00008607047334AA5
:1049600030B41168324B11F00C0106D0314C0429DF
:1049700008BF046002D008291ED0036011680F230D
:1049800003EA11112C4B595CD0F800C02CFA01F14C
:104990004160D2F800C0072404EA9C2C13F80CC034
:1049A00021FA0CFCC0F808C0126804EA52329A5C82
:1049B000D140C16030BC70472049D1F800C0CCF371
:1049C0008055D1F800C0002D0CF03F0C14BFB4FB93
:1049D000FCF3B3FBFCF3D1F800C00968CCF3881CEE
:1049E00003FB0CF3C1F30141491C4900B3FBF1F196
:1049F0000160C3E7124A0029116814BF084321EA85
:104A00000000106070470F4A0029116814BF084366
:104A100021EA0000106070470B4A0029116814BF9A
:104A2000084321EA00001060704700000838024087
:104A30000024F40040787D014C000020043802403E
:104A400030380240403802404438024030B5044615
:104A5000008A85B00D46C98820F440500843208262
:104A6000A089A9882A8920F4037011436A8920F457
:104A7000A05010430843A081A08AA98920F4407067
:104A80000843A0826846FFF76AFFA4F18040B0F5B2
:104A900088301BBFA4F18040B0F58A30039802989B
:104AA000A18911F4004F00EBC00101EB001029684F
:104AB00014BF49008900B0FBF1F0204A6FF0180CD8
:104AC000A2FB0031490909010B0903FB0CF300EBC0
:104AD0008300A38913F4004F4FF0320314BF03EB9C
:104AE000C00003EB0010A2FB00204FEA501014BFDF
:104AF00000F0070000F00F000843208105B030BD32
:104B00000029818914BF41F4005121F400518181B1
:104B100070478088C0F30800704702460020128862
:104B20000A4218BF01207047C2B2054800680188D8
:104B300011F0400FFBD08280012070471F85EB51A0
:104B40005C00002010B402882B4BDFF8B0C0984204
:104B500018BF604511D0B0F1804F1CBFA0F1804458
:104B6000B4F5806409D0A0F18044B4F500641CBFA2
:104B7000A0F18044B4F5406403D14C8822F0700267
:104B80002243A0F18044B4F580541CBFA0F18044BE
:104B9000B4F5A05403D00C8922F440722243028061
:104BA0004A68C2620A880285984212BF6045897AC3
:104BB00001860121818210BC70470029018814BF41
:104BC00041F0010121F0010101807047002A828932
:104BD00014BF114322EA010181817047038A002238
:104BE00080890B4200EA01001CBF00280122104608
:104BF0007047C94301827047000001400004014032
:104C000030B4C27801784FF0010C4FF0E024FAB1D3
:104C10001A4A12680F2502F4E062C2F5E062C2F39C
:104C20000722C2F10403D54042789A4083782B4092
:104C30001A43134B1201CA54007800F01F010CFAFA
:104C400001F1400904EB8000C0F8001130BC70474E
:104C500001F01F000CFA00F0490904EB8101C1F8D2
:104C6000800130BC70474FF0E021042808690CBF78
:104C700040F0040020F00400086170470CED00E0F3
:104C800000E400E010B402880B88B1F802C0CC88C0
:104C900043EA0C03B1F804C002F441524CEA040C9C
:104CA00043EA0C03B1F808C043EA0C03B1F80AC0A8
:104CB00043EA0C03B1F80CC043EA0C03B1F80EC090
:104CC00043EA0C031A430280828B22F4006282833F
:104CD000098A018210BC70470021018041808180D7
:104CE000C180018141818181C18107210182704799
:104CF0000029018814BF41F0400121F040010180EA
:104D000070470029818814BF41F0040121F004019B
:104D1000818070478181018911F0010FFBD080896A
:104D20007047000070B505460088401E84B204F448
:104D300078402146B0F5C05F1CBFFA48005D16D030
:104D400002462146F8A005F0E3F8A87B40F0800079
:104D5000A873FBF71EFD0221FDA20846FBF7BDFC70
:104D6000BDE870400321FDA20220FBF7B6BCB1F5FF
:104D7000E05F2CBFFC48FD4803F0DFFCE0E710B427
:104D8000FB4A0188037B1268491CA3F1010C0C0A41
:104D900080F80CC0D454037BA3F1010C80F80CC044
:104DA000D154017B90F80BC04B1E037302F801C075
:104DB000C17A41F00401C172EE490988018010BC3A
:104DC0007047EB4B0188027B1B68491C4FEA112C92
:104DD00003F802C0521ED2B29954511E0173418889
:104DE00001807047017B491CCAB2E14909688B5CAC
:104DF000C372521CD3B2CA5C5B1CDBB2C95C42EA10
:104E00000121018003737047017B491CCAB2D84954
:104E10000B68995C521CD2B29B5C41EA0321491C8D
:104E200001800273704782788272018802F08003E9
:104E3000491C0180C17A21F082011943002A08BF70
:104E400041F00201C1727047817A82780388A1EB38
:104E5000020C5B1C0380C37A0CF0800C23F08303EC
:104E600043EA0C0391420CBF4FF0020C4FF0000CD0
:104E700043EA0C038A4294BF012100211943C17205
:104E80007047417A82780388A1EB020C5B1C038097
:104E9000C37A0CF0800C23F0830343EA0C039142A5
:104EA0000CBF4FF0020C4FF0000C43EA0C038A4297
:104EB00094BF012100211943C1727047F0B4037AF5
:104EC00090F80BC0DCB204EB01051CF0080F0CF0ED
:104ED000010284EA01043DD003F00F0601F00F0740
:104EE0003E4432440A2A24BF961D66F30702202A54
:104EF00004D302F00F06103666F3070203F0F00643
:104F000001F0F001314411442CF0C20201F0FF0C19
:104F10001CF0800F18BF42F0800202F001063544F9
:104F200015F0FF0F08BF42F002028CEA0303A3430F
:104F300013F0800F18BF42F040020B46A02926BF95
:104F400042F0010203F1600102F0FE020172C2723E
:104F5000F0BC7047A9182CF0C30211F0FF0C0CF044
:104F6000800542EA0502C1F3072542EA050208BFAF
:104F700042F002028CEA0303A34313F0800F18BF30
:104F800042F04002E2E710B504468078617A0844B6
:104F9000C1B264480144098801F47842B2F5C05FA7
:104FA00018BF405C11D0217A01432172E07A01F0F0
:104FB000800220F0820040EA020008BF40F00200B8
:104FC000E0722088401C208010BDB1F5E05F2CBF4E
:104FD0006548664803F0B1FBE5E72DE9F04101F4CF
:104FE0007846504F04460D46B6F5C05F18BF785D51
:104FF00017D000BFE17A10F0800F14BF41F001011B
:1050000021F00101E17240064FEA1068294642464C
:10501000B5F5006F34BF07F80580B6F5C05F0FD156
:1050200007E0B1F5E05F2CBF4F48504803F085FB27
:10503000E0E7B1F5E05F2CBF4B484C4803F0F8FACD
:10504000207A50EA08012172E07A01F0800220F013
:10505000820040EA020008BF40F00200E072BDE8B2
:10506000F0812DE9F04101F478462E4F04460D46BB
:10507000B6F5C05F18BF785D16D000BFE17A10F0BA
:10508000010F14BF41F0010121F00101E1724FEA6B
:10509000500829464246B5F5006F34BF07F8058031
:1050A000B6F5C05F0FD107E0B1F5E05F2CBF2E4829
:1050B0002E4803F042FBE1E7B1F5E05F2CBF2A4840
:1050C0002A4803F0B5FA207A90EA08012172E07AC2
:1050D00001F0800220F0820040EA020008BF40F0A8
:1050E0000200E072BDE8F0812DE9F04101F478465C
:1050F0000C4F05460C46B6F5C05F18BF385D42D070
:10510000E97A10F0800F14BF41F0010321F0010390
:1051100060F35F0101F0FF08EB7221464246B4F5EF
:10512000006F29E000000010496C6C6567616C201D
:10513000696E737472756374696F6E206174202474
:10514000253034582C20253032580D0A000000003C
:105150004350552048414C5445440000505245535B
:10516000532052455345540078050120480501203D
:1051700060000020FEFF001034BF07F80480B6F581
:10518000C05F0FD107E0B1F5E05F2CBFFD48FE48DE
:1051900003F0D3FAB4E7B1F5E05F2CBFF948FA4861
:1051A00003F046FA287A10EA08012972E87A01F039
:1051B000800220F0820040EA020008BF40F00200B6
:1051C000E872BDE8F0812DE9F04101F47846EF4F37
:1051D00005460C46B6F5C05F18BF385D18D0E97AB1
:1051E00010F0010F14BF41F0010321F0010340084A
:1051F00001F0010140EAC118EB7221464246B4F5C4
:10520000006F34BF07F80480B6F5C05F0FD107E028
:10521000B1F5E05F2CBFDB48DB4803F08EFADEE738
:10522000B1F5E05F2CBFD748D74803F001FA4146FB
:105230002846FFF743FEE87A297A20F0820001F041
:1052400080021043002908BF40F00200E872BDE868
:10525000F08110B504468078617A0844CB49C0B229
:10526000084401882046FFF7B8FE2088401C2080B3
:1052700010BD10B504468078617A0844C349C0B2B5
:10528000084401882046FFF72FFF2088401C20801B
:1052900010BD10B504468078617A0844BB49C0B29D
:1052A000084401882046FFF78EFF2088401C20809C
:1052B00010BD10B504468078617A0844B349C0B285
:1052C000084401882046FFF7CCFE2088401C20803F
:1052D00010BD10B504468078617A0844C1B2AB486D
:1052E0000144098801F47842B2F5C05F18BF405C00
:1052F00011D0217A01402172E07A01F0800220F081
:10530000820040EA020008BF40F00200E0722088FC
:10531000401C208010BDB1F5E05F2CBF99489A4831
:1053200003F00BFAE5E710B504468078617A08448B
:10533000C1B296480144098801F47842B2F5C05FD1
:1053400018BF405C11D0217A41402172E07A01F00F
:10535000800220F0820040EA020008BF40F0020014
:10536000E0722088401C208010BDB1F5E05F2CBFAA
:105370008448854803F0E1F9E5E710B504468078F4
:10538000617A0844C1B281480144098801F4784235
:10539000B2F5C05F18BF405C07D001462046FFF75A
:1053A0008DFD2088401C208010BDB1F5E05F2CBF32
:1053B0007448754803F0C1F9EFE710B504468078EA
:1053C000617A227A0844C1B2704801440988B1F573
:1053D000006F2ABF01F478404254B0F5C05F06D197
:1053E000B1F5E05F2CBF6748674803F021F92088DA
:1053F000401C208010BD10B504468078627A237A64
:105400001044C1B261481A4001440988B1F5006FE7
:105410002ABF01F478404254B0F5C05F06D1B1F51F
:10542000E05F2CBF5748584803F002F92088401C21
:10543000208010BD10B504468078617A0844C1B25E
:1054400052480144098801F47842B2F5C05F18BFA0
:10545000405C0FD02072E17A00F0800221F08201DE
:105460001143002808BF41F00201E1722088401C6E
:10547000208010BDB1F5E05F2CBF4248424803F0E8
:105480005CF9E7E710B504468078617A0844C1B258
:105490003E480144098801F47842B2F5C05F18BF64
:1054A000405C10D060722072E17A00F0800221F03E
:1054B00082011143002808BF41F00201E1722088F7
:1054C000401C208010BDB1F5E05F2CBF2D482E4858
:1054D00003F033F9E6E710B504468078617A0844B2
:1054E000C1B22A480144098801F47842B2F5C05F8C
:1054F00018BF415C19D0227AE07AA2EB010320F0B8
:10550000820003F0800340EA03008A4208BF40F0B3
:105510000200E0722CBF40F0010000F0FE00E072DB
:10552000208800F10100208010BDB1F5E05F2CBFA4
:105530001448154803F001F90146DCE7F0B4C57AD8
:10554000047A0022EBB24FF0010CE6B215F0080F1E
:105550002CEA030386EA01064AD004F00F0201F0A8
:105560000F0702F580723B44D21A92B2B2F5807FE7
:105570003CBF921F92B2F02A3CBF103292B204F0AC
:10558000F00305E078050120480501200000001027
:105590001A4401F0F003D21A93B225F0C202DDB230
:1055A00015F0800F18BF42F08002641A2CEA020C3A
:1055B000A4EB0C0C1CF0FF0F08BF42F00202694084
:1055C00026EA010111F0800F18BF42F04002C3F338
:1055D0000721002918BF42F0010205D1A5F16001A1
:1055E00061F3070302F0FE020372C272F0BC70475F
:1055F00064F307026CF30F220B44D21A93B213F038
:10560000FF0C25F0C3020CF0800442EA040242EAD7
:10561000132208BF42F002028CEA010126EA0101CE
:1056200011F0800F18BF42F04002DDE710B50446CC
:105630008078617A0844C1B2FE480144098801F4C7
:105640007842B2F5C05F18BF405C07D001462046E3
:10565000FFF774FF2088401C208010BDB1F5E05F8B
:105660002CBFF548F54803F068F8EFE72DE9F04165
:1056700005468078697AEF4F0844C0B24FF00008C1
:105680003C5CB8F5C05F214618BF385D0BD0401CAC
:10569000C6B221463246B4F5006F34BF3E55B8F568
:1056A000C05F0FD107E0B1F5E05F2CBFE248E348EF
:1056B00003F043F8EBE7B1F5E05F2CBFDE48DF48CD
:1056C00002F0B6FF31462846FFF738FF2888401C15
:1056D0002880BDE8F0812DE9F04104468078617AA8
:1056E000D44F0844C0B24FF000083D5CB8F5C05F2D
:1056F000294618BF785D0BD0401EC6B229463246F7
:10570000B5F5006F34BF7E55B8F5C05F0FD107E027
:10571000B1F5E05F2CBFC848C84803F00EF8EBE7CE
:10572000B1F5E05F2CBFC448C44802F081FF207A85
:10573000E17AB0422CBF41F0010121F00101E17298
:10574000801B10F0FF01E07A01F0800220F082005F
:1057500040EA020008BF40F00200E0722088401CCE
:105760002080BDE8F08110B501880446481C2080E7
:1057700001F47840B0F5C05F1CBFAE48405C0CD06F
:105780006072E17A00F0800221F08201114300286A
:1057900008BF41F00201E17210BDB1F5E05F2CBF1E
:1057A000A548A64802F0C9FFEAE78278A14BC17A72
:1057B0009A5C038821F0C2015B1C038002F0C003E5
:1057C0001943037A134208BF41F00201C1727047C6
:1057D00010B58178827A0446B1F5006F2DBF0020A4
:1057E00094484254B0F5C05F06D1B1F5E05F2CBFDC
:1057F0009148924802F01CFF2088401C208010BD78
:1058000081788C4A525C8272C17A02F0800321F066
:1058100082011943002A08BF41F00201C1720188C8
:10582000491C018070478378DFF808C2827AC17A08
:105830001CF8033021F08301A2EB030C0CF0800C68
:1058400041EA0C01934208BF41F0020198BF41F0C8
:105850000101C172018801F1010101807047837863
:10586000DFF8D0C1427AC17A1CF8033021F08301FD
:10587000A2EB030C0CF0800C41EA0C01934208BF30
:1058800041F0020198BF41F00101C172018801F1AC
:105890000101018070478278664B017A9A5C0A4365
:1058A0000272C17A02F0800321F0820141EA030111
:1058B00008BF41F00201C1720188491C0180704794
:1058C00082785C4B017A9A5C0A400272C17A02F0DB
:1058D000800321F0820141EA030108BF41F0020187
:1058E000C1720188491C018070478278514B017A4E
:1058F0009A5C4A400272C17A02F0800321F0820170
:1059000041EA030108BF41F00201C1720188491C4C
:105910000180704710B5044680784649095C2046EE
:10592000FFF7CCFA2088401C208010BD10B581788C
:10593000027A0446B1F5006F2DBF00203D48425465
:10594000B0F5C05F06D1B1F5E05F2CBF3A483B48E7
:1059500002F06EFE2088401C208010BD8178354A00
:10596000525C0272C17A02F0800321F08201194375
:10597000002A08BF41F00201C1720188491C018060
:10598000704781782B4B027A5B5CC17AA2EB030CE7
:1059900021F082010CF0800C41EA0C019A4208BF10
:1059A00041F00201C172934294BF41F0010101F044
:1059B000FE01C1720188491C0180704710B5044680
:1059C00080781C49095C2046FFF7B8FD2088401C00
:1059D000208010BD10B504468078164A115C491C21
:1059E000C9B211542046FFF7A9FD2088401C208031
:1059F00010BD82780F4B995C491EC9B29954027A46
:105A0000C37A8A422CBF43F0010323F00103C3721F
:105A1000511A11F0FF0203F07D0102F0800341EA08
:105A2000030108BF41F00201C1720188491C0180D5
:105A30007047000000000010780501204805012093
:105A400010B48378DFF82CC4C17A1CF8032012F05C
:105A5000800F14BF41F0010101F0FE01C172510637
:105A60000A0E0CF80320C17A02F0800321F08201B3
:105A700041EA030108BF41F00201C1720188491CDB
:105A8000018010BC704710B504468078F949095C64
:105A90002046FFF7A2FA2088401C208010BD10B5D8
:105AA00004468078F349095C2046FFF71DFB2088F7
:105AB000401C208010BD10B504468078ED49095C7B
:105AC0002046FFF780FB2088401C208010BD10B5C9
:105AD00004468078E749095C2046FFF7C2FA20882F
:105AE000401C208010BD10B48378DFF888C3C17AD1
:105AF0001CF803400A4664F35F02140A14BF41F025
:105B0000010101F0FE01C17212F0FF040CF8034024
:105B1000C17AC2F3C01221F0820141EAC21108BF6A
:105B200041F00201C1720188491C018010BC70471C
:105B300010B48378DFF83CC3C17A1CF8032012F05C
:105B4000010F14BF41F0010101F0FE01C1725208C2
:105B50000CF80320C17A21F0820108BF41F0020154
:105B6000C1720188491C018010BC704730B4837831
:105B7000DFF800C3C27A1CF8031001F001044908E1
:105B800012F0010F18BF41F08001002C14BF42F049
:105B9000010202F0FE02C2720CF80310C27A01F098
:105BA000800322F082021A43002908BF42F0020259
:105BB000C2720188491C018030BC704710B58178E1
:105BC000427A0446B1F5006F2DBF0020A948425427
:105BD000B0F5C05F06D1B1F5E05F2CBFA648A7487D
:105BE00002F026FD2088401C208010BD8178A14A4B
:105BF000525C4272C17A02F0800321F082011943A3
:105C0000002A08BF41F00201C1720188491C0180CD
:105C100070478278974B995C491E11F0FF019954A7
:105C2000C27A01F0800322F0820242EA030208BF36
:105C300042F00202C2720188491C018070478278DA
:105C40008C4B995C491C11F0FF019954C27A01F008
:105C5000800322F0820242EA030208BF42F00202FD
:105C6000C2720188491C018070478549C37AD1F806
:105C700000C0017B4A1E02730CF801307047017BA3
:105C80007F4A491CC9B201731268515C41F030016E
:105C9000C17270477A49037AD1F800C0017B4A1E6D
:105CA00002730CF801307047017B754A491CC9B278
:105CB00001731268525C0272C17A02F0800321F013
:105CC00082011943002A08BF41F00201C1727047E6
:105CD000817A491E11F0FF028272C17A02F08003BC
:105CE00021F0820141EA030108BF41F00201C172C3
:105CF0007047027A8272C17A02F0800321F0820139
:105D00001943002A08BF41F00201C1727047817A2D
:105D1000491C11F0FF028272C17A02F0800321F067
:105D2000820141EA030108BF41F00201C1727047DC
:105D3000417A491C11F0FF024272C17A02F08003DD
:105D400021F0820141EA030108BF41F00201C17262
:105D50007047017A82780A430272C17A02F08003A6
:105D600021F0820141EA030108BF41F00201C17242
:105D70000188491C01807047017A82780A400272CA
:105D8000C17A02F0800321F0820141EA030108BFD9
:105D900041F00201C1720188491C01807047017AFB
:105DA00082784A400272C17A02F0800321F08201B7
:105DB00041EA030108BF41F00201C1720188491C98
:105DC0000180704710B504468178FFF777F8208886
:105DD000401C208010BD82780272C17A02F08003DC
:105DE00021F082011943002A08BF41F00201C1726B
:105DF0000188491C01807047037A8278C17AA3EB3D
:105E0000020C21F082010CF0800C41EA0C0193425B
:105E100008BF41F00201C1729A4294BF41F00101F2
:105E200001F0FE01C1720188491C0180704710B564
:105E300004468178FFF782FB2088401C208010BD3B
:105E4000027AC17A12F0800F14BF41F0010101F013
:105E5000FE01C17251060A0EC17A02F0800321F0E0
:105E6000820141EA030108BF41F00201C1720272DE
:105E7000704700000000001078050120480501204F
:105E800060000020017AC27ACB094FEA416102F03A
:105E9000010C4CEA116114BF42F0010202F0FE0253
:105EA000C27202F07D0201F080031A43002908BF8C
:105EB00042F00202C27201727047027AC17A12F095
:105EC000010F14BF41F0010101F0FE01C17252083F
:105ED00001F07D0108BF41F00201C17202727047FA
:105EE000017AC27A01F00103490812F0010F18BFCC
:105EF00041F08001002B14BF42F0010202F0FE02CB
:105F0000C27202F07D0201F080031A43002908BF2B
:105F100042F00202C27201727047427A0272C17A82
:105F200002F0800321F082011943002A08BF41F0EA
:105F30000201C1727047027A4272C17A02F0800394
:105F400021F082011943002A08BF41F00201C17209
:105F50007047417A491E11F0FF024272C17A02F085
:105F6000800321F0820141EA030108BF41F00201F0
:105F7000C1727047704710B54188044601F47840FB
:105F8000B0F5C05F1CBFFE48405C10D0E17A227AB9
:105F900021F0C20102420CBF02220022114300F094
:105FA000C0000843E0722088801C208010BDB1F53D
:105FB000E05F2CBFF348F44802F0BFFBE6E74188FE
:105FC000018070472DE9F041418805464A1C01F4E3
:105FD0007F40D2B240EA020401F47840E84FB0F5C5
:105FE000C05F18BF7E5C0CD004F478402146B0F549
:105FF000C05F18BF385D0DD046EA00202880BDE89C
:10600000F081B1F5E05F2CBFDE48DF4802F095FB80
:106010000646E9E7B1F5E05F2CBFDA48DA4802F05E
:106020008CFBE9E710B54188827A0446B1F5006F30
:106030002DBF01F47840D2484254B0F5C05F06D17C
:10604000B1F5E05F2CBFCF48CF4802F0F1FA2088CD
:10605000801C208010BD10B54188044601F47840B2
:10606000B0F5C05F1CBFC648405C0FD0A072E17A9B
:1060700000F0800221F082011143002808BF41F0A6
:106080000201E1722088801C208010BDB1F5E05F24
:106090002CBFBC48BC4802F050FBE7E770B5418814
:1060A0000446857A01F47840B0F5C05F1CBFB4485F
:1060B000405C15D0E17A2A1A21F0830102F08002B7
:1060C000114385420CBF022200221143A84294BF13
:1060D000012000200843E0722088801C208070BDD1
:1060E000B1F5E05F2CBFA748A74802F026FBE1E727
:1060F00070B541880446457A01F47840B0F5C05F38
:106100001CBF9F48405C15D0E17A2A1A21F0830118
:1061100002F08002114385420CBF0222002211438B
:10612000A84294BF012000200843E0722088801C10
:10613000208070BDB1F5E05F2CBF9248924802F01C
:10614000FCFAE1E710B54188044601F47840B0F567
:10615000C05F1CBF8A48405C11D0217A0143217284
:10616000E07A01F0800220F0820040EA020008BFDD
:1061700040F00200E0722088801C208010BDB1F544
:10618000E05F2CBF7F48804802F0D7FAE5E710B502
:106190004188044601F47840B0F5C05F1CBF7848E0
:1061A000405C11D0217A01402172E07A01F0800236
:1061B00020F0820040EA020008BF40F00200E072D6
:1061C0002088801C208010BDB1F5E05F2CBF6D4899
:1061D0006D4802F0B2FAE5E710B54188044601F4D3
:1061E0007840B0F5C05F1CBF6548405C11D0217A93
:1061F00041402172E07A01F0800220F0820040EA02
:10620000020008BF40F00200E0722088801C20805D
:1062100010BDB1F5E05F2CBF5A485B4802F08DFA23
:10622000E5E710B54188044601F47840B0F5C05F59
:106230001CBF5348405C07D001462046FEF73EFE97
:106240002088801C208010BDB1F5E05F2CBF4D4838
:106250004D4802F072FAEFE710B54188027A044621
:10626000B1F5006F2DBF01F4784045484254B0F5B8
:10627000C05F06D1B1F5E05F2CBF4248424802F052
:10628000D7F92088801C208010BD10B541880446B5
:1062900001F47840B0F5C05F1CBF3948405C0FD0B6
:1062A0002072E17A00F0800221F08201114300287F
:1062B00008BF41F00201E1722088801C208010BDDF
:1062C000B1F5E05F2CBF2F482F4802F036FAE7E720
:1062D00070B541880446057A01F47840B0F5C05F96
:1062E0001CBF2748405C15D0E17AA5EB000221F0E5
:1062F000830102F0800241EA0201A84208BF41F096
:10630000020198BF41F00101E172208800F1020012
:10631000208070BDB1F5E05F2CBF1A481A4802F02A
:106320000CFAE1E710B54188044601F47840B0F575
:10633000C05F1CBF1248405C07D001462046FFF7F3
:10634000FDF82088801C208010BDB1F5E05F2CBFD7
:106350000C480D4802F0F1F9EFE770B541880446AA
:1063600001F47840064EB0F5C05F18BF705C15D0E0
:10637000401C6188C5B22A46B1F5006F06E00000F6
:106380000000001078050120480501202ABF01F413
:1063900078407554B0F5C05F0FD107E0B1F5E05F0C
:1063A0002CBFF948F94802F0C8F9E1E7B1F5E05F20
:1063B0002CBFF548F54802F03BF929462046FFF787
:1063C000BDF82088801C208070BD70B541880446CF
:1063D00001F47840EE4EB0F5C05F18BF705C0DD090
:1063E000401E6188C5B22A46B1F5006F2ABF01F48C
:1063F00078407554B0F5C05F0FD107E0B1F5E05FAC
:106400002CBFE148E14802F098F9E9E7B1F5E05F17
:106410002CBFDD48DD4802F00BF9207AE17AA84272
:106420002CBF41F0010121F00101E172401B10F08D
:10643000FF01E07A01F0800220F0820040EA0200D1
:1064400008BF40F00200E0722088401C208070BD30
:1064500070B54188044601F47840CD4EB0F5C05F78
:1064600018BF705C17D000BFE17A10F0800F14BF26
:1064700041F0010101F0FE01E1724006050E618864
:106480002A46B1F5006F2ABF01F478407554B0F583
:10649000C05F0FD107E0B1F5E05F2CBFBA48BB4841
:1064A00002F04BF9E0E7B1F5E05F2CBFB648B74822
:1064B00002F0BEF8E07A05F0800120F08200084387
:1064C000002D08BF40F00200E0722088801C208070
:1064D00070BD10B504464188FEF77FFD2088801C02
:1064E000208010BD10B504464188FEF7FDFD2088D0
:1064F000801C208010BD10B504464188FEF763FE65
:106500002088801C208010BD10B504464188FEF70D
:10651000A8FD2088801C208010BD70B541880446ED
:1065200001F478409A4EB0F5C05F18BF705C17D088
:10653000E17AC2090B4660F35F03DDB214BF41F09C
:10654000010001F0FE00E07261882A46B1F5006F9B
:106550002ABF01F478407554B0F5C05F0FD107E051
:10656000B1F5E05F2CBF8848884802F0E6F8DFE725
:10657000B1F5E05F2CBF8448844802F059F8E07A16
:1065800005F0800120F082000843002D08BF40F094
:106590000200E0722088801C208070BD70B54188A8
:1065A000044601F478407A4EB0F5C05F18BF705CC5
:1065B00016D000BFE17A10F0010F14BF41F00101C5
:1065C00001F0FE01E172450861882A46B1F5006FCD
:1065D0002ABF01F478407554B0F5C05F0FD107E0D1
:1065E000B1F5E05F2CBF6848684802F0A6F8E1E723
:1065F000B1F5E05F2CBF6448644802F019F8E07A16
:10660000002D20F0820008BF40F00200E0722088D8
:10661000801C208070BD70B54188044601F478402C
:106620005B4EB0F5C05F18BF705C1BD000F001017D
:106630004508E07A10F0010F18BF45F080050029E9
:1066400014BF40F0010000F0FE00E07261882A46AD
:10665000B1F5006F2ABF01F478407554B0F5C05F02
:106660000FD107E0B1F5E05F2CBF4748474802F083
:1066700064F8DBE7B1F5E05F2CBF4348434801F025
:10668000D7FFE07A05F0800120F082000843002D5A
:1066900008BF40F00200E0722088801C208070BD9E
:1066A00010B54188427A0446B1F5006F2DBF01F460
:1066B000784037484254B0F5C05F06D1B1F5E05F8D
:1066C0002CBF3148314801F0B3FF2088801C208066
:1066D00010BD10B54188044601F47840B0F5C05FA4
:1066E0001CBF2B48405C0FD06072E17A00F0800242
:1066F00021F082011143002808BF41F00201E1723C
:106700002088801C208010BDB1F5E05F2CBF1E48A2
:106710001E4802F012F8E7E770B54188044601F41C
:1067200078401B4EB0F5C05F18BF705C0DD0401EA6
:106730006188C5B22A46B1F5006F2ABF01F47840DE
:106740007554B0F5C05F0FD107E0B1F5E05F2CBF25
:106750000D480E4801F0F1FFE9E7B1F5E05F2CBF0D
:1067600009480A4801F064FFE07A05F0800120F052
:1067700082000843002D08BF40F00200E07220882C
:10678000801C208070BD0000780501204805012094
:106790000000001070B54188044601F47840FE4EB8
:1067A000B0F5C05F18BF705C0DD0401C6188C5B2E9
:1067B0002A46B1F5006F2ABF01F478407554B0F550
:1067C000C05F0FD107E0B1F5E05F2CBFF348F4489C
:1067D00001F0B3FFE9E7B1F5E05F2CBFEF48F04807
:1067E00001F026FFE07A05F0800120F082000843E6
:1067F000002D08BF40F00200E0722088801C20803D
:1068000070BD0188C37A4A1C114613F0800F01D075
:106810000180704790F90230D118120AB2EB112FA3
:1068200014BF0222012243681A444260F0E7018843
:10683000C37A4A1C114613F0800F0BD090F9023036
:10684000D118120AB2EB112F0CBF012202224368A9
:106850001A444260018070470188C37A4A1C11467D
:1068600013F0400F01D00180704790F90230D11829
:10687000120AB2EB112F14BF0222012243681A44FC
:106880004260F0E70188C37A4A1C114613F0400FBA
:106890000BD090F90230D118120AB2EB112F0CBFB5
:1068A0000122022243681A44426001807047018835
:1068B000C37A4A1C114613F0010F01D001807047C2
:1068C00090F90230D118120AB2EB112F14BF022234
:1068D000012243681A444260F0E70188C37A4A1CE7
:1068E000114613F0010F0BD090F90230D118120AA3
:1068F000B2EB112F0CBF0122022243681A444260FE
:10690000018070470188C37A4A1C114613F0020FB8
:1069100001D00180704790F90230D118120AB2EB11
:10692000112F14BF0222012243681A444260F0E78B
:106930000188C37A4A1C114613F0020F0BD090F95C
:106940000230D118120AB2EB112F0CBF0122022221
:1069500043681A4442600180704770B504468178EC
:106960008D48A57A01440E88711989B201F47842E4
:10697000B2F5C05F18BF405C18D0217A0143217284
:1069800055FA86F0000A02D06068401C6060E07A28
:1069900001F0800220F082001043002908BF40F07F
:1069A0000200E0722088401C208070BDB1F5E05FDD
:1069B0002CBF7A487A4801F0C0FEDEE770B5044685
:1069C00081787548A57A01440E88711989B201F45D
:1069D0007842B2F5C05F18BF405C0ED00146204639
:1069E000FEF7FBFA55FA86F0000A02D06068401CF8
:1069F00060602088401C208070BDB1F5E05F2CBF36
:106A00006648674801F099FEE8E770B5044681786A
:106A10006148A57A01440E88711989B201F478425F
:106A2000B2F5C05F18BF405C0ED001462046FEF7AD
:106A300018FB55FA86F0000A02D06068401C6060BE
:106A40002088401C208070BDB1F5E05F2CBF53480A
:106A5000534801F072FEE8E770B5044681784E486D
:106A6000A57A01440E88711989B201F47842B2F511
:106A7000C05F18BF405C0ED001462046FEF734FBD5
:106A800055FA86F0000A02D06068401C60602088D9
:106A9000401C208070BDB1F5E05F2CBF3F484048EE
:106AA00001F04BFEE8E770B5044681783A48A57AD4
:106AB00001440E88711989B201F47842B2F5C05FC1
:106AC00018BF405C18D0217A0140217255FA86F037
:106AD000000A02D06068401C6060E07A01F0800229
:106AE00020F082001043002908BF40F00200E0724D
:106AF0002088401C208070BDB1F5E05F2CBF274886
:106B0000274801F01AFEDEE770B504468178224876
:106B1000A57A01440E88711989B201F47842B2F560
:106B2000C05F18BF405C18D0217A4140217255FAED
:106B300086F0000A02D06068401C6060E07A01F0D4
:106B4000800220F082001043002908BF40F00200BC
:106B5000E0722088401C208070BDB1F5E05F2CBF42
:106B60000E480F4801F0E9FDDEE770B50446817874
:106B70000948A57A01440E88711989B201F4784256
:106B8000B2F5C05F18BF405C15D001462046FEF745
:106B900095F955FA86F005E000000010780501200F
:106BA00048050120000A02D06068401C606020880F
:106BB000401C208070BDB1F5E05F2CBFFD48FE4851
:106BC00001F0BBFDE1E710B504468178FB48A27AED
:106BD00001440988114489B2227AB1F5006F2ABFB5
:106BE00001F478404254B0F5C05F06D1B1F5E05FE2
:106BF0002CBFF048F04801F01BFD2088401C20808D
:106C000010BD70B504468178EC48A57A01440E8821
:106C1000711989B201F47842B2F5C05F18BF405CC7
:106C200016D0207255FA86F1090A02D06168491C13
:106C30006160E17A00F0800221F0820111430028B6
:106C400008BF41F00201E1722088401C208070BD25
:106C5000B1F5E05F2CBFD748D74801F06EFDE0E703
:106C600070B504468178D548A57A01440E8871191B
:106C700089B201F47842B2F5C05F18BF405C17D00A
:106C80006072207255FA86F1090A02D06168491CC7
:106C90006160E17A00F0800221F082011143002856
:106CA00008BF41F00201E1722088401C208070BDC5
:106CB000B1F5E05F2CBFBF48BF4801F03EFDDFE704
:106CC0002DE9F04104468178BC48A67A0144257A32
:106CD0000F88B91989B201F47842B2F5C05F18BFC4
:106CE000415C1ED056FA87F0000A02D06068401C52
:106CF0006060E07A6A1A20F0820002F0800210439D
:106D00008D4208BF40F00200E072A94294BF40F0FB
:106D1000010000F0FE00E0722088401C2080BDE8E9
:106D2000F081B1F5E05F2CBFA248A34801F005FD5A
:106D30000146D7E770B504468178A048A57A01449A
:106D40000E88711989B201F47842B2F5C05F18BF9C
:106D5000405C0ED001462046FEF7F0FB55FA86F067
:106D6000000A02D06068401C60602088401C2080BF
:106D700070BDB1F5E05F2CBF8E488F4801F0DDFC9F
:106D8000E8E72DE9F04104468078DFF83082A77A01
:106D900040440588E81981B201F47840B0F5C05F3D
:106DA00018BF18F801000ED0401CC2B21646294682
:106DB000B5F5006F2ABF01F4784008F80560B0F51A
:106DC000C05F0FD107E0B1F5E05F2CBF79487A488A
:106DD00001F0B3FCE8E7B1F5E05F2CBF75487648F9
:106DE00001F026FC31462046FEF7A8FB57FA85F055
:106DF000000A02D06068401C60602088401C20802F
:106E0000BDE8F0812DE9F04104468078DFF8AC81DF
:106E1000A77A40440588E81981B201F47840B0F5BA
:106E2000C05F18BF18F801000ED0401EC2B216464F
:106E30002946B5F5006F2ABF01F4784008F80560CF
:106E4000B0F5C05F0FD107E0B1F5E05F2CBF594846
:106E5000594801F072FCE8E7B1F5E05F2CBF5548F6
:106E6000554801F0E5FB207AE17AB0422CBF41F0B1
:106E7000010121F00101E172801B10F0FF01E07AB5
:106E800001F0800220F0820040EA020008BF40F0DA
:106E90000200E07257FA85F0000A02D06068401CD8
:106EA00060602088401C2080BDE8F08110B5044659
:106EB0008078617AA27A0844C1B2B1F5006F2DBF23
:106EC00000203E484254B0F5C05F06D1B1F5E05F06
:106ED0002CBF3848384801F0ABFB2088401C20808C
:106EE00010BD10B504468078617A0844C1B2002014
:106EF000B0F5C05F1CBF3148405C0FD0A072E17A92
:106F000000F0800221F082011143002808BF41F007
:106F10000201E1722088401C208010BDB1F5E05FC5
:106F20002CBF2448244801F008FCE7E78178427A26
:106F30001144224A52FA81F10978027A0A43027214
:106F4000C17A02F0800321F0820141EA030108BF07
:106F500041F00201C1720188491C018070478178AB
:106F6000427A1144154A52FA81F10978027A0A40AC
:106F70000272C17A02F0800321F0820141EA03012A
:106F800008BF41F00201C1720188491C01807047AD
:106F90008178427A1144094A52FA81F10978027AD9
:106FA0004A400272C17A02F0800321F0820141EA74
:106FB000030105E0780501204805012000000010CC
:106FC00008BF41F00201C1720188491C018070476D
:106FD00010B504468078617A0844F64951FA80F089
:106FE00001782046FDF76AFF2088401C208010BDF4
:106FF0008278437A017A1A44EE4B53FA82F2117086
:107000000188491C018070478178427A1144E94A1D
:1070100052FA81F10A780272C17A02F0800321F0FB
:1070200082011943002A08BF41F00201C1720188A0
:10703000491C018070478178427A037A1144DD4A05
:1070400052FA81F10A78C17AA3EB020C21F0820195
:107050000CF0800C41EA0C01934208BF41F00201A0
:10706000C1729A4294BF41F0010101F0FE01C17268
:107070000188491C0180704710B504468078617A08
:107080000844CC4951FA80F001782046FEF756FAC0
:107090002088401C208010BD10B504468078617A9D
:1070A000C44A0844C0B2115C491CC9B211542046FC
:1070B000FEF744FA2088401C208010BD8178427A77
:1070C000BC4B1144CAB2995C491EC9B29954027AA8
:1070D000C37A8A422CBF43F0010323F00103C37239
:1070E000511A11F0FF0203F07D0102F0800341EA22
:1070F000030108BF41F00201C1720188491C0180EF
:10710000704710B48178427ADFF8A8C21144C9B23E
:10711000C27A1CF8013013F0800F14BF42F0010254
:1071200002F0FE02C2725A06120E0CF80120C17A59
:1071300002F0800321F0820141EA030108BF41F01F
:107140000201C1720188491C018010BC704710B552
:1071500004468078617A0844C1B22046FDF73DFFBD
:107160002088401C208010BD10B504468078617ACC
:107170000844C1B22046FDF774FF2088401C2080DF
:1071800010BD10B504468078617A0844C1B220462B
:10719000FDF7AAFF2088401C208010BD10B50446D2
:1071A0008078617A0844C1B22046FEF70CF8208846
:1071B000401C208010BD30B48178427ADFF8F4C1E1
:1071C0001144CAB2C37A1CF8021003F00105CC09BD
:1071D0004FEA416145EA116114BF43F0010303F036
:1071E000FE03C3720CF80210C27A01F0800322F091
:1071F00082021A43002908BF42F00202C2720188CB
:10720000491C018030BC704710B48178427ADFF8A5
:10721000A4C11144CAB2C17A1CF8023013F0010FA4
:1072200014BF41F0010101F0FE01C1725B080CF8CE
:107230000230C17A21F0820108BF41F00201C1721F
:107240000188491C018010BC704730B48178427AB3
:10725000DFF860C11144CAB2C37A1CF8021001F011
:107260000104490813F0010F18BF41F08001002C00
:1072700014BF43F0010303F0FE03C3720CF80210C5
:10728000C27A01F0800322F082021A43002908BF6B
:1072900042F00202C2720188491C018030BC704772
:1072A0008278837A417A1A44424B53FA82F21170FF
:1072B0000188491C01807047017A427A837A114023
:1072C00082781A443B4B53FA82F211700188491CB0
:1072D000018070478178827A1144364A52FA81F1EE
:1072E0000A784272C17A02F0800321F082011943C8
:1072F000002A08BF41F00201C1720188491C0180C7
:1073000070478178827A11442A4A52FA81F10A78C8
:1073100042720272C17A02F0800321F082011943A5
:10732000002A08BF41F00201C1720188491C018096
:1073300070478178427A1F4B1144CAB2995C491E4A
:1073400011F0FF019954C27A01F0800322F0820209
:1073500042EA030208BF42F00202C2720188491CDD
:10736000018070478178427A124B1144CAB2995C0D
:10737000491C11F0FF019954C27A01F0800322F0F8
:10738000820242EA030208BF42F00202C27201888E
:10739000491C01807047C17A21F00101C172704718
:1073A000C17A41F00101C1727047C17A21F0040134
:1073B000C172704700000010C17A41F00401C1722F
:1073C0007047827A0272C17A02F0800321F0820152
:1073D0001943002A08BF41F00201C1727047C17A07
:1073E00021F04001C1727047C17A21F00801C172D9
:1073F0007047C17A41F00801C172704770B5468884
:10740000857A0446701981B201F47840B0F5C05F06
:107410001CBFF848405C18D0217A0143217255FA0C
:1074200086F0000A02D06068401C6060E07A01F0DB
:10743000800220F082001043002908BF40F00200C3
:10744000E0722088801C208070BDB1F5E05F2CBF09
:10745000E948EA4801F071F9DEE770B54588867AB7
:107460000446A81981B22046FDF7B7FD56FA85F00B
:10747000000A02D06068401C60602088801C208068
:1074800070BD70B54588867A0446A81981B2204639
:10749000FDF7E7FD56FA85F0000A02D06068401C4F
:1074A00060602088801C208070BD70B54588867A19
:1074B0000446A81981B22046FDF716FE56FA85F05B
:1074C000000A02D06068401C60602088801C208018
:1074D00070BD70B54588867A0446A81981B22046E9
:1074E000FDF771FE56FA85F0000A02D06068401C74
:1074F00060602088801C208070BD70B54688857AC9
:107500000446701981B201F47840B0F5C05F1CBF29
:10751000B848405C18D0217A0140217255FA86F0B3
:10752000000A02D06068401C6060E07A01F08002CE
:1075300020F082001043002908BF40F00200E072F2
:107540002088801C208070BDB1F5E05F2CBFAA4868
:10755000AA4801F0F2F8DEE770B54688857A04465D
:10756000701981B201F47840B0F5C05F1CBFA1482A
:10757000405C18D0217A4140217255FA86F0000A09
:1075800002D06068401C6060E07A01F0800220F068
:1075900082001043002908BF40F00200E0722088FA
:1075A000801C208070BDB1F5E05F2CBF92489348ED
:1075B00001F0C3F8DEE770B54688857A0446701995
:1075C00081B201F47840B0F5C05F1CBF8948405CCF
:1075D0000ED001462046FDF771FC55FA86F0000AF0
:1075E00002D06068401C60602088801C208070BDD4
:1075F000B1F5E05F2CBF8048804801F09EF8E8E7D5
:1076000010B504464088A17A227A084481B2B1F5C7
:10761000006F2DBF01F4784076484254B0F5C05F4A
:1076200006D1B1F5E05F2CBF7348744801F000F853
:107630002088801C208010BD70B54688857A04465D
:10764000701981B201F47840B0F5C05F1CBF694881
:10765000405C16D0207255FA86F1090A02D06168A2
:10766000491C6160E17A00F0800221F0820111433F
:10767000002808BF41F00201E1722088801C2080B0
:1076800070BDB1F5E05F2CBF5B485C4801F055F878
:10769000E0E770B54688857A0446701981B201F436
:1076A0007840B0F5C05F1CBF5248405C1AD0217BC7
:1076B000084020736072207255FA86F1090A02D0E0
:1076C0006168491C6160E17A00F0800221F082016A
:1076D0001143002808BF41F00201E1722088801C9C
:1076E000208070BDB1F5E05F2CBF4348434801F0F6
:1076F00024F8DCE770B54688857A0446701981B2B3
:1077000001F47840B0F5C05F1CBF3A48415C20D01E
:1077100055FA86F0000A02D06068401C6060227A48
:10772000E07AA2EB010320F0820003F0800340EA3C
:1077300003008A4208BF40F00200E0722CBF40F014
:10774000010000F0FE00E072208800F102002080BD
:1077500070BDB1F5E05F2CBF2748284800F0EDFF71
:107760000146D5E770B54688857A0446701981B21E
:1077700001F47840B0F5C05F1CBF1E48405C0ED0DD
:1077800001462046FDF7DAFE55FA86F0000A02D0DF
:107790006068401C60602088801C208070BDB1F54E
:1077A000E05F2CBF1448154800F0C7FFE8E72DE95B
:1077B000F0474688857ADFF83C8006EB05091FFA1A
:1077C00089F101F478470446B7F5C05F18BF18F88F
:1077D000010015D0401C00F0FF0A1FFA89F1524643
:1077E000B1F5006F34BF08F801A0B7F5C05F16D13E
:1077F0000EE000000000001078050120480501207F
:10780000B1F5E05F2CBFFB48FB4800F096FFE1E7D5
:10781000B1F5E05F2CBFF748F74800F009FF51468B
:107820002046FDF78BFE55FA86F0000A02D060680C
:10783000401C60602088801C2080BDE8F0872DE916
:10784000F0474788867ADFF8B49307EB060A1FFAF9
:107850008AF101F478480446B8F5C05F18BF19F8FA
:1078600001000DD0401EC5B21FFA8AF12A46B1F5BB
:10787000006F34BF09F80150B8F5C05F0FD107E0C1
:10788000B1F5E05F2CBFDB48DB4800F056FFE9E7CD
:10789000B1F5E05F2CBFD748D74800F0C9FE207A89
:1078A000E17AA8422CBF41F0010121F00101E1720F
:1078B000401B10F0FF01E07A01F0800220F082000E
:1078C00040EA020008BF40F00200E07256FA87F07A
:1078D000000A02D06068401C60602088401C208044
:1078E000BDE8F087417A01737047027B4272C17A2A
:1078F00002F0800321F082011943002A08BF41F001
:107900000201C172704710B504464088617A08448C
:1079100081B201F47840B0F5C05F1CBFB748405C4D
:107920000FD0A072E17A00F0800221F082011143B1
:10793000002808BF41F00201E1722088801C2080ED
:1079400010BDB1F5E05F2CBFAA48AB4800F0F5FED2
:10795000E7E770B54688457A0446701981B201F4AC
:107960007840B0F5C05F1CBFA448405C18D0217AB5
:107970000143217255FA86F0000A02D06068401C6B
:107980006060E07A01F0800220F08200104300295C
:1079900008BF40F00200E0722088801C208070BD8B
:1079A000B1F5E05F2CBF9348934800F0C6FEDEE7D8
:1079B00070B54688457A0446701981B201F4784062
:1079C000B0F5C05F1CBF8D48405C18D0217A0140E3
:1079D000217255FA86F0000A02D06068401C60608F
:1079E000E07A01F0800220F082001043002908BFF5
:1079F00040F00200E0722088801C208070BDB1F54C
:107A0000E05F2CBF7B487C4800F097FEDEE770B556
:107A10004688457A0446701981B201F47840B0F581
:107A2000C05F1CBF7548405C18D0217A414021726C
:107A300055FA86F0000A02D06068401C6060E07A67
:107A400001F0800220F082001043002908BF40F0BE
:107A50000200E0722088801C208070BDB1F5E05FDC
:107A60002CBF6448644800F068FEDEE770B54688C5
:107A7000457A0446701981B201F47840B0F5C05FD0
:107A80001CBF5E48405C0ED001462046FDF716FA4A
:107A900055FA86F0000A02D06068401C60602088B9
:107AA000801C208070BDB1F5E05F2CBF514852486A
:107AB00000F043FEE8E710B504464088617A227A78
:107AC000084481B2B1F5006F2DBF01F478404B48F6
:107AD0004254B0F5C05F06D1B1F5E05F2CBF454818
:107AE000454800F0A5FD2088801C208010BD70B5A1
:107AF0004688457A0446701981B201F47840B0F5A1
:107B0000C05F1CBF3D48405C16D0207255FA86F11C
:107B1000090A02D06168491C6160E17A00F08002C4
:107B200021F082011143002808BF41F00201E172F7
:107B30002088801C208070BDB1F5E05F2CBF2D48EF
:107B40002D4800F0FAFDE0E770B54688457A044616
:107B5000701981B201F47840B0F5C05F1CBF2748AE
:107B6000415C20D055FA86F0000A02D06068401CC3
:107B70006060227AE07AA2EB010320F0820003F039
:107B8000800340EA03008A4208BF40F00200E0722E
:107B90002CBF40F0010000F0FE00E072208800F1F0
:107BA0000200208070BDB1F5E05F2CBF1148124883
:107BB00000F0C3FD0146D5E770B54688457A044616
:107BC000701981B201F47840B0F5C05F1CBF0B485A
:107BD000405C15D001462046FDF7B0FC55FA86F012
:107BE000000A02D06068401C60602088801C2080F1
:107BF00070BD00007805012048050120000000103C
:107C0000B1F5E05F2CBFF848F84800F096FDE1E7D9
:107C10002DE9F0474688457ADFF8D48306EB05095D
:107C20001FFA89F101F478470446B7F5C05F18BF21
:107C300018F801000ED0401C00F0FF0A1FFA89F16D
:107C40005246B1F5006F34BF08F801A0B7F5C05F28
:107C50000FD107E0B1F5E05F2CBFE348E34800F047
:107C60006CFDE8E7B1F5E05F2CBFDF48DF4800F0CE
:107C7000DFFC51462046FDF761FC55FA86F0000A0C
:107C800002D06068401C60602088801C2080BDE8B5
:107C9000F0872DE9F0474788467ADFF8549307EBE1
:107CA000060A1FFA8AF101F478480446B8F5C05F65
:107CB00018BF19F801000DD0401CC5B21FFA8AF197
:107CC0002A46B1F5006F34BF09F80150B8F5C05F1E
:107CD0000FD107E0B1F5E05F2CBFC348C34800F007
:107CE0002CFDE9E7B1F5E05F2CBFBF48BF4800F0CD
:107CF0009FFC207AE17AA8422CBF41F0010121F0DB
:107D00000101E172401B10F0FF01E07A01F08002F6
:107D100020F0820040EA020008BF40F00200E0725A
:107D200056FA87F0000A02D06068401C6060208824
:107D3000401C2080BDE8F0872DE9F0410546407ADF
:107D40006988DFF8AC82084484B204F4784721469D
:107D5000B7F5C05F18BF18F8040015D0E97A10F025
:107D6000800F14BF41F0010101F0FE01E9724006ED
:107D7000060E21463246B4F5006F34BF08F80460A1
:107D8000B7F5C05F0FD107E0B1F5E05F2CBF9648B3
:107D9000964800F0D2FCE1E7B1F5E05F2CBF9248D5
:107DA000924800F045FCE87A06F0800120F082005D
:107DB0000843002E08BF40F00200E8722888801CAB
:107DC0002880BDE8F08110B504464088617A0844F7
:107DD00081B22046FDF701F92088801C208010BD6B
:107DE00010B504464088617A084481B22046FDF708
:107DF00038F92088801C208010BD10B504464088CA
:107E0000617A084481B22046FDF76EF92088801C13
:107E1000208010BD10B504464088617A084481B2C4
:107E20002046FDF7D0F92088801C208010BD2DE968
:107E3000F0410546407A6988DFF8B481084484B28D
:107E400004F478472146B7F5C05F18BF18F804005E
:107E50001AD0C1094FEA40604FEA1062E87A00F098
:107E6000010343EA020614BF40F0010000F0FE00E7
:107E7000E87221463246B4F5006F34BF08F804605A
:107E8000B7F5C05F0FD107E0B1F5E05F2CBF5648F2
:107E9000564800F052FCDCE7B1F5E05F2CBF5248D9
:107EA000524800F0C5FBE87A06F0800120F082001D
:107EB0000843002E08BF40F00200E8722888801CAA
:107EC0002880BDE8F0812DE9F0410446407A6188C0
:107ED000474F084485B205F478462946B6F5C05F99
:107EE00018BF785D16D000BFE17A10F0010F14BF03
:107EF00041F0010101F0FE01E1724FEA500829460C
:107F00004246B5F5006F34BF07F80580B6F5C05F8F
:107F10000FD107E0B1F5E05F2CBF3348334800F0E4
:107F20000CFCE1E7B1F5E05F2CBF2F482F4800F0D3
:107F30007FFBE07AB8F1000F20F0820008BF40F02C
:107F40000200E0722088801C2080BDE8F0812DE9CD
:107F5000F0410546407A6988DFF89480084484B28D
:107F600004F478472146B7F5C05F18BF18F804003D
:107F70001BD000BF00F001014608E87A10F0010FA5
:107F800018BF46F08006002914BF40F0010000F041
:107F9000FE00E87221463246B4F5006F34BF08F89F
:107FA0000460B7F5C05F0FD107E0B1F5E05F2CBF0B
:107FB0000D480E4800F0C1FBDCE7B1F5E05F2CBFD7
:107FC00009480A4800F034FBE87A06F0800120F006
:107FD00082000843002E08BF40F00200E8722888A3
:107FE000801C2880BDE8F08178050120480501202B
:107FF0000000001010B504464088A17A084481B200
:1080000001F47840B0F5C05F1CBFFE48405C0FD063
:108010006072E17A00F0800221F0820111430028B1
:1080200008BF41F00201E1722088801C208010BD51
:10803000B1F5E05F2CBFF448F44800F07EFBE7E7C1
:108040002DE9F0410546807A6988DFF8B883084455
:1080500084B204F478472146B7F5C05F18BF18F81A
:1080600004000CD0401EC6B221463246B4F5006F63
:1080700034BF08F80460B7F5C05F0FD107E0B1F571
:10808000E05F2CBFE048E14800F057FBEAE7B1F5BC
:10809000E05F2CBFDC48DD4800F0CAFAE87A06F061
:1080A000800120F082000843002E08BF40F002004B
:1080B000E8722888801C2880BDE8F0812DE9F04115
:1080C0000546807A6988DFF83C83084484B204F46A
:1080D00078472146B7F5C05F18BF18F804000CD0E8
:1080E000401CC6B221463246B4F5006F34BF08F8D2
:1080F0000460B7F5C05F0FD107E0B1F5E05F2CBFBA
:10810000C148C24800F019FBEAE7B1F5E05F2CBFB7
:10811000BD48BE4800F08CFAE87A06F0800120F0F5
:1081200082000843002E08BF40F00200E872288851
:10813000801C2880BDE8F081017A827811400172AC
:10814000C27A11F0800F14BF42F0010222F0010246
:10815000C27202F07D0201F080031A43002908BFB9
:1081600042F00202C2720188491C01807047017A04
:10817000827811400172C27A11F0010F14BF42F0EF
:10818000010202F0FE02C2724A080272C17A21F0B4
:10819000820108BF41F00201C1720188491C0180BF
:1081A0007047017A82781140C27A02F0010341EAF5
:1081B0000321490822F0820201F08003017242EAA1
:1081C000030208BF42F00202C2720188491C01800A
:1081D0007047017A427A8B4B11408278995401881A
:1081E000491C0180704710B504464188007A627AC4
:1081F0000240B1F5006F2DBF01F478408148425430
:10820000B0F5C05F06D1B1F5E05F2CBF7E487F4876
:1082100000F00EFA2088801C208010BD8178794AF9
:10822000515C41720172C27A01F0800322F0820235
:108230001A43002908BF42F00202C2720188491C99
:1082400001807047817841720172C27A01F0800327
:1082500022F082021A43002908BF42F00202C272D1
:108260000188491C01807047417A82780A40027275
:10827000C17A02F0800321F0820141EA030108BFC4
:1082800041F00201C1720188491C0180704710B59C
:108290004188044601F47840B0F5C05F1CBF5948DE
:1082A000405C10D060722072E17A00F0800221F010
:1082B00082011143002808BF41F00201E1722088C9
:1082C000801C208010BDB1F5E05F2CBF4E484F48A8
:1082D00000F033FAE6E710B504464088A17A084476
:1082E00081B201F47840B0F5C05F1CBF4548405CE6
:1082F00010D060722072E17A00F0800221F08201D9
:108300001143002808BF41F00201E1722088801C5F
:10831000208010BDB1F5E05F2CBF3B483B4800F02A
:108320000CFAE6E7417A037A82780B40C17A9342ED
:108330002CBF41F0010121F00101C172991A11F025
:10834000FF024272C17A02F0800321F0820141EA09
:10835000030108BF41F00201C1720188491C01807C
:1083600070470188491C018070470188891C018081
:1083700070474FF0E0222649136923F0020313618E
:1083800000224A73244B8873224818608A724A720A
:108390000A723020C8722148FF230B7300880880BE
:1083A0001A481949DFF878C0026042608260C260F2
:1083B000026142618261C2610A604A608A60CA6089
:1083C0000A614A618A61CA61C0F820C0DFF854C0FE
:1083D000C0F824C0DFF850C0C0F828C0DFF84CC097
:1083E000C0F82CC0DFF848C0DCF800C04FEA1C2CF5
:1083F00080F817C0C3740F4808620F4848620F48DE
:1084000088621DE000000010780501204805012069
:10841000240501200001001060000020FCFF001076
:10842000BF870008E3870008EB870008ED87000896
:1084300010040240BF880008C5880008FB880008B7
:108440005448C862CB748A775349FA2008600020E8
:1084500000F0CCB9514CFFF78CFF0020E073A8214D
:108460004F4FDFF840A1DFF840B14FF6FE704FF0FC
:108470000D094FF0E02507EB0008CE06C4F81810F0
:10848000C6F82490A07B002842D010F0800F06D1BF
:1084900010F0400F10D02288618A8A420CD100204F
:1084A000A073286940F00200286100F0E1FD28690E
:1084B00020F0020028612BE010F0200F12D00020E5
:1084C000FFF757FF394940F21A400860286940F029
:1084D000020028614FF47A70F7F735FFA07B20F097
:1084E0002001A173A07B10F0100F06D00020F9F737
:1084F000A5F9A07B20F01001A173A07B10F0010F63
:1085000006D00020F9F79AF9A07B20F00101A173B1
:108510002088411C218039184A78A2708978E1703E
:10852000385C1AF8001061605BF82010204688471C
:10853000606800F03FF8606801F045FB607BF0B1D7
:10854000E07A10F0040F1AD12088217B030A184822
:108550004A1E006822734354217B22784B1E2373EA
:108560004254E17A01F0EF02217B4B1E2373425407
:10857000E07A40F00400E072B8F800002080606803
:10858000C0EBC00000EB4000716AB1EBC00FFBD341
:1085900076E70000F9870008680400202405012020
:1085A000000000105CAD0008640000200000002006
:1085B0006000002070B4E849E84C01F1300C8A6892
:1085C000131A0A4616D50D682B440D7E95B18D7C85
:1085D00005F040050D760D7D45F040050D75567D85
:1085E000354205D19CF814509CF81560354000D0F8
:1085F000012565738B60DA498B68181A15D50B68ED
:1086000018440B7E8BB18B7C03F040030B760B7D03
:1086100043F040030B75157D527D154203D19CF844
:1086200015201A4000D001226273886070BC704728
:1086300001F00F010F2928BF7047DFE801F0080F94
:1086400016181A20373C4147175D5F617400417C62
:1086500062EA0101CAB2C16A10460847017C62EAB7
:108660000101CAB2816A1046084742747047027419
:108670007047018801F47F41114301607047017820
:1086800041EA02210160816001210176017D21F032
:1086900040010175B048017D407D014204D1B048E0
:1086A000017D407D08403BD0012039E0018801F484
:1086B0007F41114302E0017841EA022101607047E5
:1086C000818801F47F41114341607047017941EA9B
:1086D00002214160C16001214176017D21F020012C
:1086E00001759D48017D407D0142DDD19C48017DA1
:1086F000407D0840D8D113E082747047C27470473F
:10870000D143027D01F07F01114001759248017D46
:10871000407D0142C8D19248017D407D0840C3D1CF
:108720008E4948737047417D12F0800F1ABF02F0E6
:108730007F02114391434175704701F00F011029E9
:108740003BD2DFE801F008380A0C0E14181A1C237B
:108750003A27292B3638406A0047407C7047007C16
:108760007047017D21F040010175007A7047008952
:10877000C0F307207047007A06E0008907E0017D1A
:1087800021F020010175007BC0B270478089C0F3E1
:1087900007207047807C7047C07C7047017D407D1A
:1087A000084010F07F0018BF802001F07F010843CF
:1087B0007047407D7047006A004700207047664858
:1087C000017D21F002010175407D014204D1644820
:1087D000017D407D084000D0012060494873FE20A3
:1087E000704760480068C0B2704770474FF6E57147
:1087F00008435D49086070472DE9F05FDFF860913C
:1088000006465B4C99F8170006F0030200F00301DE
:10881000481C00F00303554F6078564D4FF0080A8E
:108820004FF0040B4FF001089A4213D153283CBF7C
:10883000401C6070C0B208EB5000207040B201F0E4
:108840002EF9A5F81AA0A5F818B0388840F0010054
:10885000388017E0491E01F003018A4212D1002836
:108860001CBF401E6070C0B208EB5000207040B2C8
:1088700001F015F9A5F81AB0A5F818A0388840F04D
:1088800001003880A17806F00400A07029B100280A
:1088900004BF4FF0FF3001F0A8F816F0080F14BF26
:1088A000A5F81A80A5F8188016F0040F4FF0020002
:1088B00014BF6883288389F81760BDE8F09F2848B3
:1088C000807E704726482C49837F0A6803B152B1E5
:1088D000521C02F010030A6083773F2A03D3102250
:1088E000827700220A60C17EC27D01F0800102F021
:1088F0006F02807F1143084370471949087770471A
:108900001E49086810F0800F04D0134A137D43F00D
:108910000203137510F4407F05D04FF0E022136975
:1089200043F002031361086070471449086810F4AB
:10893000805F04D0094A937B43F02003937310F4C3
:108940000C4F05D04FF0E020026942F002020261B4
:1089500008680860704700004805012024050120D0
:1089600078050120100C0240140C0240000C00405D
:10897000840800200000024064040020143C0140F0
:108980002DE9F041074620222721F54801F0BEF9E4
:10899000F34E0D20F34D86F82700002086F82800BE
:1089A00015F80780781C84B243463A46EEA106F1DA
:1089B0002A0001F0BDFAF04806F12A0710F8281045
:1089C00000EB88003174417871748178B174C0789B
:1089D00036287DD009DCA0F13000062880F0DB804D
:1089E000DFE800F0142B3C4C5C62392800F0AC80CE
:1089F00005DC37286DD038286CD000F0CCB8522870
:108A000000F0B880592865D000F0C5B8601C80B26D
:108A1000295D2A5C401C41EA022584B22B0AEAB295
:108A2000D6A107F1080001F083FA2A46D6A106F183
:108A3000180001F07DFA00F0AEB82D5D601C84B224
:108A40002A46D4A107F1080001F072FA2A46D3A100
:108A500006F1180001F06CFA00F09DB82D5D601C65
:108A600084B22A46CBA107F1080001F061FA2A4638
:108A7000CDA106F1180001F05BFA8CE02D5D601CC1
:108A800084B22A46C3A107F1080001F051FA2A4630
:108A9000C7A106F1180001F04BFA7CE0C6A106F16F
:108AA000180001F045FA76E0601C80B2295D2A5C6E
:108AB000401C41EA022584B22B0AEAB2AFA107F1B9
:108AC000080001F035FA2A46BCA106F1180002E0C0
:108AD00004E013E022E001F02BFA5CE02D5D601C65
:108AE00084B22A46ABA107F1080001F021FA2A4618
:108AF000B4A106F1180001F01BFA4CE02D5D601CDA
:108B000084B22A46A3A107F1080001F011FA2A460F
:108B1000AFA106F1180001F00BFA3CE0601C80B236
:108B2000295D2A5C401C41EA022584B22B0AEAB284
:108B300092A107F1080001F0FBF92A46A7A106F16E
:108B4000180001F0F5F926E0601C80B2295D2A5C6E
:108B5000401C41EA022584B22B0AEAB287A107F140
:108B6000080001F0E5F92A469FA106F1180001F07E
:108B7000DFF910E02D5D601C84B22A4685A107F163
:108B8000080001F0D5F944FA85F082B28BA106F114
:108B9000180001F0CDF90020395C19B13154401CA6
:108BA0001028F9D36E4993A001F0B2F92046BDE830
:108BB000F08110B46A4B904C4FF0000C0268995C45
:108BC00019B1521C02602029F8D0A1F130022170A5
:108BD000092A98BF42EA0C1107D9A1F14102052ADE
:108BE0009CBF373941EA0C1102D81FFA81FCE5E736
:108BF00010BC604670472DE9F04389B04FF0000883
:108C00000D4606467D4C564FCDF8208014E0082EC8
:108C10003CD0A6F120005A289CBF0898262806D2EE
:108C20003E54401C0890314675A001F071F9F8F7E8
:108C300049F810F0FF06FAD00D2E18BF1B2EE6D112
:108C4000089807F800806FA001F062F91B2E18BF8A
:108C5000CDF8208000F081810899785C18B1491C1A
:108C600008912028F8D0644E4D28307076D018DC5A
:108C7000654E412800F09081422800F0C8814428C8
:108C80006DD0472800F0548100F0BDB90898002845
:108C9000CDD031465AA001F03BF90898401E08900B
:108CA000C5E7522807D0532800F05B81582800F010
:108CB000698100F0A8B9785C60B1491C089120284E
:108CC000F9D03070532822D006DC412810D050282B
:108CD00007D020E030701EE058280ED0592811D05F
:108CE00019E008A8FFF765FF002818BF208012E0F0
:108CF00008A8FFF75EFF20720DE008A8FFF759FFF4
:108D0000607208E008A8FFF754FFA07203E008A80B
:108D1000FFF74FFF2073394804ADC17AC1F3800CCF
:108D2000CC09C1F38013C1F34002A5E81C10027BFB
:108D3000837A90F809C001F001010391CDF800C0D9
:108D4000CDE90132037A02883049054801F0F0F894
:108D500003492F4801F0DCF800F055B97BE059E0F9
:108D6000A80501200000001025303458202530329D
:108D70005820202020202000700400202530325868
:108D80002025303258000000282425303458290D81
:108D90000000000025303258000000002824253053
:108DA00032582C58290D000024253032580D00006F
:108DB00023253032580D0000410D000024253034A9
:108DC000580D0000282425303258292C590D000058
:108DD00024253032582C580D000000002425303452
:108DE000582C590D0000000024253034582C580D03
:108DF0000000000025730A006C04002024050120F7
:108E0000256300000D0A00007208002060AE000813
:108E10005CAE000808A8FFF7CCFE002818BF288029
:108E200008A8FFF7C6FE040007D028880021FFF736
:108E3000A7FD2880A042F8D907E028880021FFF785
:108E40009FFD641C2880102CF7D3AFF2480001F07E
:108E50005FF800F0D8B808A8FFF7ABFE00281CBFE9
:108E600020F00F00708008A8FFF7A3FE002814BFB1
:108E700040F00F0700262DD0B04CB148218801F0FA
:108E800047F800252088284480B201F00DF80146FB
:108E9000AC4801F03DF86D1C102DF3D3002520885F
:108EA000284480B201F000F8A0F12001602928BF19
:108EB0002E200146A44801F02BF86D1C102DEED396
:108EC000208810302080A14801F022F87088B84234
:108ED000D2D9BAE7994C9A48218801F019F80025AF
:108EE0002088284480B200F0DFFF0146954801F059
:108EF0000FF86D1C102DF3D300252088284480B274
:108F000000F0D2FFA0F12001602928BF2E200146E9
:108F10008D4800F0FDFF6D1C102DEED32088103021
:108F200020808A4800F0F4FF761C102ED2D38CE704
:108F300008A8FFF73EFE38B1A0F57F412080FF3939
:108F400004BF0020FFF715FA08A8FFF732FE20B192
:108F50006082A07B40F04000A07309B00120BDE812
:108F6000F08308A8FFF725FE044608A8FFF721FEB6
:108F7000C1B22046621C94B200F0AEFF30780028E7
:108F8000F3D140E0E07B90F00100E07314BF70A0EB
:108F900071A000F0BDFF36E071A000F0B9FFDFF86E
:108FA000D4913078002519F80000002884BF724F52
:108FB0004FF00F0827D92A46317870A000F0A8FF9B
:108FC0005FF0000414F00F0F03D121466EA000F0F3
:108FD0009FFF04EB0520395CAFF25C2000F098FFA6
:108FE00038EA040004BF5BA000F092FF641CB4F5F3
:108FF000807FE7D357A000F08BFF30786D1C19F805
:1090000000008542D7D309B00020BDE8F08361A0FD
:1090100000F07EFFDFF8908130780024254638F894
:10902000100000287FF611AF6048074690F80090C6
:1090300029465FA000F06CFF4946AFF2BC2000F06B
:1090400067FF641C102C08D2B9F1FF0F09D104E0AE
:1090500017F80590002CEFD1EAE700243DA000F0BE
:1090600057FF30786D1C38F81000A842F0D8ECE6B5
:1090700030B5524C89B00DF1100E2088ADF82000AB
:10908000012020742046C17AC1F3800CCD09C1F3C0
:109090008013C1F34002AEE82C10027B837A90F873
:1090A00009C001F001010391CDF800C0CDE9013202
:1090B000037A02884249434800F03AFF4149424856
:1090C00000F026FF0021BDF82000FFF759FCADF8A5
:1090D00020000025F7F7F6FD10F0FF00FAD010F0A1
:1090E000800FF7D11B2808D0452814D054280DD064
:1090F00008A9FFF780FD0028ECD0207C00281CBFC9
:1091000032A000F005FF257409B030BDA07B40F00F
:109110008000A073F1E7208800F0C6FE2028A07B25
:109120001CBF40F08000A07301D02574EBE740F035
:109130004000A0732088C01C6082F6E76E04002007
:109140009CAE0008A4AE0008ACAE0008B0AE0008AB
:1091500054524F4E0D0A000054524F46460D0A001D
:10916000747261636B4275666665725F4436340D76
:109170000A00000064AF0008EC250120543A256481
:1091800020533A25640D0A002020253032583E2015
:1091900000000000747261636B4275666665725F01
:1091A0004743520D0A00000090AF0008EC05012073
:1091B0002020253034583E200000000024050120E6
:1091C00060AE0008A80501205CAE000852554E0DA7
:1091D0000A000000F0B40023FB4E1A461C4600BFF4
:1091E00001EB540C14F0010F9CF800C008BF4FEACB
:1091F0001C1C0CF00F0C521C16F80CC0D2B2CCF395
:10920000001545EA43034FEA4C6CDBB24FEA1C6C95
:10921000082A03D300F8013B00231A465FF0020539
:10922000CCF30017521C47EA43034FEA4C6CD2B20E
:10923000DBB24FEA1C6C082A03D300F8013B002381
:109240001A46CCF30017521C47EA43034FEA4C6C12
:10925000D2B2DBB24FEA1C6C082A03D300F8013B00
:1092600000231A466D1EDBD1641C082CB8D3F0BC59
:1092700070472DE9F74F86B04FF0000B07995D4618
:10928000DA46002984BFC0B2049040F21981092453
:109290001AF0010F0BD00798112808BF0A2406D036
:1092A000122808BF0D2402D0132808BF1324C74872
:1092B00010F80A60032E08BF082012D0C44AFF210C
:1092C000681C51551154A81C1154E81C1154281D38
:1092D0006D1D115408208DF80800022E08BF0020D3
:1092E00001D18DF8080041218DF80C100AF0FF0023
:1092F0008DF80D108DF80A00049A0F218DF80E10CC
:1093000050408DF80B208DF80F10092E08BFC04378
:109310008DF8090002A96846FFF75CFFDFF8B0820C
:109320009DF8000008F80500681C9DF8011008F879
:109330000010A81C9DF8021008F80010E81C9DF809
:10934000031008F80010281D9DF8041008F80010FC
:109350006D1D03A96846FFF73DFF9DF8000008F862
:109360000500681C9DF8011008F80010A81C9DF865
:10937000021008F80010E81C9DF8031008F800100F
:10938000281D9DF8041008F800106D1D08EB05005D
:109390005522092100F0BAFC0935032E0BD04246B4
:1093A000FF21681C51551154A81C1154E81C11547C
:1093B000281D6D1D115407218DF808104FF001086C
:1093C000042E04BF00218DF808100027B9468148FB
:1093D00002A910F80B0001F8080008F10108474045
:1093E0000BF1010BB8F1040F19D34FF000086846D8
:1093F000FFF7F0FE76489DF800104155691C9DF876
:1094000001204254A91C9DF802204254E91C9DF8F9
:1094100003204254291D9DF8042042546D1D09F17A
:109420000109B9F5807FD2D3052E08BFFF438DF81F
:10943000097000278DF80A708DF80B7002A9684634
:10944000FFF7C8FE102E08BF8DF800709DF80010C1
:109450005F484155691C9DF801204254A91C9DF8A4
:1094600002204254E91C9DF803204254291D9DF816
:1094700004206D1D4254B4F1004F28BF552104D380
:1094800041556D1C641EFBD114E0012CD8BF012492
:109490002844401E14F0010F02D0552100F8011F8E
:1094A000611018BF552204D0427000F8022F491EE7
:1094B000FAD1254407980AF1010A8245FFF4E7AE84
:1094C0000898854239BF4248552109B0BDE8F08F60
:1094D0004155089A6D1C9542FAD309B0BDE8F08F4A
:1094E0002DE9F74FADF5267D00200146A290401EE4
:1094F000979003209690A898031F3548425CFF2A56
:109500000FD1421892F801C0BCF1FF0F04BF92F8CE
:1095100002C0BCF1520F04D1D27802F0C002402A3E
:109520002BD0491C9942E9D9DFF8A0C0A79991B185
:10953000A79AACF1010112F0010F02D0969A01F83E
:10954000012FA79A520806D0969B4B70969B01F864
:10955000023F521EF8D19799002912DBA89981B1D8
:109560009799939100219F9194910A4699919A918C
:1095700093990025184E415C15E097910221969130
:10958000D2E70DF5297D0020BDE8F08F10489399B2
:10959000415C42B1012A2BD0022A7DD0032A40F03F
:1095A000A88100F0EDB8FF2918D09F9802281BD39E
:1095B0000120024696900A2094900020999093985A
:1095C00000286AD10EE0000014B00008EC3A012037
:1095D000EC050120EC25012024B000089F98401CD8
:1095E000C0B202E0A898C8E000209F9000F081B9C6
:1095F000949B999883427DD84FF0000BDA46002B5C
:1096000088BF0DF5827E78D901270DEB0B040EEB98
:109610000A00002103E000BFBCF1000F03D110F8E5
:10962000013B4FF0080CACF1010245EAD31C4FEAB4
:10963000436312F0FF024FEA136302D110F8013BBB
:1096400008224FEA4C0C4CEAD31C521E4FEA4363EB
:1096500012F0FF024FEA136302D110F8013B082217
:109660004FEA4C0C4CEAD31C521E4FEA436312F0F3
:10967000FF024FEA136302D110F8013B08224FEAC0
:109680004C0C4CEAD318521E4FEA436312F0FF020F
:109690004FEA136305D101E05EE06EE010F8013B94
:1096A0000822521E02F0FF0C4FEA480242EAD3128F
:1096B0005B06B25C1B0E802A24BF0022174611F005
:1096C000010F08BF120104EB51081CBF98F800906D
:1096D00049EA020288F80020491C08299CD3002F7F
:1096E00004BF102096900BF1040B94980AF1050A20
:1096F000824501E048E000E086D39DF801009DF836
:1097000002209DF8031050409DF80430484083EA41
:10971000000C9DF80500969C80EA0C0C012C13D1DE
:109720009DF80040082C18BF022001D096900BE055
:10973000BCF1000F18BF0920F8D1DDF898C26145CF
:1097400002D1A7998A4201D30022D2E0FF499A921E
:109750000222CB718871CCE0FF293FF43FAF9F9884
:109760000228FFF441AF40F24510949000209990F8
:109770009398032200283FF435AF401E939033E7BF
:10978000949B9998834206D9999B41A8C154999872
:10979000401C9990ADE04FF0000BDA46002B88BFDB
:1097A0000DF5827E73D900BF01270DEB0B040EEB84
:1097B0000A00002103E000BFBCF1000F03D110F844
:1097C000013B4FF0080CACF1010245EAD31C4FEA13
:1097D000436312F0FF024FEA136302D110F8013B1A
:1097E00008224FEA4C0C4CEAD31C521E4FEA43634A
:1097F00012F0FF024FEA136302D110F8013B082276
:109800004FEA4C0C4CEAD31C521E4FEA436312F051
:10981000FF024FEA136302D110F8013B08224FEA1E
:109820004C0C4CEAD318521E4FEA436312F0FF026D
:109830004FEA136302D110F8013B0822521E02F0D6
:10984000FF0C4FEA480242EAD3125B06B25C1B0EE1
:10985000802A24BF0022174611F0010F08BF120111
:1098600004EB51081CBF98F8009049EA020288F8FE
:109870000020491C08299FD3002F04BF1020969078
:109880000BF1040B94980AF1050A82458CD39DF8DC
:1098900001000DF1010180224B78584011F8023F80
:1098A0005840521EF8D19699012902D005290BD0B3
:1098B00018E09DF8001007291CBF0420969011D1D4
:1098C00000281CBF052096909A984FF480720102E0
:1098D0009F4808440DF1010100F006FAA298401CCF
:1098E000C0B2A2909B499A9A96988854002002464A
:1098F0009A909398A899401C9390884224BF002086
:109900009390979988427FF441AEA2980DF5297DF6
:10991000BDE8F08F2DE9F8438F4D04460126D5F8B8
:109920005802002808BFBDE8F883884B002CBCBF54
:10993000987844B2894F002137F8142072B18848D2
:1099400012F0010F18BF00F8011F37F81420520859
:1099500004D0417000F8021F521EFAD18148012C38
:10996000C0F80011C0F80411C0F80811C0F80C11BB
:10997000C0F81011C0F81411A4BFD878A04231DB90
:109980007949DFF8E891002611F80480197A91B13D
:1099900009EB800059F82410406800EB112105F50F
:1099A0001670F9F7F6FF30B96B464246694905F57E
:1099B0001670F9F772FD59F8241005F51670F9F7CD
:1099C000E8FF78B94FEA08226B46614905F5167041
:1099D000F9F763FD30B937F8142041462046FFF708
:1099E00048FC01263046BDE8F8832DE9F8435A4D7E
:1099F00004460127D5F85802002808BFBDE8F883BF
:109A0000524E002CBCBFB07844B27078002841D0D0
:109A1000307900283ED1012CA4BFF078A04239DB78
:109A2000514810F804802C30414630F81420E0B240
:109A3000FFF756FDDFF8349180B1002759F8241064
:109A400005F51670F9F7A5FF40B94FEA08226B46F5
:109A50003F4905F51670F9F7E2FD0127307AA8B104
:109A6000F07859F8241009EB80000027406800EBDB
:109A7000112105F51670F9F78CFF38B96B4642468F
:109A8000344905F51670F9F7CAFD012705F516707A
:109A9000F9F7B1FE002070703846BDE8F88370B564
:109AA00001250128B8BF012002DB2A28C8BF2A20CF
:109AB0000446264EB17888420CD048B2FFF795FF95
:109AC000002808BF0025B47060B2FFF723FF00280C
:109AD00008BF0025284670BD2DE9F001264824491D
:109AE00000238478A0F11400CE7CDFF8888002691E
:109AF00016F0200F4FF001071D4617D09C4644B1C9
:109B000018F802C0BCF1FF0F04BF437A4FF0010800
:109B100001D04FF0000880F8098081F81AC0077062
:109B2000002B18BF4FF0000C31D12EE04FF0FF0C8E
:109B300081F81AC03CB390F804C0BCF1000F04BF18
:109B400090F800C0BCF1000F1DD117E07008002094
:109B5000EC250120EC3A0120B009002090AF00086C
:109B6000EB050120EC39012064AF0008B4AE000819
:109B700078050120EC05012084080020477091F849
:109B80001CC008F802C0057045724FF0800C81F8C7
:109B90001BC016F0020F05D023B94A49CB7A43F017
:109BA0004003CB72002C04BFBDE8F0017047511C8C
:109BB00001618378444A32F813208A4298BF0561D4
:109BC000BDE8F00170474149CA68101AC86058BF23
:109BD00070473F4A8B78D25C00EB4200C8607BE75D
:109BE0002DE9F0413B4D0746D5F8580238B14FF00A
:109BF000FF30FFF7FAFE05F51670F9F74CFE334C0F
:109C000000260322E67026712672394605F5167085
:109C1000F9F790FB00281CBF0020BDE8F081D5F8C3
:109C20006402010AB0EB012F07D040F20111B0FB32
:109C3000F1F101EB012282420DD1A1F2AB27782F85
:109C400009D2254880FB0710C110A1EBE07808EB92
:109C50000810B84206D005F51670F9F71CFE002072
:109C6000BDE8F081002105F51670F9F792FE267126
:109C700008F12300E070380200F50030D5F86412D6
:109C800000F52B40884234BF01200020207260790B
:109C90004121401CC0B26071A37901EB10129A42BD
:109CA00007D100F00F02E37941329A4204BF401C11
:109CB0006071A171E171A07840B2FFF72BFE012025
:109CC000BDE8F0812405012090AF00087008002055
:109CD000E8AF0008B009002079787878A0F1610138
:109CE000192900D82038704740EA01039B0703D0A8
:109CF00009E008C9121F08C0042AFAD203E011F8CB
:109D0000013B00F8013B521EF9D27047D2B201E08C
:109D100000F8012B491EFBD270470022F6E710B570
:109D200013460A4604461946FFF7F0FF204610BDC9
:109D3000421E12F8013F002BFBD111F8013B02F843
:109D4000013B002BF9D17047421C10F8011B002980
:109D5000FBD1801A704710B5002200E0521C835CD2
:109D60008C5CA34201D1002BF8D1D8B2E1B2401AE9
:109D700010BD034611F8012B00F8012B002AF9D180
:109D8000184670472DE9F05F0546002092469B4635
:109D900088460646814640241BE028464146474601
:109DA000224600F042F853465A46C01A914110D359
:109DB00011461846224600F029F82D1A67EB0108D3
:109DC0004F4622460120002100F020F817EB000941
:109DD0004E41201EA4F10104DFDC484631462A46EC
:109DE0004346BDE8F09F0000064C074D06E0E068E2
:109DF00040F0010394E8070098471034AC42F6D3D2
:109E0000F6F7C6F944F0000864F00008202A04DBE5
:109E1000203A00FA02F1002070479140C2F120037D
:109E200020FA03F3194390407047202A04DB203ABC
:109E300021FA02F00021704721FA02F3D040C2F16A
:109E40002002914008431946704770B501EB0204A7
:109E500010F8015B15F0070301D110F8013B2A113E
:109E600006D110F8012B03E010F8016B01F8016B2B
:109E70005B1EF9D12B0705D40023521E0FD401F825
:109E8000013BFAE710F8013B02F10202A1EB0303E8
:109E900003E013F8015B01F8015B521EF9D5A14202
:109EA000D6D3002070BD000000F47841B1F5C05F4A
:109EB0001EBF0649085C7047B0F5E05F2CBF044A3E
:109EC000044A01461046FEF738BC000000000010AE
:109ED0007805012048050120B0F5006F2DBF00F482
:109EE0007842084A1154B2F5C05F18BF7047B0F508
:109EF000E05F2CBF044B054B0A4601461846FEF7AF
:109F000097BB0000000000107805012048050120E3
:109F10000FB4054B10B503A9044A029800F02CF8C1
:109F200010BC5DF814FB0000294B00088C080020D1
:109F30000FB4084B10B504A902AA039800F01CF84E
:109F4000044602A9002000F046FA204610BC5DF845
:109F500014FB0000D7A3000802E008C8121F08C1C4
:109F6000002AFAD170477047002001E001C1121F9A
:109F7000002AFBD1704700002DE9FF4F8DB00F463E
:109F800005460026DEE1252874D100246D1CF14928
:109F9000A246A14601222B78203B02FA03F0084298
:109FA00002D004436D1CF6E728782A2810D06FF001
:109FB0002F022878A0F13001092915D80AEB8A016F
:109FC00002EB410144F0020400EB010A6D1CF0E7D2
:109FD00057F804ABBAF1000F03DA44F40054CAF1A5
:109FE000000A44F002046D1C28782E2817D115F8B9
:109FF000010F44F004042A280ED06FF02F022878B5
:10A00000A0F1300109290AD809EB890102EB4101CD
:10A0100000EB01096D1CF2E757F8049B6D1C2878D2
:10A020006C280FD006DC4C2817D068280DD06A2881
:10A0300014D104E0742810D07A280FD10DE044F434
:10A0400000140AE044F4801401E044F440146978F8
:10A05000814202D16D1C04F580146D1C2A786E2A91
:10A0600020D00DDC632A33D005DC002A6FD0582ABB
:10A0700012D1A2E011E0642A6AD0692A0CD167E00B
:10A08000732A2FD004DC6F2A6FD0702A04D199E094
:10A09000752A6BD0782A6AD01046DDE90F129047F6
:10A0A000761C4EE1C4F30250022806D003280AD0E1
:10A0B000042801CF0AD0066043E101CF4FEAE671E0
:10A0C000C0E900613DE101CF06803AE1067038E168
:10A0D00017F8040B8DF8000000208DF80100EB4606
:10A0E000012003E057F804BB4FF0FF3061074FF049
:10A0F000000102D40DE008F10101884649450FDA5C
:10A100008045F8DB1BF808100029F4D108E008F1BD
:10A11000010188468142FADB1BF808100029F6D1BC
:10A12000DDE90F23AAEB08008146214600F03BF948
:10A13000304400EB080604E0DDE90F121BF8010BC8
:10A140009047B8F10108F7D221464846F4E0FDE017
:10A150000A21C4F302534FF0000B0891022B07D0E1
:10A1600001CFC117032B09D00AE034E023E024E03B
:10A17000FF1D27F00707F7E8020105E000B2C1174D
:10A18000042B01D140B2C117002907DA4FF0000CAF
:10A19000D0EB0C006CEB01012D2302E0230504D56C
:10A1A0002B238DF82430012303E0E30701D0202383
:10A1B000F7E7984650E00A210EE010204FF0000B20
:10A1C00008900CE010214FF0000B44F004044FF015
:10A1D0000809089103E008214FF0000B0891C4F32F
:10A1E0000253022B04D001CF0021032B06D006E03E
:10A1F000FF1D27F00707F7E8020103E080B2042BF8
:10A2000000D1C0B24FF00008230725D5702A2AD00C
:10A21000DDF820C08CF0100C5CEA0B0C09D150EA80
:10A22000010306D030238DF824308DF82520022339
:10A230009846DDF820C08CF0080C5CEA0B0C0BD1C2
:10A2400050EA010301D1630706D530238DF824308D
:10A250004FF00108A9F10109582A09D03EA20B923A
:10A2600008AA0A9211E040238DF824300123DFE789
:10A270003EA2F4E75B46089AFFF784FD0B9B9B5CCC
:10A280000A9AA2F101020A92137050EA0102F1D176
:10A290000A98ADEB000000F1200B600702D524F412
:10A2A000803401E04FF00109D94502DDA9EB0B0034
:10A2B00000E0002000EB0B0141440890AAEB010AEA
:10A2C000E00306D4DDE90F232146504600F06BF889
:10A2D0000644002008E009A911F80900DDE90F1281
:10A2E0009047761C09F1010081464045F3DBE0030D
:10A2F0000CD5DDE90F232146504600F054F8064402
:10A3000004E0DDE90F1230209047761C0899481EC2
:10A3100008900029F5DC08E00A980A990078491CA1
:10A320000A91DDE90F129047761CBBF10001ABF1F9
:10A33000010BF1DC21465046DDE90F2300F020F847
:10A3400006446D1C287800287FF41DAE11B03046FD
:10A35000BDE8F08F0928010030313233343536370B
:10A360003839616263646566000000003031323361
:10A370003435363738394142434445460000000001
:10A380002DE9F041044600251E461746880405D4F1
:10A3900006E039462020B04705F10105641EF8D5D6
:10A3A0002846BDE8F0812DE9F041044600251E460F
:10A3B0009046C80301D5302700E02027880405D542
:10A3C00006E041463846B04705F10105641EF8D560
:10A3D0002846BDE8F0810A68531C0B601070704776
:10A3E000000C02400001000001000000000C0240CF
:10A3F0000002000001000000000C02400004000008
:10A4000001000000000C02400008000001000000F4
:10A41000000C02400080000001000000000002402B
:10A4200010000100010000000000024020000200B6
:10A430000100000000000240400002000100000096
:10A440000000024080000200010000000000024005
:10A4500000100000010000000004024000040100A0
:10A46000010000000004024000080100010000009B
:10A47000000402400010010001000000000402403E
:10A480000020020001000000000402400040020021
:10A4900001000000000402400080020001000000F2
:10A4A0000000024001000101010000000000024024
:10A4B000020001010100000000000240040001014F
:10A4C000010000000000024008000101010000003E
:10A4D00000080240400002000100000000080240A5
:10A4E0008000020001000000000C0240010000009A
:10A4F00000000000000C024002000100010000000A
:10A50000000C02400400000000000000000C0240AB
:10A510000800010001000000000C024010000100D2
:10A5200001000000000C02402000000001000000BB
:10A53000000C02404000000001000000000C02403E
:10A54000800000000000000000000000010000008A
:10A5500001000000000000000000005F0000000794
:10A56000000700147F147F14242A7F2A1223130863
:10A57000646236495522500005030000001C224148
:10A58000000041221C0014083E081408083E080878
:10A590000050300000080808080800606000002033
:10A5A000100804023E5149453E00427F400042618E
:10A5B0005149462141454B311814127F102745451A
:10A5C00045393C4A49493001710905033649494931
:10A5D00036064949291E003636000000563600006E
:10A5E0000814224100141414141400412214080207
:10A5F00001510906324979413E7E1111117E7F4990
:10A600004949363E414141227F4141221C7F49490F
:10A6100049417F090909013E4149497A7F080808F3
:10A620007F00417F41002040413F017F08142241CB
:10A630007F404040407F020C027F7F0408107F3E35
:10A640004141413E7F090909063E4151215E7F0992
:10A65000192946464949493101017F01013F4040DE
:10A66000403F1F2040201F3F4038403F63140814E4
:10A670006307087008076151494543007F41410065
:10A6800002040810200041417F000402010204403E
:10A6900040404040000102040020545454787F4858
:10A6A0004444383844444420384444487F3854545F
:10A6B0005418087E0901020C5252523E7F080404CD
:10A6C0007800447D40002040443D007F1028440035
:10A6D00000417F40007C041804787C08040478382A
:10A6E000444444387C14141408081414187C7C085E
:10A6F0000404084854545420043F4440203C404043
:10A70000207C1C2040201C3C4030403C4428102829
:10A71000440C5050503C4464544C440008364100B2
:10A7200000007F000000413608001008081008787B
:10A730004641467800000000000080C0C0E0E0F024
:10A74000F0F0F0F0F0F0F0E0000000000000000099
:10A75000000000000080E0F8FCFFFFFFFFFF3F1F4C
:10A760001F0F0F0F0F0F0F0F1FE0E0E0E0E0E0E022
:10A77000E0E0E0E06020FFFFFFFFFFFFFFE70000F9
:10A7800000000000000000000000EFEFEFEFEFEF2F
:10A79000EFE7C38100000001071F3F7FFFFFFFFFBE
:10A7A000FEFCF8F0F0F0F0F0F0F0F807070707070C
:10A7B0000707070707070604000000000000010361
:10A7C000030707070F0F0F0F0F0F0F070000000001
:10A7D0000000000000000000000000007DB20549FC
:10A7E0004DFEFC306A3463BFA71725ED434F4D4D36
:10A7F0004F444F5245203135343100003C25733EE3
:10A8000000000000257300003E2000002020000111
:10A81000030507090E10121416181C1E809A90B614
:10A820008EDE8F809DD38A8AD78D8E8F909191E214
:10A830009995959797999A9B9B9D9E9FB5D6E0E990
:10A84000A4A4A6A6A8A8AA8DACB8AEAFB0B1B2B366
:10A85000B4B5B6B7B8B9BABBBCBDBDBFC0C1C2C341
:10A86000C4C5C6C6C8C9CACBCCCDCECFD1D1D2D330
:10A87000D2D5D6D7B7D9DADBDCDDDEDFE0E1E2E343
:10A88000E3D5E6E6E8E9E8EBEDEDDDEFF0F1F2F334
:10A89000F4F5F6F7F8F9FAEBFCFCFEFFC700FC0054
:10A8A000E900E200E4006F010701E7004201EB006C
:10A8B00050015101EE007901C4000601C9003901BF
:10A8C0003A01F400F6003D013E015A015B01D60059
:10A8D000DC00640165014101D7000D01E100ED00DC
:10A8E000F300FA00040105017D017E011801190140
:10A8F000AC007A010C015F01AB00BB0091259225F1
:10A90000932502252425C100C2001A015E0163259A
:10A91000512557255D257B017C0110251425342503
:10A920002C251C2500253C25020103015A25542510
:10A9300069256625602550256C25A40011011001AC
:10A940000E01CB000F014701CD00CE001B011825E1
:10A950000C258825842562016E018025D300DF0047
:10A96000D400430144014801600161015401DA004F
:10A9700055017001FD00DD006301B400AD00DD0292
:10A98000DB02C702D802A700F700B800B000A80099
:10A99000D902710158015901A025A000610062008F
:10A9A00063006400650066006700680069006A0073
:10A9B0006B006C006D006E006F0070007100720023
:10A9C00073007400750076007700780079007A00D3
:10A9D000A100A200A300A500AC00AF00E000E100D0
:10A9E000E200E300E400E500E600E700E800E9003B
:10A9F000EA00EB00EC00ED00EE00EF00F000F100EB
:10AA0000F200F300F400F500F600F800F900FA0097
:10AA1000FB00FC00FD00FE00FF0001010301050139
:10AA2000070109010B010D010F01110113011501AE
:10AA3000170119011B011D011F012101230125011E
:10AA4000270129012B012D012F013101330135018E
:10AA500037013A013C013E014001420144014601F7
:10AA600048014B014D014F0151015301550157015F
:10AA700059015B015D015F016101630165016701CE
:10AA800069016B016D016F0171017301750177013E
:10AA90007A017C017E019201B103B203B303B403D6
:10AAA000B503B603B703B803B903BA03BB03BC03CA
:10AAB000BD03BE03BF03C003C103C303C403C50377
:10AAC000C603C703C803C903CA03300431043204F0
:10AAD00033043404350436043704380439043A04A2
:10AAE0003B043C043D043E043F0440044104420452
:10AAF00043044404450446044704480449044A0402
:10AB00004B044C044D044E044F04510452045304AE
:10AB10005404550456045704580459045A045B0459
:10AB20005C045E045F047021712172217321742121
:10AB3000752176217721782179217A217B217C2149
:10AB40007D217E217F2141FF42FF43FF44FF45FFDE
:10AB500046FF47FF48FF49FF4AFF4BFF4CFF4DFFB1
:10AB60004EFF4FFF50FF51FF52FF53FF54FF55FF61
:10AB700056FF57FF58FF59FF5AFF0000410042009F
:10AB800043004400450046004700480049004A0091
:10AB90004B004C004D004E004F0050005100520041
:10ABA00053005400550056005700580059005A00F1
:10ABB0002100E0FFE1FFE5FFE2FFE3FFC000C1008D
:10ABC000C200C300C400C500C600C700C800C90059
:10ABD000CA00CB00CC00CD00CE00CF00D000D10009
:10ABE000D200D300D400D500D600D800D900DA00B6
:10ABF000DB00DC00DD00DE00780100010201040161
:10AC0000060108010A010C010E01100112011401D4
:10AC1000160118011A011C011E0120012201240144
:10AC2000260128012A012C012E01300132013401B4
:10AC3000360139013B013D013F014101430145011D
:10AC400047014A014C014E01500152015401560185
:10AC500058015A015C015E016001620164016601F4
:10AC600068016A016C016E01700172017401760164
:10AC700079017B017D019101910392039303940378
:10AC8000950396039703980399039A039B039C03E8
:10AC90009D039E039F03A003A103A303A403A50395
:10ACA000A603A703A803A903AA031004110412040E
:10ACB00013041404150416041704180419041A04C0
:10ACC0001B041C041D041E041F0420042104220470
:10ACD00023042404250426042704280429042A0420
:10ACE0002B042C042D042E042F040104020403045D
:10ACF0000404050406040704080409040A040B04F8
:10AD00000C040E040F04602161216221632164217F
:10AD1000652166216721682169216A216B216C21E7
:10AD20006D216E216F2121FF22FF23FF24FF25FFCC
:10AD300026FF27FF28FF29FF2AFF2BFF2CFF2DFFCF
:10AD40002EFF2FFF30FF31FF32FF33FF34FF35FF7F
:10AD500036FF37FF38FF39FF3AFF000007060008CB
:10AD600003030505030202020404060602050008A7
:10AD70000404060602040207040407070606000886
:10AD80000303050504020202040406060205000886
:10AD90000404060602040207040407070606000866
:10ADA0000303050503020202030406060205000868
:10ADB0000404060602040207040407070606000846
:10ADC0000403050504020202050406060205000844
:10ADD000040406060204020704040707020602062A
:10ADE0000303030302020202040404040206000631
:10ADF0000404040402050205050505050206020611
:10AE00000303030302020202040404040205000512
:10AE100004040404020402040404040402060208F4
:10AE200003030505020202020404030602050008EA
:10AE300004040606020402070404070702060208C7
:10AE400003030505020202020404060602050008C7
:10AE500004040606020402070404070725730A0017
:10AE600050433A2530345820413A25303258205842
:10AE70003A2530325820593A2530325820533A2555
:10AE800030325820432564205A2564204F25642001
:10AE90004E2564204925640D0000000025303458FB
:10AEA00020000000253032582000000025630000FB
:10AEB0000D0A000000000000000000000015000066
:10AEC000002A0000003F000000540000006900005C
:10AED000007E00000093000000A8000000BD0000FC
:10AEE00000D2000000E7000000FC0000001101009B
:10AEF00000260100003B0100005001000065010038
:10AF000000780100008B0100009E010000B10100EB
:10AF100000C4010000D7010000EA010000FC0100AC
:10AF2000000E020000200200003202000044020075
:10AF3000005602000067020000780200008902004B
:10AF4000009A020000AB020000BC020000CD02002B
:10AF500000DE020000EF0200000003000011030009
:10AF600000220300001515151515151515151515D5
:10AF70001515151515151313131313131312121298
:10AF800012121211111111111111111111111111AE
:10AF90000C1E0C1E0C1E0C1E0C1E0C1E0C1E0C1E61
:10AFA0000C1E0C1E0C1E0C1E0C1E0C1E0C1E0C1E51
:10AFB0000C1E0C1EE71BE71BE71BE71BE71BE71B31
:10AFC000E71B0B1A0B1A0B1A0B1A0B1A0B1A6A181F
:10AFD0006A186A186A186A186A186A186A186A1861
:10AFE0006A186A186A186A180D0D0D0D0D0D0D0DF1
:10AFF0000D0D0D0D0D0D0D0D0D0D0E0E0E0E0E0E7B
:10B000000E0F0F0F0F0F0F10101010101010101048
:10B01000101010100A0B12130E0F161709191A1B15
:10B020000D1D1E15FFFFFFFFFFFFFFFFFF080001C3
:10B03000FF0C0405FFFF0203FF0F0607FF090A0BC1
:10B04000FF0D0EFF97AAAAAAAAAAAAAAAAAAAAAA02
:10B05000AAAAAAAAAAAAAAAAAAAAAAAAAAAAAAAA50
:10B06000AAAAAAAAAAAAAAAAAAAAAAAAAAAAAAAA40
:10B07000AAAAAAAAAAAAAAAAAAAAAAAAAAAAAAAA30
:10B08000AAAAAAAAAAAAAAAAAAAAAAAAAAAAAAAA20
:10B09000AAAAAAAAAAAAAAAAAAAAAAAAAAAAAAAA10
:10B0A000AAAAAAAAAAAAAAAAAAAAAAAAAAAAAAAA00
:10B0B000AAAAAAAAAAAAAAAAAAAAAAAAAAAAAAAAF0
:10B0C000AAAAAAAAAAAAAAAAAAAAAAAAAAAAAAAAE0
:10B0D000AAAAAAAAAAAAAAAAAAAAAAAAAAAAAAAAD0
:10B0E000AAAAAAAAAAAAAAAAAAAAAAAAAAAAAAAAC0
:10B0F000AAAAAAAAAAAAAAAAAAAAAAAAAAAAAAAAB0
:10B10000AAAAAAAAAAAAAAAAAAAAAAAAAAAAAAAA9F
:10B11000AAAAAAAAAAAAAAAAAAAAAAAAAAAAAAAA8F
:10B12000AAAAAAAAAAAAAAAAAAAAAAAAAAAAAAAA7F
:10B13000AAAAAAAAAAAAAAAAAAAAAAAAAAAAAAAA6F
:10B14000AAAAAAAA78A9F72D001C48A57FF005682D
:10B150000900D0036809088D001C586078A9080D03
:10B16000001C8D001C5860A9008D6C028D6D026062
:10B17000788A48A9508D6C02A200BDCAFE8D6D026E
:10B180000D001C8D001C68AA5860A9008DF902AD45
:10B190008E02857F20BCE6A5841009290FC90FF017
:10B1A000034CB4D720B3C2B1A38D7502A20BBD89E5
:10B1B000FECD7502F008CA10F5A9314CC8C18E2A1F
:10B1C00002E009900320EEC1AE2A02BD95FE856F14
:10B1D000BDA1FE85706C6F00A9008DF902AD6C02F7
:10B1E000D02AA000988480848184A320C7E62023ED
:10B1F000C1A57F8D8E02AAA90095FF20BDC14CDAA2
:10B20000D4A028A9009900028810FA60A0008480C8
:10B2100084814C45E6A2008E7A02A93A2068C2F0E9
:10B220000588888C7A024C68C3A000A200A93A4C19
:10B2300068C220E5C1D005A9344CC8C188888C7A81
:10B24000028AD0F3A93D2068C28AF002A9400921F0
:10B250008D8B02E88E77028E7802AD8A02F00DA9FE
:10B26000800D8B028D8B02A9008D8A0298F0299D9A
:10B270007A02AD77028D7902A98D2068C2E88E78B6
:10B2800002CAAD8A02F002A908EC7702F0020904B2
:10B2900009034D8B028D8B02AD8B02AE2A023DA5B8
:10B2A000FED001608D6C02A9304CC8C18D7502CCF6
:10B2B0007402B02EB1A3C8CD7502F028C92AF004DB
:10B2C000C93FD003EE8A02C92CD0E4989D7B02AD21
:10B2D0008A02297FF007A98095E78D8A02E8E004B9
:10B2E00090CDA000AD74029D7B02AD8A02297FF053
:10B2F00004A98095E79860A4A3F01488F010B90021
:10B3000002C90DF00A88B90002C90DF002C8C88C44
:10B310007402C02AA0FF90088C2A02A9324CC8C12E
:10B32000A0009885A38D58028D4A028D960285D380
:10B330008D79028D77028D78028D8A028D6C02A242
:10B34000059D790295D795DC95E195E69D7F029D57
:10B350008402CAD0EC60AD78028D7702A9018D78A5
:10B36000028D7902AC8E02A20086D3BD7A02203C07
:10B37000C3A6D39D7A029895E2E8EC780290EA6041
:10B38000AAA000A93ADD0102F00CDD0002D016E807
:10B39000982901A88A60BD0002E8E8C930F0F2C926
:10B3A00031F0EED0EB9809802981D0E7A9008D8B90
:10B3B00002AC7A02B1A320BDC31011C8CC7402B094
:10B3C00006AC740288D0EDCE8B02A9002901857FDE
:10B3D0004C00C1A57F49012901857F60A000AD77A0
:10B3E00002CD7802F016CE7802AC7802B97A02A8C3
:10B3F000B1A3A004D9BBFEF00388D0F8988D9602C3
:10B4000060C930F006C931F0020980298160A900C5
:10B41000856F8D8D0248AE780268056F48A9018559
:10B420006FCA300FB5E21004066F066F4A90EA0645
:10B430006FD0E668AABD3FC44829038D8C02680A14
:10B44000103EA5E22901857FAD8C02F02B203DC680
:10B45000F012208FC3A9008D8C02203DC6F01EA9DA
:10B460007420C8C1208FC3203DC608208FC328F098
:10B470000CA9008D8C02F005203DC6D0E24C00C125
:10B480002A4C00C400804101010101818181814277
:10B4900042424220CAC3A9008D920220ACC5D019F5
:10B4A000CE8C02100160A9018D8D02208FC3200077
:10B4B000C14C52C42017C6F01020D8C4AD8F02F082
:10B4C0000160AD530230ED10F0AD8F02F0D260207C
:10B4D00004C6F01AD028A9018D8D02208FC3200048
:10B4E000C1A9008D920220ACC5D0138D8F02AD8F03
:10B4F00002D028CE8C0210DE602017C6F0F020D8D3
:10B50000C4AE53021007AD8F02F0EED00EAD96021E
:10B51000F009B5E72907CD9602D0DE60A2FF8E5371
:10B5200002E88E8A022089C5F006602094C5D0FA10
:10B53000A57F55E24A900B2940F0F0A902CD8C027C
:10B54000F0E9BD7A02AA20A6C6A0034C1DC5BD0025
:10B5500002D194F00AC93FD0D2B194C9A0F0CCE88E
:10B56000C8EC7602B009BD0002C92AF00CD0DFC0D9
:10B5700013B006B194C9A0D0B2AE79028E5302B511
:10B58000E729808D8A02AD940295DDA58195D8A02A
:10B5900000B194C8482940856F6829DF300209202E
:10B5A0002927056F856FA98035E7056F95E7B5E217
:10B5B0002980057F95E2B1949D8002C8B1949D8554
:10B5C00002AD5802D007A015B1948D5802A9FF8D85
:10B5D0008F02AD78028D7902CE7902100160AE79CA
:10B5E00002B5E73005BD8002D0EEA9008D8F026064
:10B5F000A0008C9102888C5302AD85FE8580A90144
:10B6000085818D93022075D4AD9302D00160A90786
:10B610008D9502A90020F6D48D930220E8D4CE9512
:10B6200002A000B194D018AD9102D02F203BDEA52E
:10B63000818D9102A594AE92028D9202F01D60A2BE
:10B6400001EC9202D02DF013AD85FE8580AD900205
:10B6500085812075D4AD940220C8D4A9FF8D5302F2
:10B66000AD95023008A92020C6D14CD7C5204DD4B5
:10B670004CC4C5A5948D9402203BDEA5818D90021B
:10B6800060A568D028A67F561C9022A9FF8D98023D
:10B69000200ED0A0FFC902F00AC903F006C90FF0BE
:10B6A00002A000A67F9895FFD0032042D0A67FB5C8
:10B6B000FF604820A6C62088C66838ED4B02AAF075
:10B6C0000A9008A9A09194C8CAD0FA60980AA8B9AB
:10B6D00099008594B99A008595A000BD00029194C7
:10B6E000C8F006E8EC760290F260A9008D4B028A61
:10B6F00048BD0002C92CF014C93DF010EE4B02E821
:10B70000A90FCD4B029005EC740290E58E7602688D
:10B71000AA60A58348A5824820DEC6688582688520
:10B720008360A911858320EBD020E8D4AD530210AB
:10B730000AAD8D02D00A2006C81860AD8D02F01F38
:10B74000CE8D02D00DCE8D02208FC32006C8384C7E
:10B750008FC3A9008D73028D8D0220B7C73860A2F8
:10B7600018A01DB1948D7302F002A21688B1948DB9
:10B770007202E016F00AC90A9006CAC9649001CAAA
:10B7800020ACC7B194480A1005A93C9DB2026829B3
:10B790000FA8B9C5FE9DB102CAB9C0FE9DB102CACB
:10B7A000B9BBFE9DB102CACAB005A92A9DB202A9C1
:10B7B000A09DB102CAA012B1949DB102CA88C00373
:10B7C000B0F5A9229DB102E8E020B00BBDB102C9DD
:10B7D00022F004C9A0D0F0A9229DB102E8E020B077
:10B7E0000AA97F3DB1029DB10210F120B5C43860B5
:10B7F000A01BA92099B00288D0FA602019F120DF9F
:10B80000F020ACC7A9FF856FA67F8E7202A9008DBC
:10B810007302A6F9BDE0FE8595AD88FE8594A0165D
:10B82000B194C9A0D00BA9312CB194C9A0D002A960
:10B830002099B3028810F2A9128DB102A9228DB20B
:10B84000028DC302A9208DC4026020ACC7A00BB931
:10B8500017C899B1028810F74C4DEF424C4F434B3B
:10B860005320465245452E2098C32020C320CAC3EA
:10B87000A9008586209DC4303D20B7DD9033A0000F
:10B88000B1942940D02B20B6C8A013B194F00A85FA
:10B8900080C8B1948581207DC8AE5302A92035E7C8
:10B8A000D00DBD80028580BD85028581207DC8E6E2
:10B8B00086208BC410C3A5868580A901A0004CA357
:10B8C000C1205FEF2075D42019F1B5A7C9FFF0089A
:10B8D000ADF90209408DF902A90020C8D42056D143
:10B8E00085802056D18581A580D00620F4EE4C2796
:10B8F000D2205FEF204DD44C94C8A00098919420A2
:10B900005EDE4C99D5A9314CC8C1A94C8D0006A961
:10B91000C78D0106A9FA8D0206A90320D3D6A57FFB
:10B9200009E08503A50330FCC9029007A903A20022
:10B930004C0AE660A9E08D4F0220D1F02019F1A950
:10B94000FF95A7A90F8D560220E5C1D0034CC1C8B1
:10B9500020F8C12020C3AD8B022955D00FAE7A024A
:10B96000BD0002C92AD005A9304CC8C1AD8B02293F
:10B97000D9D0F44C52C9A9008D58028D8C028D800B
:10B98000028D8102A5E32901857F09018D9102AD18
:10B990007B028D7A0260204FC4AD7802C9039045C6
:10B9A000A5E2C5E3D03FA5DDC5DED039A5D8C5D910
:10B9B000D03320CCCAA9018D790220FAC92025D123
:10B9C000F004C902D005A96420C8C1A9128583ADBD
:10B9D0003C028D3D02A9FF8D3C02202ADAA2022002
:10B9E000B9C94C94C120A7C94C94C120E7CAA5E2AB
:10B9F0002901857F2086D420E4D6AE77028E790295
:10BA000020FAC9A911858320EBD02025D1D00320AD
:10BA100053CAA90885F84CD8C9209BCF2035CAA99C
:10BA20008020A6DDF0F32025D1F003209BCFAE7956
:10BA300002E8EC780290C6A91285834C02DBAE794D
:10BA400002B5E22901857FAD85FE8580B5D8858167
:10BA50002075D4AE7902B5DD20C8D4AE7902B5E741
:10BA600029078D4A02A9008D580220A0D9A00120E3
:10BA700025D1F001C8984CC8D4A9118583209BD347
:10BA80008585A682B5F2290885F8D00A2025D1F04F
:10BA900005A9802097DD6020D3D120CBE1A5D64831
:10BAA000A5D548A91285832007D120D3D120CBE189
:10BAB000209CE2A5D68587A5D58586A900858885A1
:10BAC000D485D76885D56885D64C3BE32020C3A5AF
:10BAD000E3290185E3C5E2F002098085E2204FC435
:10BAE00020E7CAA5E32901857FA5D985812057DEF6
:10BAF0002099D5A5DE18690320C8D42093DFA8AE0D
:10BB00007A02A910206EC6205EDE2099D54C94C121
:10BB1000A5E829078D4A02AE7802CAEC7702900A9E
:10BB2000BD8002D0F5A9624CC8C16020CCCABD80DE
:10BB300002F005A9634CC8C1CA10F360AD0102C987
:10BB40002DD04CAD0302856FAD04028570A000AD11
:10BB50000202C952F00E2058F2C957F037C945D039
:10BB60002E6C6F00B16F8585AD7402C906901AAE58
:10BB70000502CAF0148A18656FE66F8D4902A56F39
:10BB800085A5A57085A64C43D420EBD04C3AD4A90A
:10BB9000314CC8C1B90602916FC8CC050290F5605E
:10BBA000AC0102C030D009A9EA856BA9FF856C60A1
:10BBB0002072CB4C94C18898290F0AA8B16B857567
:10BBC000C8B16B85766C7500AD8E02857FA5834804
:10BBD000203DC6688583AE7402CAD00DA90120E25B
:10BBE000D14CF1CBA9704CC8C1A001207CCCAE8552
:10BBF00002E005B0EFA900856F857038266F2670CA
:10BC0000CA10F9A56F2D4F02D0DAA5702D5002D0C1
:10BC1000D3A56F0D4F028D4F02A5700D50028D50B0
:10BC200002A90020E2D1A682AD850295A7AAA57F30
:10BC300095009D5B02A683BD2B0209409D2B02A4AB
:10BC400082A9FF994402A98999F200B9A700993EF7
:10BC5000020AAAA9019599A90E99EC004C94C1A0D9
:10BC600000A200A92D2068C2D00AA9314CC8C1A9E0
:10BC7000304CC8C18AD0F8A205B90002DD5DCCF015
:10BC800005CA10F830E48A09808D2A02206FCCADF5
:10BC90002A020AAABD64CC8570BD63CC856F6C6F27
:10BCA0000041465257455003CDF5CC56CD73CDA338
:10BCB000CDBDCDA000A200A93A2068C2D002A00349
:10BCC000B90002C920F008C91DF004C92CD007C86A
:10BCD000CC740290EB6020A1CCEE7702AC7902E04C
:10BCE0000490ECB08AA900856F85708572A2FFB9B7
:10BCF0000002C940B018C9309014290F48A57085BA
:10BD000071A56F857068856FC8CC740290E18C79DD
:10BD10000218A900E8E003B00FB46F8830F67DF296
:10BD2000CC90F818E672D0F348AE7702A5729D80E9
:10BD300002689D850260010A6420F5CD205FEF4C0A
:10BD400094C1A9018DF90220F5CDA5814820FAF111
:10BD5000F00B68C581D0192090EF4C94C168A90000
:10BD60008581E680A580CDD7FEB00A20FAF1F0EEFD
:10BD7000A9652045E6A96520C8C120F2CD4C60D454
:10BD8000202FD1A199602036CDA90020C8D4203C15
:10BD9000CD994402A98999F200602042CD20ECD3CC
:10BDA0004C94C1206FCC2042CDB94402993E02A9E7
:10BDB000FF9944024C94C120F2CD20E8D4A888C950
:10BDC00002B002A001A90020C8D49820F1CF8A486F
:10BDD0002064D468AA20EED34C94C1206FCC20F20A
:10BDE000CD2064D44C94C12058F22036CDA90085D2
:10BDF0006FA6F9BDE0FE857020BACD4C94C16C6F82
:10BE00000020D2CDA5F90AAAAD86029599202FD19E
:10BE100020EED34C94C1A6D3E6D3BD8502A8888872
:10BE2000C00C9005A9704CC8C1858320EBD0B0F43C
:10BE30002093DF85F96020D2CDA6D3BD85022901EC
:10BE4000857FBD87028581BD86028580205FD54CB8
:10BE500000C1202CCE206ECEA59085D72071CEE6D5
:10BE6000D7E6D7A58B85D5A5900A18691085D66029
:10BE700020D9CE8592A682B5B58590B5BB8591D0E7
:10BE800004A590F00BA59038E9018590B002C69109
:10BE9000B5C7856F466F900320EDCE20E5CEA56F28
:10BEA000D0F2A5D418658B858B9006E68CD002E67F
:10BEB0008D60A9FE2CA978856FA203B58F48B58A3D
:10BEC000958F68958ACAD0F320D9CEA200B59095F7
:10BED0008FE8E00490F7A9008592246F3009068F5F
:10BEE00008468F2820E6CE20EDCE20E5CE246F3008
:10BEF0000320E2CEA58F18659085909006E691D03C
:10BF000002E692A5920591D0C2A59038E56F900CFB
:10BF1000E68BD006E68CD002E68D859060A9008580
:10BF20008B858C858D6020E5CE18269026912692F3
:10BF30006018A2FDB58E7593958EE8D0F760A200CB
:10BF40008A95FAE8E004D0F8A90695FA60A004A65C
:10BF500082B9FA0096FAC582F0078830E1AA4C0D42
:10BF6000CF602009CF20B7DFD04620D3D1208ED29A
:10BF7000304820C2DFA58048A58148A90120F6D419
:10BF80008581A90020F6D48580F01F2025D1F00BF3
:10BF900020ABDDD006208CCF4C5DCF208CCF20573E
:10BFA000DE6885816885804C6FCF68858168858073
:10BFB000208CCF2093DFAA4C99D5A9704CC8C12002
:10BFC00009CF20B7DFD008208ED230EE20C2DF604C
:10BFD000A682B5A7498095A7B5AE498095AE60A267
:10BFE0001286832007D12000C12025D19005A920E9
:10BFF000209DDDA583C90FF023D008A584298FC912
:10C000000FB0192025D1B005A5854C9DD1D0034C8A
:10C01000ABE0A58520F1CFA4824CEED3A9048582A4
:10C0200020E8D4C92AF005A58520F1CFA5F8F001B4
:10C0300060EE550260482093DF100668A9614CC885
:10C04000C10AAA688199F6996020D1C12042D04CDA
:10C0500094C1200FF1A8B6A7E0FFD01448208ED2DB
:10C06000AA1005A9702048E668A88A098099A70047
:10C070008A290F85F9A2008681AE85FE868020D3AD
:10C08000D6A9B04C8CD520D1F02013D3200ED0A649
:10C090007FA9009D51028A0AAAA5169512A5179597
:10C0A000132086D5A5F90AAAA9029599A199A67F78
:10C0B0009D0101A900951C95FF203AEFA004A9005D
:10C0C000AA18716D9001E8C8C8C8C8C048F0F8C087
:10C0D00090D0EE488AA67F9DFC02689DFA026020FF
:10C0E000D0D620C3D02099D52037D185802037D114
:10C0F000858160209BD0A580D00160201ECF20D0FC
:10C10000D620C3D04C1ECFA980D002A9908D4D025D
:10C110002093DFAA2006D58A480AAAA9009599206B
:10C1200025D1C904B006F6B5D002F6BB68AA60A551
:10C1300083C9139002290FC90FD002A910AA38BDD4
:10C140002B023006290F8582AA1860A583C9139097
:10C1500002290FAABD2B02A80A900A300A98290FBB
:10C160008582AA186030F63860A682B5EC4A2907A5
:10C17000C904602093DF0AAAA48260202FD1B944A9
:10C1800002F012A19948B599D94402D004A9FF95AB
:10C190009968F69960A199F699602037D1D03685D3
:10C1A00085B94402F008A98099F200A58560201E97
:10C1B000CFA90020C8D42037D1C900F0198580202C
:10C1C00037D18581201ECF20D3D120D0D620C3D017
:10C1D000201ECFA585602037D1A482994402A58571
:10C1E0006020F1CFF0016020D3D1201EF1A9002002
:10C1F000C8D4A58020F1CFA58120F1CF20C7D020C1
:10C200001ECF20D0D6A9024CC8D4856F20E8D41800
:10C21000656F95998594602093DFAABD5B02290123
:10C22000857F6038B0011808856F2027D2207FD322
:10C230008582A68328900209809D2B02293FA8A908
:10C24000FF99A70099AE0099CD00C66F301C208ED3
:10C25000D21008205AD2A9704CC8C199A700C66F45
:10C260003008208ED230EC99AE0060A583C90FD083
:10C270000160A683BD2B02C9FFF022293F8582A958
:10C28000FF9D2B02A682A90095F2205AD2A682A970
:10C2900001CA30030AD0FA0D56028D560260A682FA
:10C2A000B5A7C9FFF00948A9FF95A76820F3D2A652
:10C2B00082B5AEC9FFF00948A9FF95AE6820F3D258
:10C2C000A682B5CDC9FFF00948A9FF95CD6820F336
:10C2D000D2609848A00120BAD2100C8820BAD2109F
:10C2E000062039D3AA3013B50030FCA57F95009DF8
:10C2F0005B028A0AA8A90299990068A88A60A20725
:10C30000B94F023DE9EFF004CA10F560B94F025D84
:10C31000E9EF994F028A883003186908AA60A6825B
:10C32000B5A730098A186907AAB5A710F0C9FFF0A8
:10C33000EC48A9FF95A768290FA8C8A2106E500263
:10C340006E4F0288D00118CA10F360A90E858320B1
:10C3500027D2C683D0F960A90E8583A683BD2B02A0
:10C36000C9FFF014293F85822093DFAABD5B022913
:10C3700001C57FD0032027D2C68310DF60A56F4898
:10C38000A000B6FAB5A71004C9FFD0168A1869072D
:10C39000AAB5A71004C9FFD009C8C00590E4A2FF40
:10C3A000D01C866F293FAAB50030FCC9029008A6B0
:10C3B0006FE00790D7B0E2A46FA9FF99A700688546
:10C3C0006F8A60A000A9012C5602D009C80AD0F7D4
:10C3D000A9704CC8C149FF2D56028D5602986020A5
:10C3E000EBD02000C120AAD3A682BD3E0260A68267
:10C3F0002025D1D0034C20E1A583C90FF05AB5F216
:10C400002908D0132025D1C907D007A98995F24C56
:10C41000DED3A90095F260A583F0322025D1C904AE
:10C420009022202FD1B599D94402D004A900959922
:10C43000F699A199993E02B599D94402D005A981EE
:10C4400099F200602056D1A6829D3E0260AD540252
:10C45000F0F22067ED4C03D420E8D4C9D4D018A55D
:10C4600095C902D012A90D85852023C1A90020C13C
:10C47000E6C6A5A980D0122037D18585D009A9D4D8
:10C4800020C8D4A902959AA98885F7A5858D43026D
:10C49000602093DF0AAAA9009599A199F005D69981
:10C4A0004C56D160A980D002A990057F8D4D02A580
:10C4B000F920D3D6A6F94C93D5A9018D4A02A9112A
:10C4C00085832046DCA9024CC8D4A91285834CDAA6
:10C4D000DC203BDEA901856FA56948A90385692099
:10C4E0002DF1688569A90020C8D4A58020F1CFA5C9
:10C4F0008120F1CF20C7D02099D5A90020C8D42011
:10C50000F1CFD0FB20F1CFA9FF4CF1CF856F209365
:10C51000DF0AAAB59A8595A56F9599859460A911AA
:10C5200085832027D2A91285834C27D22093DF0A46
:10C53000AAB59A8595B59985946085712093DFAAEF
:10C54000BDE0FE8572A000B17160BD5B0229010DE6
:10C550004D024886F98A0AAAB5078D4D02B506F044
:10C560002DCDD7FEB028AA684829F0C990D04F68D1
:10C57000484AB005AD01019003AD0201F005CDD5EB
:10C58000FED0338A204BF2CD4D02F002B030205263
:10C59000D5A9664C45E6A5F90AAAB5068580B50772
:10C5A000858160A580F0EACDD7FEB0E5204BF2C5CD
:10C5B00081F0DE90DC602052D5A9734C45E6A6F9E7
:10C5C000688D4D0295009D5B0260A980D002A99004
:10C5D000057FA6F98D4D02AD4D02200ED520A6D5C2
:10C5E000B0FB48A9008D98026860B500301AC902F6
:10C5F0009014C908F008C90BF004C90FD00C2C988E
:10C600000230034C3FD6186038609848A57F48BD7B
:10C610005B022901857FA8B9CAFE8D6D0220A6D6CE
:10C62000C902B0034C6DD6BD5B0229F048C990D059
:10C6300007A57F09B89D5B02246A7039A9008D990E
:10C64000028D9A02AC9902AD9A0238F9DBFE8D9AFE
:10C6500002B9DBFE2076D6EE990220A6D6C902905A
:10C6600008AC9902B9DBFED0DBAD9A022076D6B5D4
:10C6700000C902902B246A100F68C990D005057F6D
:10C680009D5B02B500200AE6682C9802302348A979
:10C69000C0057F9500B50030FC20A6D6C902B0D9F0
:10C6A00068C990D00C057F9D5B0220A6D6C902B058
:10C6B000D268857F68A8B5001860C900F018300CF2
:10C6C000A0012093D638E901D0F6F00AA0FF20930C
:10C6D000D6186901D0F6604898A47F99FE02D9FE69
:10C6E00002F0FBA90099FE026860A56A293FA8AD87
:10C6F0006D024D001C8D001CBD5B029500B5003025
:10C70000FCC902900388D0E748AD6D020D001C8D76
:10C71000001C68602093DF0AA8A580990600A58107
:10C72000990700A57F0AAA60A58348A58248A5812C
:10C7300048A58048A9118583203BDEAD4A0248A563
:10C74000E22901857FA6F95D5B024A900CA2018E69
:10C75000920220ACC5F01DD028AD9102F00CC5812D
:10C76000F01F85812060D44C3DD7A9018D92022015
:10C7700017C6D00D208DD4A5818D9102A9028D926E
:10C7800002AD920220C8D4688D4A02C904D00209C1
:10C790008020F1CF688D800220F1CF688D85022046
:10C7A000F1CF2093DFA8AD7A02AAA910206EC6A00F
:10C7B00010A9009194C8C01B90F9AD4A02C904D0D9
:10C7C00013A010AD59029194C8AD5A029194C8AD0E
:10C7D000580291942064D4688582AA688583AD91BB
:10C7E0000285D89D6002AD920285DD9D6602AD4A4C
:10C7F0000285E7A57F85E260A5838D4C0220B3C248
:10C800008E2A02AE0002AD4C02D02CE02AD028A520
:10C810007EF04D8580AD6E02857F85E2A90285E7B9
:10C82000AD6F0285812000C12046DCA904057FA6EA
:10C830008299EC004C94C1E024D01EAD4C02D00390
:10C840004C55DA20D1C1AD85FE8580A900858120B7
:10C8500046DCA57F09024CEBD7E023D0124C84CBF9
:10C86000A9028D9602A900857F8D8E022042D020DC
:10C87000E5C1D004A200F00C8AF005A9304CC8C173
:10C8800088F001888C7A02A98D2068C2E88E78022F
:10C890002012C320CAC3209DC4A2008E58028E97C6
:10C8A000028E4A02E8EC7702B0102009DAE8EC7751
:10C8B00002B007C004F03E2009DAAE4C028683E0E5
:10C8C00002B0128E9702A9408DF902AD4A02D01B28
:10C8D000A9028D4A02AD4A02D011A5E729078D4A67
:10C8E00002AD8002D005A9018D4A02AD9702C901AF
:10C8F000F0184C40D9BC7A02B900028D5802AD80C4
:10C9000002D0B7A9018D9702D0B0A5E72980AAD09F
:10C9100014A92024E7F00620B6C84CE3D9AD800264
:10C92000D0034CE3D9AD0002C940F00D8AD005A96F
:10C93000634CC8C1A9334CC8C1A5E72907CD4A0239
:10C94000D067C904F06320DADCA5828D7002A911DA
:10C95000858320EBD0AD940220C8D4A000B1940907
:10C96000209194A01AA5809194C8A5819194AE704D
:10C9700002A5D89D6002A5DD9D6602203BDE2064F5
:10C98000D44CEFD9AD8002D005A9624CC8C1AD9797
:10C9900002C903F00BA92024E7F005A9604CC8C127
:10C9A000A5E72907CD4A02F005A9644CC8C1A0003B
:10C9B0008C7902AE9702E002D01AC904F0EBB19470
:10C9C000294F9194A58348A9118583203BDE2064DB
:10C9D000D468858320A0D9AD9702C902D055202AFA
:10C9E000DA4C94C1A013B1948D5902C8B1948D5AF8
:10C9F00002C8B194AE58028D58028AF00ACD58028E
:10CA0000F005A95020C8C1AE7902BD80028580BD65
:10CA1000850285812046DCA482AE7902B5D8996072
:10CA200002B5DD99660260A5E22901857F20DADC86
:10CA300020E4D6A583C902B011203EDEA580857E04
:10CA4000A57F8D6E02A5818D6F024C99C1BC7A02C3
:10CA5000B90002A004883008D9B2FED0F88C970241
:10CA6000A005883008D9B6FED0F88C4A026020397B
:10CA7000CAA98020A6DDF0F62095DEA681E88AD03E
:10CA80000520A3D1A90220C8D4A682A90195F2A9A4
:10CA9000800582A6839D2B0260A90C8D2A02A90025
:10CAA000AE7402CAF00BCAD021AD010220BDC33062
:10CAB0001985E2EE7702EE7802EE7A02A98085E728
:10CAC000A92A8D00028D0102D01820E5C1D00520D1
:10CAD000DCC2A00388888C7A022000C22098C32080
:10CAE00020C320CAC320B7C7209DC4209EEC203796
:10CAF000D1A6829D3E02A57F8D8E02090495ECA9E8
:10CB00000085A360A9008DF902A583D00BA9008D33
:10CB100054022027D24CDAD4C90FF0142002DBA52E
:10CB200083C90290F0AD6C02D0034C94C14CADC1EE
:10CB3000A90E85832002DBC68310F9AD6C02D003F9
:10CB40004C94C14CADC1A683BD2B02C9FFD001607E
:10CB5000290F85822025D1C907F00FC904F01120C3
:10CB600007D1B0092062DB20A5DB20F4EE4C27D2F0
:10CB700020F1DD201ECF20CBE1A6D58673E673A978
:10CB80000085708571A5D638E90E85722051DFA623
:10CB900082A57095B5A57195BBA94020A6DDF003CF
:10CBA00020A5DB4C27D2A682B5B515BBD00C20E85A
:10CBB000D4C902D005A90D20F1CF20E8D4C902D0F4
:10CBC0000F201ECFA682B5B5D002D6BBD6B5A90020
:10CBD00038E90148A90020C8D420F1CF6820F1CF5E
:10CBE00020C7D02099D54C1ECFA6828E7002A58377
:10CBF00048BD60028581BD66028D9402B5EC2901B5
:10CC0000857FAD85FE85802093DF4885F92060D43F
:10CC1000A000BDE0FE8587AD94028586B1862920FF
:10CC2000F0432025D1C904F044B186298F9186C8EC
:10CC3000B18685808471A01BB1864888B186D00AF0
:10CC40008580688581A9672045E648A9009186C846
:10CC5000918668A4719186C8B18685816891862085
:10CC60007DC84C29DCB186290F09809186AE7002FF
:10CC7000A01CB5B59186C8B5BB918668AAA99005D8
:10CC80007F2090D56885834C07D1A90120E2D1206F
:10CC9000B6DCAD4A02480A057F95EC209BD0A682FF
:10CCA000A580D005A5819D440268C904D03FA48316
:10CCB000B92B020940992B02AD580295C7208ED29C
:10CCC00010034C0FD2A68295CDAC59028480AC5A89
:10CCD00002848120D3D62073DE2099D5A682A902B2
:10CCE00095C1A90020C8D42053E14C3EDE2056D186
:10CCF000A6829D3E02A98895F260A682B5A70AA8E1
:10CD0000A902999900B5AE098095AE0AA8A9029921
:10CD10009900A90095B595BBA9009D44026020A982
:10CD2000F1A90120DFD120D0D620B6DCA682AD4A01
:10CD300002480A057F95EC68C904F005A90195F23F
:10CD400060A483B92B02293F0940992B02AD5802F8
:10CD500095C7208ED210034C0FD2A68295CD20C14C
:10CD6000DE201EF1A5808D5902A5818D5A02A68272
:10CD7000B5CD20D3D6A90020E9DEA900208DDDA9FC
:10CD800011208DDDA900208DDDAD5802208DDDA59F
:10CD900080208DDDA581208DDDA91020E9DE203EDB
:10CDA000DEA580208DDDA581208DDD206CDE209923
:10CDB000D5A90220C8D4A68238A900F5C795C120FC
:10CDC000E2E22019DE205EDE2099D520F4EE4C98B8
:10CDD000DC48A682B5CD4CFDCF9006A68215ECD0DE
:10CDE00006A68249FF35EC95EC60A68235EC602002
:10CDF00093DFAABD5B0229F0C99060A2008671BDD5
:10CE00002B02C9FFD008A671E8E01090F06086718F
:10CE1000293FA8B9EC0029018570AE5302B5E2297B
:10CE200001C570D0E1B96002D5D8D0DAB96602D5B3
:10CE3000DDD0D31860209EDF5006205EDE2099D51D
:10CE400060202BDEA5809194C8A58191944C05E1CA
:10CE5000202BDEB1948580C8B194858160202BDEC3
:10CE6000A9009194C8A682B5C1AACA8A91946020EB
:10CE700093DF0AAAB59A8595A9008594A000602041
:10CE8000EBD02093DF85F90AA8B906008580B907A1
:10CE900000858160A9908D4D02D028A9808D4D021A
:10CEA000D021A9908D4D02D026A9808D4D02D01F92
:10CEB000A9908D4D02D002A9808D4D02A682B5CDDC
:10CEC000AA101320D0D62093DFAAA57F9D5B022055
:10CED00015E12093DFAA4C06D5A90020C8D420373D
:10CEE000D185802037D185816048A900856F857103
:10CEF000B9E0FE8570BDE0FE857268A888B16F91CB
:10CF0000718810F960A8B9E0FE8570A900856FA846
:10CF1000916FC8D0FB60A90020DCDEA002B1946054
:10CF20008594A682B5CDAABDE0FE8595604820DC3B
:10CF3000DE488A0AAA68959A689599602066DF306B
:10CF40000E5013A682B5CD201BDF2066DF10072010
:10CF5000CBE12CCEFE60A5D620E9DE2CCDFE60858F
:10CF6000F9A980D00485F9A99048B5EC2901857FFD
:10CF700068057F8D4D02B1948580C8B1948581A5E7
:10CF8000F920D3D6A6F94C93D5A682B5CD4CEBD4D7
:10CF9000A978205CDFCA10F8A5724A205CDFA5736F
:10CFA00018657085709002E6716020D2DEC5D5D01C
:10CFB0000EA4D6B194F0042CCDFE602CCFFE60A55B
:10CFC000D5C906B00A0AA8A9048594B194D0042C46
:10CFD000D0FE602CCEFE60A682B5A71002B5AE29A9
:10CFE000BF60A6828E5702B5A710098A1869078DFF
:10CFF0005702B5AE8570291F247060A682B5A73090
:10D0000002B5AEC9FF60A6820980B4A7100395A738
:10D010006095AE60A920209DDDA98020A6DDD041CD
:10D02000A682F6B5D002F6BBA682B5C1F02E20E8E6
:10D03000D4A682D5C19003203CE0A682B5C120C809
:10D04000D4A1998585A920209DDD2004E34890285E
:10D05000A90020F6D4D02168C902F012A980209737
:10D06000DD202FD1B599994402A90D858560203521
:10D07000E0A682A90095C16068A68295C14C6EE1C8
:10D0800020D3D12095DE209EDF5016205EDE201EAC
:10D09000CFA90220C8D420ABDDD0242057DE4C9984
:10D0A000D5201ECF20ABDDD0062057DE2099D5201D
:10D0B00095DEA580F009201ECF2057DE201ECF6010
:10D0C0002005E12093DF0AAAA5858199B499C8D0EB
:10D0D00009A482B9C100F00AA00298A482D9C100B3
:10D0E000D005A9204C97DDF699D003203CE060A93B
:10D0F000A020A6DDD027A585207CE0A5F8F00D6056
:10D10000A92020A6DDF005A9518D6C0220F3E020B6
:10D1100053E1AD6C02F0034CC8C14CBCE62980D091
:10D1200005A5F8F0DB60A58548201CE3688585A986
:10D1300080209DDD4CB2E0A92020A6DDD00AA90008
:10D140008585207CE04CF3E060A9402097DD209E9F
:10D15000DF0940AE570295A760209EDF29BFAE577A
:10D160000295A760A98020A6DDD037202FD1B599E0
:10D17000D94402F022F699D006203CE0202FD1A11C
:10D1800099993E02A98999F200B599D94402F00112
:10D1900060A98199F2006020D0DF202FD1A5854CB5
:10D1A0003DE1A682A90D9D3E02A98195F2A95020DC
:10D1B000C8C1A682B5C18587C687C902D004A9FFA8
:10D1C0008587B5C7858820E8D4A682C5879019F0E1
:10D1D00017201ECF20B2E19008A6829D44024C1E6B
:10D1E000CF201ECFA9FF858720B2E1B00320E8D46D
:10D1F000A6829D440260202BDEA487B194D00D88C6
:10D20000C0029004C688D0F3C688186098386020A1
:10D21000D2DE85D5A9048594A00AD004888830265A
:10D22000B194F0F8984AC5D5F00985D5A682B5CD58
:10D23000201BDFA0008494B194D00BC8B194A888BF
:10D2400084D6984CE9DEA9672045E620B3C2AD013B
:10D2500002858320EBD09005A97020C8C1A9A02029
:10D260009DDD2025D1F005A96420C8C1B5EC2901B8
:10D27000857FAD020295B5AD030295BBA682A98953
:10D2800095F2AD0402F01038E901F00BD5C7900714
:10D29000A9518D6C02A90085D4200ECE20F8DE5055
:10D2A00008A9802097DD4C5EE12075E2A98020A6C8
:10D2B000DDF0034C5EE14C94C1209CE2A5D720C870
:10D2C000D4A682B5C738E5D4B0034C02E21865D7BE
:10D2D00090036901382009E04C38E1A95120C8C108
:10D2E000A5948589A595858A20D0E2D0016020F19A
:10D2F000DD200CDEA580F00E20D3E2D006201ECF6C
:10D300004CDAD220DAD2A000B1898580C8B18985F3
:10D31000814CAFD0203EDEA000B189C580F0016015
:10D32000C8B189C58160202BDEA002A9009194C8F4
:10D33000D0FB2004E395C1A8A9FF91942004E390B9
:10D34000F4D004A90095C160A682B5C138F00D18CB
:10D3500075C7900BD006A9022CCCFE60690138601D
:10D3600020D3D120CBE1209CE2207BCFA5D685879E
:10D37000A5D58586A9008588A90085D4200ECE2054
:10D380004DEFA482B6C7CA8A1865D7900CE6D6E6D8
:10D39000D6D006E6D5A91085D6A58718690220E95A
:10D3A000DEA5D5C9069005A95220C8C1A5D638E585
:10D3B00087B003E90F188572A5D5E5868573A200AD
:10D3C00086708671AA2051DFA571D007A670CAD0D9
:10D3D00002E688CD73029009D0CDAD7202C570907F
:10D3E000C6A90120F6D4186901A68295C1201EF1B4
:10D3F00020FDDDA588D015205EDE201ECF20D0D6F2
:10D40000201EF120FDDD20E2E24CD4E3201ECF20DF
:10D41000D0D620E2E22019DE205EDE200CDEA580E0
:10D4200048A58148203EDEA58148A580482045DFEB
:10D43000AAD00A204EE4A91020E9DEE68668208DF5
:10D44000DD68208DDD688581688580F00FA586C543
:10D45000D5D0A72045DFC5D690A0F0B02045DF4845
:10D46000A90020DCDEA900A89194C86838E90191E0
:10D4700094206CDE2099D520F4EE200ECE201ECF15
:10D4800020F8DE70034C75E2A9802097DDA95020BA
:10D49000C8C1201EF1201ECF20F1DD2093DF4820DF
:10D4A000C1DEA682B5CDA868AAA91020A5DEA90074
:10D4B00020DCDEA002B19448A90020C8D468186915
:10D4C0000191940A69048589A838E902858AA580B2
:10D4D00085879194C8A58185889194A0009891949E
:10D4E000C8A9119194A91020C8D42050DE2099D544
:10D4F000A682B5CD48209EDFA68295CD68AE5702A4
:10D5000095A7A90020C8D4A000A5809194C8A581A2
:10D5100091944CDEE42093DFA682201BDFA900203B
:10D52000C8D4C68AC68AA489A5879194C8A58891BB
:10D5300094205EDE2099D5A48AC003B0D84C1ECFBB
:10D5400000A04FCB202122232427D24541448952D9
:10D550008320544F4F204C415247C5508B062050DA
:10D56000524553454ED451CF564552464C4F572005
:10D57000494E8B25288A89268A2050524F5445438C
:10D5800054204FCE2988204944853031323334D35A
:10D59000594E54415889608A038463832045584911
:10D5A0005354D3648320545950458565CE4F20424F
:10D5B0004C4F43CB6667C94C4C4547414C205452B5
:10D5C00041434B204F5220534543544FD261830671
:10D5D0008439628306870183532053435241544365
:10D5E0004845C470CE4F204348414E4E45CC71C48F
:10D5F00049528972882046554CCC73C3424D204411
:10D600004F532056322E3620313534B174C452492E
:10D610005645062052454144D909C552524FD20AB7
:10D62000D7524954C503C6494CC504CF5045CE0511
:10D63000CD49534D415443C806CE4FD407C64F552C
:10D640004EC408C44953CB0BD245434F52C44886FD
:10D65000F98A0AAAB5068580B507858168290FF081
:10D6600008C90FD006A974D008A9060920AACACAF9
:10D670008A48AD2A02C900D00FA9FF8D2A0268206E
:10D68000C7E62042D04C48E66820C7E620BDC1A9C5
:10D69000008DF902202CC120DAD4A90085A3A2456F
:10D6A0009AA584290F8583C90FF03178A579D01CFC
:10D6B000A57AD010A683BD2B02C9FFF01F290F85C4
:10D6C000824C8EE620EBD0204EEAD0062007D120F7
:10D6D0004EEA2025D1C904B0032027D24CE7EBAA9B
:10D6E000A900F8E000F007186901CA4C9FE6D8AA23
:10D6F0004A4A4A4A20B4E68A290F093091A5C860EF
:10D700002023C1A900A00084808481A000A2D58626
:10D71000A5A20286A620ABE6A92C91A5C8ADD5028C
:10D720008D43028A2006E7A92C91A5C8A580209BDD
:10D73000E6A92C91A5C8A581209BE688981869D5F3
:10D740008D4902E6A5A98885F760AAA58648A58720
:10D7500048A9FC8586A9E485878AA200C186F021B4
:10D76000482075E790052075E790FBA587C9E690EE
:10D7700008D00AA90AC5869004684C18E7684C4D81
:10D78000E72067E790FB2054E72067E790F82054F4
:10D79000E768858768858660C920B00BAAA92091B3
:10D7A000A5C88A2006E76091A5C860E686D002E693
:10D7B00087A1860AA186297F60206DE7E686D002D0
:10D7C000E6876060AD0018AA2904F0F78A2901F005
:10D7D000F258AD00182905D0F9EE7802EE7402A9CE
:10D7E0002A8D00024CA8E7A98D2068C22058F2AD0E
:10D7F000780248A9018D7802A9FF8586204FC4AD23
:10D800008002D005A93920C8C1688D7802AD800298
:10D810008580AD85028581A9032077D4A9008587FD
:10D820002039E88588204BE82039E88589204BE8B5
:10D83000A586F00AA58848A58948A90085862039CB
:10D84000E8858A204BE82039E8A0009188204BE841
:10D85000A58818690185889002E689C68AD0E720E4
:10D8600035CAA585C587F008203EDEA9502045E6CB
:10D87000A5F8D0A86885896885886C88002035CA95
:10D88000A5F8D008203EDEA9512045E6A585601800
:10D8900065876900858760AD0118A901857C60787E
:10D8A000A900857C8579857AA2459AA98085F88525
:10D8B0007D20B7E920A5E9AD001809108D0018AD4D
:10D8C000001810572904D0F720C9E9C93FD006A98C
:10D8D000008579F071C95FD006A900857AF067C527
:10D8E00078D00AA901857AA9008579F029C577D071
:10D8F0000AA9018579A900857AF01BAA2960C96067
:10D90000D03F8A8584290F8583A58429F0C9E0D07A
:10D91000355820C0DA782C001830ADA900857DADCF
:10D92000001829EF8D0018A579F006202EEA4CE7A3
:10D93000EBA57AF009209CE920AEE92009E94C4EDC
:10D94000EAA9108D00182C001810D030F97820EBBF
:10D95000D0B006A682B5F23001602059EA20C0E9B5
:10D9600029010820B7E928F0122059EA20C0E92946
:10D9700001D0F6A682B5F22908D0142059EA20C0B9
:10D98000E92901D0F62059EA20C0E92901F0F62062
:10D99000AEE92059EA20C0E92901D0F3A908859809
:10D9A00020C0E92901D036A682BD3E026A9D3E0212
:10D9B000B00520A5E9D003209CE920B7E9A523D034
:10D9C0000320F3FE20FBFEC698D0D52059EA20C0E4
:10D9D000E92901F0F65820AAD3784C0FE94C4EEA19
:10D9E000AD001829FD8D001860AD001809028D00EA
:10D9F0001860AD001809088D001860AD001829F7EF
:10DA00008D001860AD0018CD0018D0F860A9088509
:10DA1000982059EA20C0E92904D0F6209CE9A90100
:10DA20008D05182059EAAD0D182940D00920C0E90C
:10DA30002904F0EFD01920A5E9A20ACAD0FD209C44
:10DA4000E92059EA20C0E92904F0F6A90085F8ADDB
:10DA5000001849014A2902D0F6EAEAEA6685205907
:10DA6000EA20C0E92904F0F6C698D0E320A5E9A58C
:10DA70008560782007D1B005B5F26AB00BA584297E
:10DA8000F0C9F0F0034C4EEA20C9E95820B7CF4C5A
:10DA90002EEAA9008D00184CE7EB4C5BE8A57DF061
:10DAA00006AD0018100960AD001810FA4C5BE84C88
:10DAB000D7E8A2002CA66F9ABAA9080D001C4CEA60
:10DAC000FE98186901D0FC88D0F8AD001C29F78DAC
:10DAD000001C98186901D0FC88D0F8CA10DBE0FC63
:10DAE000D0F0F0D478D8A2FF8E0318E8A000A200EE
:10DAF0008A9500E8D0FA8AD500D0B7F600C8D0FBE6
:10DB0000D500D0AE9400B500D0A8E8D0E9E66F8685
:10DB100076A9008575A8A22018C6767175C8D0FBB5
:10DB2000CAD0F66900AAC576D039E0C0D0DFA90115
:10DB30008576E66FA207981865769175C8D0F7E6E6
:10DB400076CAD0F2A207C6768898186576D175D0C5
:10DB50001249FF917551759175D00898D0EACAD0D5
:10DB6000E5F0034C71EAA2459AAD001C29F78D003F
:10DB70001CA9018D0C18A9828D0D188D0E18AD00F1
:10DB80001829600A2A2A2A0948857849608577A2D7
:10DB900000A000A9009599E8B9E0FE9599E8C8C0F1
:10DBA00005D0F0A9009599E8A9029599E8A9D5951D
:10DBB00099E8A9029599A9FFA2129D2B02CA10FA11
:10DBC000A20595A795AE95CDCA10F7A90585ABA975
:10DBD0000685ACA9FF85AD85B4A9058D3B02A98456
:10DBE0008D3A02A90F8D5602A90185F6A98885F7FD
:10DBF000A9E08D4F02A9FF8D5002A901851C851D4A
:10DC00002063CB20FACE2059F2A9228565A9EB85A5
:10DC100066A90A8569A905856AA97320C1E6A91ABA
:10DC20008D0218A9008D00182080E758AD00182932
:10DC3000E58D0018AD5502F00AA9008D55028567E3
:10DC40002046C158A57CF0034C5BE858A90E8572AC
:10DC5000A900856F8570A672BD2B02C9FFF010293F
:10DC60003F85822093DFAABD5B022901AAF66FC619
:10DC70007210E3A004B9000010052901AAF66F880C
:10DC800010F378AD001C29F748A57F8586A900858B
:10DC90007FA56FF00BA51CF0032013D3680908487B
:10DCA000E67FA570F00BA51DF0032013D3680900D3
:10DCB00048A586857F68AE6C02F021AD001CE0802F
:10DCC000D0034C8BECAE05183012A2A08E0518CEF6
:10DCD0006C02D0084D6D02A2108E6C028D001C4C9F
:10DCE000FFEBA9008583A90120E2D1A90020C8D4B7
:10DCF000A682A9009D44022093DFAAA57F9D5B0216
:10DD0000A90120F1CFA90420F1CFA90120F1CF2052
:10DD1000F1CFAD720220F1CFA90020F1CF2059ED53
:10DD20002093DF0AAAD699D699A90020F1CFA9019C
:10DD300020F1CF20F1CF20CEC6902CAD720220F181
:10DD4000CFAD730220F1CF2059EDA90020F1CFD043
:10DD5000DD2093DF0AAAA9009599A988A4828D5491
:10DD60000299F200A58560AD720220F1CFAD730279
:10DD700020F1CF2059ED2093DF0AAAD699D699A990
:10DD80000020F1CF20F1CF20F1CF2093DF0AA8B9F6
:10DD90009900A6829D4402DE44024C0DEDA000B91C
:10DDA000B10220F1CFC8C01BD0F5602037D1F001FF
:10DDB000608585A482B94402F008A98099F200A583
:10DDC00085604820EAEC686020D1C12042D0A9409B
:10DDD0008DF90220B7EEA9008D920220ACC5D03D8E
:10DDE000A9008581AD85FE858020E5EDA9008DF92E
:10DDF0000220FFEE4C94C1C8B19448C8B19448A029
:10DE000013B194F00A8580C8B194858120E5ED684E
:10DE1000858168858020E5ED2004C6F0C3A000B1AF
:10DE20009430D420B6C84CD4ED205FD52090EF209C
:10DE300075D4A90020C8D42037D185802037D1855A
:10DE400081A580D0034C27D22090EF204DD44CEEFA
:10DE5000ED2012C3A5E21005A9334CC8C1290185E4
:10DE60007F2000C1A57F0AAAAC7B02CC7402F01A05
:10DE7000B900029512B9010295132007D3A90185B3
:10DE80008020C6C82005F04C56EE2042D0A67FBDAB
:10DE90000101CDD5FEF0034C72D520B7EEA5F9A84F
:10DEA0000AAAAD88FE9599AE7A02A91B206EC6A07B
:10DEB00012A67FADD5FE9D01018A0AAAB5129194E2
:10DEC000C8B5139194C8C8A9329194C8ADD5FE9134
:10DED00094A002916DAD85FE85802093EFA9018508
:10DEE000812093EF20FFEE2005F0A001A9FF916DA6
:10DEF0002064D4C6812060D44C94C120D1F0A0000D
:10DF0000A912916DC898916DC8C8C8A900856F8580
:10DF1000708571984A4A204BF2916DC8AA38266FD5
:10DF200026702671CAD0F6B56F916DC8E8E00390EF
:10DF3000F6C09090D64C75D02093DFAABD5B022925
:10DF400001857FA47FB95102D00160A900995102D7
:10DF5000203AEFA57F0A4820A5F06818690120A59E
:10DF6000F0A58048A90185800A0A856D2020F2E687
:10DF700080A580CDD7FE90F06885804C8AD5200F93
:10DF8000F1AA20DFF0A6F9BDE0FE856EA900856D3F
:10DF900060A67FBDFA028D7202BDFC028D73026025
:10DFA00020F1EF20CFEF38D022B16D1DE9EF916D58
:10DFB0002088EFA46F18B16D6901916DA580CD85A2
:10DFC000FEF03BFEFA02D003FEFC0260A67FA90130
:10DFD0009D51026020F1EF20CFEFF036B16D5DE989
:10DFE000EF916D2088EFA46FB16D38E901916DA5B7
:10DFF00080CD85FEF00BBDFA02D003DEFC02DEFA16
:10E0000002BDFC02D00CBDFA02C903B005A9722002
:10E01000C7E6602011F098856FA5814A4A4A3865A5
:10E020006FA8A5812907AAB16D3DE9EF600102043F
:10E030000810204080A9FF2CF902F00C100A70088B
:10E04000A9008DF9024C8AD560203AEFA000989182
:10E050006DC8D0FB60A56F48A57048A67FB5FFF0DE
:10E0600005A9742048E6200FF1856F8A0A8570AAF9
:10E07000A580DD9D02F00BE88670DD9D02F0032097
:10E080005BF0A570A67F9D9B020A0A1869A1856DA9
:10E09000A9026900856EA00068857068856F60A61A
:10E0A0006F20DFF0A57FAA0A1D9B02490129038585
:10E0B0007020A5F0A5F90AAAA5800A0A9599A5706D
:10E0C0000A0AA8A19999A102A9008199F699C8986C
:10E0D0002903D0EFA670A5809D9D02ADF902D00363
:10E0E0004C8AD509808DF90260A8B99D02F02548B7
:10E0F000A900999D02A5F90AAA680A0A9599980AA1
:10E100000AA8B9A1028199A90099A102F699C89813
:10E110002903D0EE60A57F0AAAA9009D9D02E89D73
:10E120009D0260B5A7C9FFD0258A48208ED2AA10CB
:10E1300005A97020C8C186F968A88A098099A70036
:10E140000AAAAD85FE9506A90095074C86D5290F2C
:10E1500085F960A906A67FD00318690760200FF132
:10E16000AA60203EDEA903856FA9010DF9028DF991
:10E1700002A56F482011F068856FB16DD039A58078
:10E18000CD85FEF019901CE680A580CDD7FED0E1AC
:10E19000AE85FECA8680A9008581C66FD0D3A972DC
:10E1A00020C8C1C680D0CAAE85FEE88680A9008599
:10E1B00081C66FD0BCF0E7A5811865698581A5800F
:10E1C000204BF28D4E028D4D02C581B00C38A581D9
:10E1D000ED4E028581F002C68120FAF1F0034C90E9
:10E1E000EFA900858120FAF1D0F44CF5F1A9010DD9
:10E1F000F9028DF902A58648A9018586AD85FE380C
:10E20000E58685809009F0072011F0B16DD01BAD37
:10E2100085FE1865868580E686CDD7FE9005A967C0
:10E220002045E62011F0B16DF0D2688586A9008501
:10E230008120FAF1F0034C90EFA9712045E62011FE
:10E24000F098482020F2A580204BF28D4E02688580
:10E250006FA581CD4E02B00920D5EFD006E681D062
:10E26000F0A90060A56F48A900856FAC86FE88A262
:10E2700007B16D3DE9EFF002E66FCA10F488D0EF08
:10E28000B16DC56FD00468856F60A9712045E6AE99
:10E29000D6FEDDD6FECAB0FABDD1FE6060A96F8D94
:10E2A000021C29F08D001CAD0C1C29FE090E09E092
:10E2B0008D0C1CA9418D0B1CA9008D061CA93A8D43
:10E2C000071C8D051CA97F8D0E1CA9C08D0D1C8DF2
:10E2D0000E1CA9FF853E8551A9088539A9078547E8
:10E2E000A9058562A9FA8563A9C88564A904855E24
:10E2F000A904855FBA8649AD041CAD0C1C090E8DBE
:10E300000C1CA005B90000102EC9D0D004984C7088
:10E31000F32901F007843FA90F4C69F9AA853DC58F
:10E320003EF00A207EF9A53D853E4C9CF9A52030A3
:10E33000030A10094C9CF98810CA4C9CF9A9208545
:10E3400020A005843F2093F3301AC63F10F7A44164
:10E350002095F3A542854A064AA9608520B13285F9
:10E36000224C9CF92901C53DD0E0A522F01238F1DC
:10E3700032F00D49FF8542E642A53F85414C06F348
:10E38000A204B1328540DDD6FECAB0FABDD1FE8509
:10E39000438A0A0A0A0A0A8544AD001C299F0544DB
:10E3A0008D001CA63DA545C940F015C960F0034C81
:10E3B000B1F3A53F1869038531A90085306C3000A1
:10E3C000A9608520AD001C29FC8D001CA9A4854AEC
:10E3D000A90185224C69F9A43FB900004810102911
:10E3E000788545980A69068532981869038531A0B1
:10E3F0000084306860A25A864BA200A9528524206E
:10E4000056F550FEB8AD011CC524D03F50FEB8AD46
:10E41000011C9525E8E007D0F32097F4A004A9009B
:10E420005916008810FAC900D038A63EA5189522C2
:10E43000A545C930F01EA53E0AA8B91200C516D0E0
:10E440001EB91300C517D0174C23F4C64BD0B0A982
:10E45000022069F9A5168512A5178513A9012CA913
:10E460000B2CA9094C69F9A97F854CA519186902DB
:10E47000C5439002E543854DA205863FA2FF209348
:10E48000F3104485442901C53ED03CA000B132C5FB
:10E4900040D034A545C960F00CA00138B132E54D3B
:10E4A0001003186543C54CB01E48A545F01468C953
:10E4B000099014C90CB010854CA53FAA6903853199
:10E4C000D00568C90690F0C63F10B38A10034C9C73
:10E4D000F9863F2093F3A5454CCAF4A53048A531F1
:10E4E00048A9248530A9008531A900853420E6F7A4
:10E4F000A5558518A5548519A553851A20E6F7A5B5
:10E50000528517A553851668853168853060C90026
:10E51000F0034C6EF5200AF550FEB8AD011C9130A9
:10E52000C8D0F5A0BA50FEB8AD011C990001C8D002
:10E53000F420E0F8A538C547F005A9044C69F92096
:10E54000E9F5C53AF003A9052CA9014C69F9201099
:10E55000F54C56F5A53D0AAAB5128516B5138517D3
:10E56000A000B1328518C8B1328519A900451645F9
:10E570001745184519851A2034F9A25A2056F5A0D6
:10E580000050FEB8AD011CD92400D006C8C008D088
:10E59000F060CAD0E7A9024C69F9A9D08D0518A985
:10E5A000032C051810F12C001C30F6AD011CB8A08E
:10E5B0000060C910F0034C91F620E9F5853AAD00F2
:10E5C0001C2910D005A9084C69F9208FF72010F5F7
:10E5D000A20850FEB8CAD0FAA9FF8D031CAD0C1CCE
:10E5E000291F09C08D0C1CA9FFA2058D011CB85064
:10E5F000FEB8CAD0FAA0BBB9000150FEB88D011C0C
:10E60000C8D0F4B13050FEB88D011CC8D0F550FE12
:10E61000AD0C1C09E08D0C1CA9008D031C20F2F52B
:10E62000A43FB9000049309900004CB1F3A900A8FB
:10E630005130C8D0FB60A900852E8530854FA531AB
:10E64000854EA9018531852FA9BB8534853620E605
:10E65000F7A5528538A436A553912EC8A554912EFE
:10E66000C8A555912EC8843620E6F7A436A5529148
:10E670002EC8A553912EC8F00EA554912EC8A555AD
:10E68000912EC88436D0E1A5549130C8A55591305B
:10E69000C8843620E6F7A436A5529130C8A5539118
:10E6A00030C8A5549130C8A5559130C88436C0BB38
:10E6B00090E1A945852EA531852FA0BAB130912EC4
:10E6C00088D0F9B130912EA2BBBD00019130C8E8CD
:10E6D000D0F7865060C920F0034CCAF620E9F585D2
:10E6E0003A208FF7200AF5A0BBB9000150FEB84DC3
:10E6F000011CD015C8D0F2B13050FEB84D011CD06D
:10E7000008C8C0FDD0F14C18F4A9074C69F92010D5
:10E71000F54C18F4A9008557855AA434A55229F060
:10E720004A4A4A4AAABD7FF70A0A0A8556A55229CB
:10E730000FAABD7FF76A66576A6657290705569183
:10E7400030C8A55329F04A4A4A4AAABD7FF70A05AC
:10E75000578557A553290FAABD7FF72A2A2A2A854C
:10E76000582A290105579130C8A55429F04A4A4A28
:10E770004AAABD7FF7186A05589130C86A29808572
:10E7800059A554290FAABD7FF70A0A297C05598586
:10E7900059A55529F04A4A4A4AAABD7FF76A665ADE
:10E7A0006A665A6A665A290305599130C8D004A589
:10E7B0002F8531A555290FAABD7FF7055A9130C87D
:10E7C0008434600A0B12130E0F161709191A1B0D49
:10E7D0001D1E15A9008530852E8536A9BB8534857B
:10E7E00050A531852FA9018531A5478552A436B1A1
:10E7F0002E8553C8B12E8554C8B12E8555C8843690
:10E8000020D0F6A436B12E8552C8F011B12E855312
:10E81000C8B12E8554C8B12E8555C8D0E1A53A851A
:10E8200053A900855485554CD0F6A434B13029F84D
:10E830004A4A4A8556B13029070A0A8557C8D00680
:10E84000A54E8531A44FB13029C02A2A2A05578503
:10E8500057B130293E4A8558B13029010A0A0A0ABF
:10E860008559C8B13029F04A4A4A4A05598559B1F3
:10E8700030290F0A855AC8B1302980182A2A29015F
:10E88000055A855AB130297C4A4A855BB130290343
:10E890000A0A0A855CC8D006A54E8531A44FB1305E
:10E8A00029E02A2A2A2A055C855CB130291F855D6A
:10E8B000C88434A656BDA0F8A6571DC0F88552A638
:10E8C00058BDA0F8A6591DC0F88553A65ABDA0F89A
:10E8D000A65B1DC0F88554A65CBDA0F8A65D1DC052
:10E8E000F8855560FFFFFFFFFFFFFFFFFF8000106F
:10E8F000FFC04050FFFF2030FFF06070FF90A0B0DD
:10E90000FFD0E0FFFFFFFFFFFFFFFFFFFF08000159
:10E91000FF0C0405FFFF0203FF0F0607FF090A0BA8
:10E92000FF0D0EFFA9008534852E8536A901854E81
:10E93000A9BA854FA531852F20E6F7A5528538A4C1
:10E9400036A553912EC8A554912EC8A555912EC811
:10E95000843620E6F7A436A552912EC8F011A553AF
:10E96000912EC8A554912EC8A555912EC8D0E1A5C9
:10E9700053853AA52F853160A531852FA9008531B2
:10E98000A9248534A5398552A51A8553A51985541E
:10E99000A518855520D0F6A5178552A5168553A92B
:10E9A000008554855520D0F6A52F853160A43F9968
:10E9B0000000A550F00320F2F5208FF9A6499A4CEB
:10E9C000BEF2A9A08520AD001C09048D001CA93C45
:10E9D000854860A63EA52009108520A9FF854860CE
:10E9E000AD071C8D051CAD001C2910C51E851EF031
:10E9F00004A901851CADFE02F015C902D007A900CB
:10EA00008DFE02F00A854AA9028DFE024C2EFAA65E
:10EA10003E3007A520A8C920D0034CBEFAC648D076
:10EA20001D981004297F85202910F012AD001C29A3
:10EA3000FB8D001CA9FF853EA9008520F0DC9829EC
:10EA400040D0034CBEFA6C6200A54A100549FF187D
:10EA50006901C564B00AA93B8562A9FA8563D01231
:10EA6000E55EE55E8561A55E8560A97B8562A9FAA4
:10EA70008563A54A1031E64AAE001CCA4C69FAA566
:10EA80004AD0EFA94E8562A9FA8563A90585604C35
:10EA9000BEFAC660D06CA52029BF8520A905856275
:10EAA000A9FA85634CBEFAC64AAE001CE88A29035F
:10EAB000854BAD001C29FC054B8D001C4CBEFA3863
:10EAC000AD071CE55F8D051CC660D00CA55E85609A
:10EAD000A9978562A9FA85634C2EFAC661D0F9A977
:10EAE000A58562A9FA8563D0EFAD071C18655F8D17
:10EAF000051CC660D0E2A94E8562A9FA8563A90506
:10EB00008560AD0C1C29FD8D0C1C60A551102AA63A
:10EB10003DA9609520A90195228551A9A4854AADFA
:10EB2000001C29FC8D001CA90A8D2006A9A08D219E
:10EB300006A90F8D22064C9CF9A000D132F0059158
:10EB4000324C9CF9AD001C2910D005A9084CD3FD0E
:10EB500020A3FD20C3FDA9558D011C20C3FD20006D
:10EB6000FE2056F5A9400D0B188D0B18A9628D06D5
:10EB700018A9008D07188D0518A000A2002C001CF4
:10EB800030FB2C001C10FBAD04182C001C1011AD28
:10EB90000D180A10F5E8D0EFC8D0ECA9024CD3FD4F
:10EBA00086718472A200A000AD04182C001C3011E4
:10EBB000AD0D180A10F5E8D0EFC8D0ECA9024CD37F
:10EBC000FD388AE571AA857098E572A88571100BE9
:10EBD00049FFA88A49FFAAE8D001C898D004E004F8
:10EBE00090180670267118A5706D21068D2106A556
:10EBF000716D22068D22064C0CFBA200A000B8AD60
:10EC0000001C100E50F9B8E8D0F5C8D0F2A9034C9A
:10EC1000D3FD8A0A8D2506982A8D2406A9BF2D0BBF
:10EC2000188D0B18A9668D2606A643A00098186DAE
:10EC300026069001C8C8CAD0F549FF386900186D8A
:10EC40002506B003CE2406AA9849FF386900186D3E
:10EC500024061005A9044CD3FDA88AA20038E54378
:10EC6000B003883003E8D0F58E2606E004B005A98D
:10EC7000054CD3FD1865438D2706A9008D2806A0F5
:10EC800000A63DA539990003C8C8AD280699000320
:10EC9000C8A551990003C8B513990003C8B51299C6
:10ECA0000003C8A90F990003C8990003C8A9005917
:10ECB000FA0259FB0259FC0259FD0299F902EE28A9
:10ECC00006AD2806C54390BB9848E88A9D0005E834
:10ECD000D0FAA90385312030FE68A88820E5FD2000
:10ECE000F5FDA905853120E9F5853A208FF7A900C2
:10ECF0008532200EFEA9FF8D011CA20550FEB8CA68
:10ED0000D0FAA20AA43250FEB8B900038D011CC883
:10ED1000CAD0F3A20850FEB8A9558D011CCAD0F57F
:10ED2000A9FFA20550FEB88D011CCAD0F7A2BB50A6
:10ED3000FEB8BD00018D011CE8D0F4A00050FEB863
:10ED4000B1308D011CC8D0F5A955AE260650FEB8CD
:10ED50008D011CCAD0F7A53218690A8532CE280663
:10ED6000D09350FEB850FEB82000FEA9C88D2306EF
:10ED7000A9008530A9038531A5438D28062056F5C5
:10ED8000A20AA00050FEB8AD011CD130D00EC8CAF6
:10ED9000D0F218A530690A85304C62FDCE2306D02A
:10EDA000CFA9064CD3FD2056F5A0BB50FEB8AD014F
:10EDB0001CD90001D0E6C8D0F2A2FC50FEB8AD01CB
:10EDC0001CD90005D0D6C8CAD0F1CE2806D0AEE6F0
:10EDD00051A551C924B0034C9CF9A9FF8551A90044
:10EDE0008550A9014C69F9AD0C1C291F09C08D0C77
:10EDF0001CA9FF8D031C8D011CA228A00050FEB889
:10EE000088D0FACAD0F760AE2106AC220650FEB810
:10EE1000CAD0FA8810F760CE2006F0034C9CF9A007
:10EE2000FF8451C884504C69F9B90003994503889F
:10EE3000D0F7AD00038D450360A044B9BB0191300C
:10EE40008810F860AD0C1C09E08D0C1CA9008D0326
:10EE50001C60AD0C1C291F09C08D0C1CA9FF8D0363
:10EE60001CA9558D011CA228A00050FEB888D0FA1C
:10EE7000CAD0F760A9008530852E8536A9BB8534B8
:10EE8000A531852FA9018531A436B12E8552C8B18F
:10EE90002E8553C8B12E8554C8B12E8555C8F008AB
:10EEA000843620D0F64C44FE4CD0F6488A48984828
:10EEB000AD0D182902F0032053E8AD0D1C0A100314
:10EEC00020B0F268A868AA68401204049056494429
:10EED0004D425550264352534E8405C1F81B5C07E2
:10EEE000A3F088230DEDD0C8CACCCBE2E7C8CAC8CE
:10EEF000EE51DD1C9E1C5257414D445350554C441D
:10EF00005350555245455253454C5147524C0800B9
:10EF1000003F7FBFFF111213154104241F19120176
:10EF2000FFFF0100030405060707106C65008D0054
:10EF30001C8D021C4C7DEA8AA205CAD0FDAA602065
:10EF4000AEE94C9CE9AD0202C92DF00538E92BD0A1
:10EF5000DA852360AAAAAAAAAAAAAAAAAAAAAAAAD7
:10EF6000AAAAAAAAAAAAAAAAAAAAAAAAAAAAAAAA01
:10EF7000AAAAAAAAAAAAAAAAAAAAAAAAAAAAAAAAF1
:10EF8000AAAAAAAAAAAAAAAAAAAAAAAAAAAAAAAAE1
:10EF9000AAAAAAAAAAAAAAAAAAAAAAAAAAAAAAAAD1
:10EFA000AAAAAAAAAAAAAAAAAAAAAAAAAAAAAAAAC1
:10EFB000AAAAAAAAAAAAAAAAAAAAAAAAAAAAAAAAB1
:10EFC000AAAAAAAAAAAAAAAAAAAAAAAAAAAAAAAAA1
:10EFD000AAAAAAAAAAAAAAAAAAAAAAAAAAAAAAAA91
:10EFE000AAAAAAAAAAAAAAAAAAAAAAAAAAAAAAAA81
:10EFF000AAAAAAAAAAAAAAAAAAAAAAAAAAAAAAAA71
:10F00000AAAAAAAAAAAAAAAAAAAAAAAAAAAAAAAA60
:10F01000AAAAAAAAAAAAAAAAAAAAAAAAAAAAAAAA50
:10F02000AAAAAAAAAAAA525352AAC6C88FF95FCD01
:10F0300097CD00050305060509050C050F0501FF21
:10F04000A0EA67FE64F000080000002090080000BD
:10F050004A9E000858F60008900800207836010003
:10F06000689F0008D1847A030A400A01020304065B
:10F07000070809B41916021BFF32019AF038693CDF
:10F080001144140140137F4D1408874F1B082508B5
:10F0900013535214086383140897581C08415A18D4
:10F0A00019041B6B5C181A5D10125E1C0839811064
:10F0B0001920134561140851641B08D30413036815
:10F0C0004C085B69401ABD0829401B2D6F1812714E
:10F0D0001B084F041397731B08FD041B755F284A18
:10F0E00074401B53794C127D1B08C7041AC3381A8D
:10F0F000D37829401A730813AB571B08C1801AE74D
:10F100007C1A9F041A7F801A79805A85801A774862
:10F110001A8F80131B651B08E5801A2F804BA76A86
:10F12000401A590829801A5F801AB77C1A83041A7A
:10F13000A17C1AFB7829805AAB801AB1801B2F7EE4
:10F140001819801AE5384B2753401AB38029401A02
:10F15000EB8013315B1B08CF801A95801A9F801AB1
:10F16000BB801A6F801ABF481AD9801A9D801A096D
:10F17000041A59804B096B405A0B801A918013096D
:10F18000721B0869801AAB804B5975805A83801BAB
:10F190000F7AFC19801AE18013094E5B087B805AB4
:10F1A00093801315591B086D801AB7801AA9801A0D
:10F1B000C5801AE1801AA3801AC548132362140877
:10F1C00017661408F7641B0885805A6B80293C2950
:10F1D000041AD1801A4B801A9D801AB9805AB780C0
:10F1E0005AD3801A6D801B4F7F68198429301ABB4F
:10F1F0008029081AF70813D1571B082D801ABD80E3
:10F200001AD3701AD180291C1A1B401B6982681AF4
:10F2100060D019801AA1801AE7201AAF809AC7809F
:10F2200013AD6E1B08F1801AA1801AB9041AC380AD
:10F230001301764C08E5787C29041AB780690C1311
:10F24000274E140835541B0867781A85081301588F
:10F250001B085D801AED801A1D701AF38013D75DAC
:10F260001B0837801A45101A57801A8B801AD380D2
:10F270001A8F101ADB804B036C801A61081AE38026
:10F280001309701B08D57C1A037C1ADF041A398015
:10F290001AEB801A93081307791B08EF801BF57F80
:10F2A0005819401A49801AD77829BC1BD75690198B
:10F2B000801A83801A13781AF3081A0F7C1AF9043B
:10F2C0001A53801A25241A9D801AD18013196714A5
:10F2D00008CB63140805695B08C1801A057C2948BE
:10F2E0001A37801A33781ABD081AE9081AF5781AFD
:10F2F00075401A3F8429F413497B1C084180901AF9
:10F300007C6C19801A2D7829381A6D081A5F801ABA
:10F31000BD781A3F801AD5081A317C4B2F5E4029E0
:10F32000081AF1801A25781A95801A5B081A31801C
:10F330004B356D801A830829481A79781A65781A2E
:10F3400099081AF3084B6577401AAF0829801AB953
:10F35000801ABD801A1180C1181542524B204F529D
:10F3600041313F3F3F20534C4F314E4F5032101EE2
:10F370003241534C32102D32504850201A33101E57
:10F3800034414E4333201A35101A35101A35201ED9
:10F390003542504C52105A36401A36201A37101A3D
:10F3A00037201A37102D37434C43401A381829207C
:10F3B00029081A39101A39201A39103809394A53CC
:10F3C0005235414E44801809524C41314249543221
:10F3D000101E32524F4C32101E32504C5020101A18
:10F3E00033103980192029301A35101A35201E356E
:10F3F000424D49521039801910398019101A37209E
:10F400001A37102D37534543403980191039801968
:10F41000101A39201A391038093952544920454FE9
:10F4200052801D53524531201A32101E324C535215
:10F4300032102D32504841201A3310180A34414CF2
:10F4400052334A4D5035101A35101A35201E3542A8
:10F450005643521039801910398019101A37201A62
:10F4600037103C37434C6039801910398019101A15
:10F4700039201A391019803E5320414443803C52B0
:10F4800052418019101B32528419102D32504C41B8
:10F49000201A33103C344152801A30101A35101A99
:10F4A000352019801B5352103980191039801910DA
:10F4B0001A37201A37102D37534549403980191013
:10F4C000398019101A39201A39101A39103C33535F
:10F4D0005478180A3353415831535459321019048F
:10F4E0001B5832102E32444559203C1808545841BC
:10F4F000205841412C1B59352019041B5835201E1A
:10F5000035424343521039803B4148401A37101965
:10F51000041B5859201E375459412010180E3854D6
:10F520005853205441533853485939101E395348C1
:10F53000583830180F384C4459334C4441314C44FE
:10F5400058334C8019101A321019041B5832101EEF
:10F550003254415920101E335441582010192C1B8D
:10F5600059351019041B58351019801B5352103986
:10F570008019101A36201A371019041B5859102DEB
:10F5800037434C56402C385453402A53701A391084
:10F590001904197C180C41583843505933434D50C5
:10F5A00031E41E3344435031101A321019F8180B4D
:10F5B000433244504332494E592010180A334445CF
:10F5C000582053425833201A35101A35201A353036
:10F5D0001E35424E455210398019101A36482930CE
:10F5E0001A37201A37402D36434C44102A38181940
:10F5F0001029081A39101A39201A393038093943B4
:10F60000505833534243801C495342801B58321098
:10F61000197819041B53420829782B4333402908D1
:10F6200019201A35081A35201A35201E3542455141
:10F63000521039801910398019101A37201A3710D2
:10F640002D375345441039801910398019101A3953
:08F65000201A3910031F3901D3
:020000041000EA
:1000000001FF01FF01FF01FF01FF01FF01FF01FFF0
:1000100001FF01FF01FF01FF01FF01FF01FF01FFE0
:1000200001FF01FF01FF01FF01FF01FF01FF01FFD0
:1000300001FF01FF01FF01FF01FF01FF01FF01FFC0
:1000400001FF01FF01FF01FF01FF01FF01FF01FFB0
:1000500001FF01FF01FF01FF01FF01FF01FF01FFA0
:1000600001FF01FF01FF01FF01FF01FF01FF01FF90
:1000700001FF01FF01FF01FF01FF01FF01FF01FF80
:1000800001FF01FF01FF01FF01FF01FF01FF01FF70
:1000900001FF01FF01FF01FF01FF01FF01FF01FF60
:1000A00001FF01FF01FF01FF01FF01FF01FF01FF50
:1000B00001FF01FF01FF01FF01FF01FF01FF01FF40
:1000C00001FF01FF01FF01FF01FF01FF01FF01FF30
:1000D00001FF01FF01FF01FF01FF01FF01FF01FF20
:1000E00001FF01FF01FF01FF01FF01FF01FF01FF10
:1000F00001FF01FF01FF01FF01FF01FF01FF01FF00
:1001000001FF01FF01FF01FF01FF01FF01FF01FFEF
:1001100001FF01FF01FF01FF01FF01FF01FF01FFDF
:1001200001FF01FF01FF01FF01FF01FF01FF01FFCF
:1001300001FF01FF01FF01FF01FF01FF01FF01FFBF
:1001400001FF01FF01FF01FF01FF01FF01FF01FFAF
:1001500001FF01FF01FF01FF01FF01FF01FF01FF9F
:1001600001FF01FF01FF01FF01FF01FF01FF01FF8F
:1001700001FF01FF01FF01FF01FF01FF01FF01FF7F
:1001800001FF01FF01FF01FF01FF01FF01FF01FF6F
:1001900001FF01FF01FF01FF01FF01FF01FF01FF5F
:1001A00001FF01FF01FF01FF01FF01FF01FF01FF4F
:1001B00001FF01FF01FF01FF01FF01FF01FF01FF3F
:1001C00001FF01FF01FF01FF01FF01FF01FF01FF2F
:1001D00001FF01FF01FF01FF01FF01FF01FF01FF1F
:1001E00001FF01FF01FF01FF01FF01FF01FF01FF0F
:1001F00001FF01FF01FF01FF01FF01FF01FF01FFFF
:0402000001FF1100E9
:040000050800018965
:00000001FF
